:020000040800F2
:10000000005000208932000839330008B14400084C
:100010003933000839330008393300080000000084
:10002000000000000000000000000000393300085C
:10003000393300080000000039330008596900080E
:1000400039330008393300083933000839330008E0
:10005000393300083933000839330008F92500081E
:1000600039330008393300083933000839330008C0
:1000700039330008393300080D68000839330008A7
:1000800039330008393300083933000839330008A0
:10009000393300083933000839330008FD250008DA
:1000A0003933000839330008393300085D3200085D
:1000B00069320008713200087D320008C15F000813
:1000C00041630008C55F00083D630008393300083C
:1000D00039330008416800087D680008393300089A
:1000E0005D1C0008393300083933000800000000A7
:1000F0000000000000000000000000000000000000
:0C01000000000000000000005FF808F1A3
:1001100010B5054C237833B9044810B10448AFF347
:1001200000800121217010BDB405002000000000F6
:10013000BC35010808B5064B1BB106480649AFF3AC
:1001400000800648016811B1054A02B1904708BD18
:1001500000000000BC350108B8050020B4050020EF
:100160000000000081F0004102E000BF83F0004386
:1001700030B54FEA41044FEA430594EA050F08BF42
:1001800090EA020F1FBF54EA000C55EA020C7FEA06
:10019000645C7FEA655C00F0E2804FEA5454D4EB83
:1001A0005555B8BF6D420CDD2C4480EA020281EA4D
:1001B000030382EA000083EA010180EA020281EA85
:1001C0000303362D88BF30BD11F0004F4FEA0131D7
:1001D0004FF4801C4CEA113102D0404261EB4101E6
:1001E00013F0004F4FEA03334CEA133302D052426C
:1001F00063EB430394EA050F00F0A780A4F1010428
:10020000D5F1200E0DDB02FA0EFC22FA05F2801861
:1002100041F1000103FA0EF2801843FA05F3594147
:100220000EE0A5F120050EF1200E012A03FA0EFCC6
:1002300028BF4CF0020C43FA05F3C01851EBE371F0
:1002400001F0004507D54FF0000EDCF1000C7EEB0D
:1002500000006EEB0101B1F5801F1BD3B1F5001F4B
:100260000CD349085FEA30004FEA3C0C04F101046A
:100270004FEA445212F5800F80F09A80BCF1004F93
:1002800008BF5FEA500C50F1000041EB045141EA15
:10029000050130BD5FEA4C0C404141EB010111F416
:1002A000801FA4F10104E9D191F0000F04BF0146C1
:1002B0000020B1FA81F308BF2033A3F10B03B3F19F
:1002C00020020CDA0C3208DD02F1140CC2F10C022F
:1002D00001FA0CF021FA02F10CE002F11402D8BF8D
:1002E000C2F1200C01FA02F120FA0CFCDCBF41EA59
:1002F0000C019040E41AA2BF01EB0451294330BD28
:100300006FEA04041F3C1CDA0C340EDC04F1140404
:10031000C4F1200220FA04F001FA02F340EA0300DB
:1003200021FA04F345EA030130BDC4F10C04C4F121
:10033000200220FA02F001FA04F340EA0300294601
:1003400030BD21FA04F0294630BD94F0000F83F44B
:10035000801306BF81F480110134013D4EE77FEA2E
:10036000645C18BF7FEA655C29D094EA050F08BF7A
:1003700090EA020F05D054EA000C04BF194610465B
:1003800030BD91EA030F1EBF0021002030BD5FEA9F
:10039000545C05D14000494128BF41F0004130BDC7
:1003A00014F580043CBF01F5801130BD01F000451B
:1003B00045F0FE4141F470014FF0000030BD7FEA8E
:1003C000645C1ABF194610467FEA655C1CBF0B4689
:1003D000024650EA013406BF52EA033591EA030FA0
:1003E00041F4002130BD00BF90F0000F04BF002198
:1003F000704730B54FF4806404F132044FF00005CB
:100400004FF0000150E700BF90F0000F04BF002143
:10041000704730B54FF4806404F1320410F00045A9
:1004200048BF40424FF000013EE700BF42004FEAA4
:10043000E2014FEA31014FEA02701FBF12F07F4321
:1004400093F07F4F81F06051704792F0000F14BF1E
:1004500093F07F4F704730B54FF4607401F0004562
:1004600021F0004120E700BF50EA010208BF7047B9
:1004700030B54FF000050AE050EA010208BF7047AE
:1004800030B511F0004502D5404261EB41014FF417
:10049000806404F132045FEA915C3FF4DCAE4FF01B
:1004A00003025FEADC0C18BF03325FEADC0C18BF02
:1004B000033202EBDC02C2F1200300FA03FC20FA53
:1004C00002F001FA03FE40EA0E0021FA02F11444A0
:1004D000C1E600BF70B54FF0FF0C4CF4E06C1CEAB5
:1004E00011541DBF1CEA135594EA0C0F95EA0C0F2A
:1004F00000F0DEF82C4481EA030621EA4C5123EA9D
:100500004C5350EA013518BF52EA033541F48011CB
:1005100043F4801338D0A0FB02CE4FF00005E1FB7E
:1005200002E506F00042E0FB03E54FF00006E1FBC8
:1005300003569CF0000F18BF4EF0010EA4F1FF040B
:10054000B6F5007F64F5407404D25FEA4E0E6D414B
:1005500046EB060642EAC62141EA55514FEAC5205C
:1005600040EA5E504FEACE2EB4F1FD0C88BFBCF5D8
:10057000E06F1ED8BEF1004F08BF5FEA500E50F189
:10058000000041EB045170BD06F0004646EA01014F
:1005900040EA020081EA0301B4EB5C04C2BFD4EB81
:1005A0000C0541EA045170BD41F480114FF0000E7A
:1005B000013C00F3AB8014F1360FDEBF002001F0E8
:1005C000004170BDC4F10004203C35DA0C341BDC62
:1005D00004F11404C4F1200500FA05F320FA04F034
:1005E00001FA05F240EA020001F0004221F0004168
:1005F00010EBD37021FA04F642EB06015EEA430EDB
:1006000008BF20EAD37070BDC4F10C04C4F120050A
:1006100000FA04F320FA05F001FA04F240EA0200BD
:1006200001F0004110EBD37041F100015EEA430E8E
:1006300008BF20EAD37070BDC4F1200500FA05F2AE
:100640004EEA020E20FA04F301FA05F243EA02032D
:1006500021FA04F001F0004121FA04F220EA02003C
:1006600000EBD3705EEA430E08BF20EAD37070BD82
:1006700094F0000F0FD101F00046400041EB010162
:1006800011F4801F08BF013CF7D041EA060195F044
:10069000000F18BF704703F00046520043EB0303FE
:1006A00013F4801F08BF013DF7D043EA06037047EB
:1006B00094EA0C0F0CEA135518BF95EA0C0F0CD0F6
:1006C00050EA410618BF52EA4306D1D181EA03013C
:1006D00001F000414FF0000070BD50EA410606BF36
:1006E0001046194652EA430619D094EA0C0F02D17B
:1006F00050EA013613D195EA0C0F05D152EA0336C0
:100700001CBF104619460AD181EA030101F00041DD
:1007100041F0FE4141F470014FF0000070BD41F026
:10072000FE4141F4780170BD70B54FF0FF0C4CF400
:10073000E06C1CEA11541DBF1CEA135594EA0C0F1F
:1007400095EA0C0F00F0A7F8A4EB050481EA030E6C
:1007500052EA03354FEA013100F088804FEA033353
:100760004FF0805545EA131343EA12634FEA022221
:1007700045EA111545EA10654FEA00260EF00041E2
:100780009D4208BF964244F1FD0404F5407402D234
:100790005B084FEA3202B61A65EB03055B084FEAC5
:1007A00032024FF480104FF4002CB6EB020E75EBC2
:1007B000030E22BFB61A754640EA0C005B084FEAEA
:1007C0003202B6EB020E75EB030E22BFB61A754667
:1007D00040EA5C005B084FEA3202B6EB020E75EBB2
:1007E000030E22BFB61A754640EA9C005B084FEA2A
:1007F0003202B6EB020E75EB030E22BFB61A754637
:1008000040EADC0055EA060E18D04FEA051545EA25
:1008100016754FEA06164FEAC30343EA52734FEACE
:10082000C2025FEA1C1CC0D111F4801F0BD141EA47
:1008300000014FF000004FF0004CB6E711F4801FAC
:1008400004BF01430020B4F1FD0C88BFBCF5E06F8C
:100850003FF6AFAEB5EB030C04BFB6EB020C5FEA9C
:10086000500C50F1000041EB045170BD0EF0004EF1
:100870004EEA113114EB5C04C2BFD4EB0C0541EA23
:10088000045170BD41F480114FF0000E013C90E620
:1008900045EA060E8DE60CEA135594EA0C0F08BFE4
:1008A00095EA0C0F3FF43BAF94EA0C0F0AD150EAE3
:1008B00001347FF434AF95EA0C0F7FF425AF104676
:1008C00019462CE795EA0C0F06D152EA03353FF49E
:1008D000FDAE1046194622E750EA410618BF52EA1B
:1008E00043067FF4C5AE50EA41047FF40DAF52EAEF
:1008F00043057FF4EBAE12E74FF0FF3C06E000BF8C
:100900004FF0010C02E000BF4FF0010C4DF804CD98
:100910004FEA410C7FEA6C5C4FEA430C18BF7FEA58
:100920006C5C1BD001B050EA410C0CBF52EA430C86
:1009300091EA030F02BF90EA020F0020704710F106
:10094000000F91EA030F58BF994208BF90422CBF95
:10095000D8176FEAE37040F0010070474FEA410C8E
:100960007FEA6C5C02D150EA013C07D14FEA430CAC
:100970007FEA6C5CD6D152EA033CD3D05DF8040B1D
:10098000704700BF8446104662468C46194663464F
:1009900000E000BF01B5FFF7B7FF002848BF10F126
:1009A000000F01BD4DF808EDFFF7F4FF0CBF01206B
:1009B00000205DF808FB00BF4DF808EDFFF7EAFFE7
:1009C00034BF012000205DF808FB00BF4DF808EDA2
:1009D000FFF7E0FF94BF012000205DF808FB00BF97
:1009E0004DF808EDFFF7CEFF94BF012000205DF821
:1009F00008FB00BF4DF808EDFFF7C4FF34BF01202E
:100A000000205DF808FB00BF4FEA4102B2F1E0436D
:100A100024BFB3F5001CDCF1FE5C0DD901F0004CE5
:100A20004FEAC0024CEA5070B2F1004F40EB830035
:100A300008BF20F00100704711F0804F21D113F161
:100A40003872BCBF01F00040704741F480114FEA9A
:100A50005252C2F11802C2F1200C10FA0CF320FA23
:100A600002F018BF40F001004FEAC1234FEAD32340
:100A700003FA0CFC40EA0C0023FA02F34FEA4303AA
:100A8000CCE77FEA625307D150EA01331EBF4FF033
:100A9000FE4040F44000704701F0004040F0FE404E
:100AA00040F40000704700BF80F0004002E000BF4B
:100AB00081F0004142001FBF5FEA410392EA030F49
:100AC0007FEA226C7FEA236C6AD04FEA1262D2EB93
:100AD0001363C1BFD218414048404140B8BF5B4298
:100AE000192B88BF704710F0004F40F4000020F031
:100AF0007F4018BF404211F0004F41F4000121F047
:100B00007F4118BF494292EA030F3FD0A2F1010290
:100B100041FA03FC10EB0C00C3F1200301FA03F1CE
:100B200000F0004302D5494260EB4000B0F5000FF1
:100B300013D3B0F1807F06D340084FEA310102F1B0
:100B40000102FE2A51D2B1F1004F40EBC25008BF62
:100B500020F0010040EA03007047490040EB00002C
:100B600010F4000FA2F10102EDD1B0FA80FCACF15B
:100B7000080CB2EB0C0200FA0CF0AABF00EBC2505A
:100B800052421843BCBFD0401843704792F0000F48
:100B900081F4000106BF80F400000132013BB5E79B
:100BA0004FEA41037FEA226C18BF7FEA236C21D011
:100BB00092EA030F04D092F0000F08BF0846704776
:100BC00090EA010F1CBF0020704712F07F4F04D144
:100BD000400028BF40F00040704712F100723CBF57
:100BE00000F50000704700F0004343F0FE4040F481
:100BF000000070477FEA226216BF08467FEA23633F
:100C00000146420206BF5FEA412390EA010F40F429
:100C1000800070474FF0000304E000BF10F0004375
:100C200048BF40425FEA000C08BF704743F096435C
:100C300001464FF000001CE050EA010208BF704777
:100C40004FF000030AE000BF50EA010208BF7047FE
:100C500011F0004302D5404261EB41015FEA010C13
:100C600002BF84460146002043F0B64308BFA3F10B
:100C70008053A3F50003BCFA8CF2083AA3EBC253ED
:100C800010DB01FA02FC634400FA02FCC2F120020C
:100C9000BCF1004F20FA02F243EB020008BF20F043
:100CA0000100704702F1200201FA02FCC2F12002A9
:100CB00050EA4C0021FA02F243EB020008BF20EA9E
:100CC000DC7070474FF0FF0C1CEAD0521EBF1CEACC
:100CD000D15392EA0C0F93EA0C0F6FD01A4480EABA
:100CE000010C400218BF5FEA41211ED04FF00063A3
:100CF00043EA501043EA5111A0FB01310CF00040CF
:100D0000B1F5000F3EBF490041EAD3715B0040EAF4
:100D1000010062F17F02FD2A1DD8B3F1004F40EBC4
:100D2000C25008BF20F00100704790F0000F0CF097
:100D3000004C08BF49024CEA502040EA51207F3A5B
:100D4000C2BFD2F1FF0340EAC250704740F4000036
:100D50004FF00003013A5DDC12F1190FDCBF00F027
:100D600000407047C2F10002410021FA02F1C2F1D5
:100D7000200200FA02FC5FEA310040F1000053EA71
:100D80004C0308BF20EADC70704792F0000F00F0BF
:100D9000004C02BF400010F4000F013AF9D040EAC5
:100DA0000C0093F0000F01F0004C02BF490011F459
:100DB000000F013BF9D041EA0C018FE70CEAD15357
:100DC00092EA0C0F18BF93EA0C0F0AD030F0004CD7
:100DD00018BF31F0004CD8D180EA010000F000408B
:100DE000704790F0000F17BF90F0004F084691F049
:100DF000000F91F0004F14D092EA0C0F01D1420283
:100E00000FD193EA0C0F03D14B0218BF084608D14B
:100E100080EA010000F0004040F0FE4040F4000095
:100E2000704740F0FE4040F4400070474FF0FF0C28
:100E30001CEAD0521EBF1CEAD15392EA0C0F93EA6F
:100E40000C0F69D0A2EB030280EA010C49024FEAC1
:100E5000402037D04FF0805343EA111143EA10137A
:100E60000CF000408B4238BF5B0042F17D024FF432
:100E7000000C8B4224BF5B1A40EA0C00B3EB510F0D
:100E800024BFA3EB510340EA5C00B3EB910F24BFF6
:100E9000A3EB910340EA9C00B3EBD10F24BFA3EB7B
:100EA000D10340EADC001B0118BF5FEA1C1CE0D143
:100EB000FD2A3FF650AF8B4240EBC25008BF20F0F6
:100EC000010070470CF0004C4CEA50207F32C2BF4A
:100ED000D2F1FF0340EAC250704740F400004FF0E7
:100EE0000003013A37E792F0000F00F0004C02BF18
:100EF000400010F4000F013AF9D040EA0C0093F0E2
:100F0000000F01F0004C02BF490011F4000F013B3B
:100F1000F9D041EA0C0195E70CEAD15392EA0C0FA3
:100F200008D142027FF47DAF93EA0C0F7FF470AFDB
:100F3000084676E793EA0C0F04D14B023FF44CAF1E
:100F400008466EE730F0004C18BF31F0004CCAD1B3
:100F500030F000427FF45CAF31F000437FF43CAFEF
:100F60005FE700BF4FF0FF3C06E000BF4FF0010C11
:100F700002E000BF4FF0010C4DF804CD4FEA4002F3
:100F80004FEA41037FEA226C18BF7FEA236C11D03D
:100F900001B052EA530C18BF90EA010F58BFB2EBF0
:100FA000030088BFC81738BF6FEAE17018BF40F070
:100FB000010070477FEA226C02D15FEA402C05D124
:100FC0007FEA236CE4D15FEA412CE1D05DF8040BA9
:100FD000704700BF844608466146FFE70FB5FFF73C
:100FE000C9FF002848BF10F1000F0FBD4DF808EDF4
:100FF000FFF7F4FF0CBF012000205DF808FB00BFE5
:101000004DF808EDFFF7EAFF34BF012000205DF83E
:1010100008FB00BF4DF808EDFFF7E0FF94BF01208B
:1010200000205DF808FB00BF4DF808EDFFF7D2FF88
:1010300094BF012000205DF808FB00BF4DF808EDCB
:10104000FFF7C8FF34BF012000205DF808FB00BF98
:101050004FEA4002B2F1FE4F0FD34FF09E03B3EBC5
:1010600012620DD94FEA002343F0004310F0004F05
:1010700023FA02F018BF404270474FF0000070475B
:1010800012F1610F01D1420205D110F0004008BFFA
:101090006FF0004070474FF00000704742000ED2E2
:1010A000B2F1FE4F0BD34FF09E03B3EB126209D4A3
:1010B0004FEA002343F0004323FA02F070474FF059
:1010C0000000704712F1610F01D1420202D14FF0CE
:1010D000FF3070474FF00000704700BF2DE9FF411F
:1010E000334B8046187800283BD0002425462646FE
:1010F0002746082232210DEB0203532004F0FCFFA7
:101100009DF809109DF80800013400EB01239DF8BB
:101110000B109DF80A001AB200EB01239DF80D1088
:101120009DF80C00E4B2BF181AB200EB01239DF841
:101130000F10B618202C1AB2154401F07F0001D010
:101140000028D6D11B4B97FBF4F796FBF4F695FBE2
:10115000F4F5ADF80070ADF80260ADF804501C7005
:101160001DE03221062202AB532004F0C5FF9DF89A
:1011700009209DF808109DF80B0001EB02239DF853
:101180000A20ADF8003002EB00219DF80C309DF8EC
:101190000D00ADF8021003EB0022ADF80420064A62
:1011A00068464146127802F0EDF9BDE8FF8100BFC4
:1011B000D0050020D105002000000020154B10B5FF
:1011C0001B7804462D21532008227BB105F058F8E6
:1011D00031210A22532005F053F82C210C225320F0
:1011E00005F04EF853203821902209E005F048F828
:1011F00031210A22532005F043F853202C210A22E2
:1012000005F03EF8044840F2091202800CB103498F
:101210000C7010BDD005002026000020000000202A
:1012200037B5104B05461A680F480C46002182421C
:101230008DF8071001D1002013E0532001220DF199
:10124000070304F059FF0028F5D09DF80710E529A1
:10125000F1D12A780548064B064920601A70616072
:1012600001203EBD60010020001BB700BD11000839
:10127000D0050020DD1000081FB50446022106221B
:101280006B46182004F038FF9DF800309DF80120CF
:1012900098089DF8023000EB02219DF80320980881
:1012A0009DF80430ADF8081000EB02219DF80520F0
:1012B0009808ADF80A1000EB0221044AADF80C10B2
:1012C00002A82146127802F05DF91FBD010000203E
:1012D00010B50F2108220446182004F0D1FF0E2279
:1012E0001820102104F0CCFF034B4FF480521A80D9
:1012F0000CB10248047010BD26000020010000203F
:1013000037B5002402AB054603F8014D18202146ED
:10131000012204F0F1FE50B19DF80730FB2B05D1FE
:101320000348044928606960012000E020463EBD72
:10133000D1120008791200081FB50446A821062220
:101340006B46682004F0D8FE9DF800209DF801301F
:1013500043EA022001B2042391FBF3F29DF802005C
:101360009DF80310ADF8082041EA002210B290FB6E
:10137000F3F19DF805209DF80400ADF80A1042EA4B
:101380000021064A08B290FBF3F3214602A8127826
:10139000ADF80C3002F0F6F81FBD00BF02000020CF
:1013A00010B50446642005F00AFB68202321F022D2
:1013B00004F066FF10B9032005F09EFB052005F040
:1013C000FEFA064B68201A78202142F00F0204F042
:1013D00057FF0CB10248047010BD00BFD2050020B9
:1013E0000200002037B5054619200C4605F0E7FA43
:1013F00068200F2101220DF1070304F07DFE9DF806
:101400000730D32B16D10C480C490D4A4E2C2860BE
:101410006960EA600B4B07D05D2C09D0362C01D0F7
:10142000002002E0402000E080201870012002E04F
:10143000C020FAE700203EBDA113000839130008C0
:10144000DDE9A731D20500201FB50446012106229F
:101450006B461C2004F050FE9DF800209DF80130E2
:1014600043EA022040F38D01042391FBF3F29DF83F
:1014700002009DF80310ADF8082041EA002242F373
:101480008D0090FBF3F19DF805209DF80400ADF868
:101490000A1042EA0021064A41F38D0090FBF3F363
:1014A000214602A81278ADF80C3002F06BF81FBD8F
:1014B0000300002037B50421202302248DF80610F4
:1014C000054669441B48ADF804308DF8074004F028
:1014D0003FFF2A2100221C2004F0D2FE0E211C20F6
:1014E000224604F0CDFE0F2103221C2004F0C8FE8A
:1014F0002B2112221C2004F0C3FE2C211C2022468A
:1015000004F0BEFE2D2101221C2004F0B9FE2E2184
:1015100000221C2004F0B4FE05221C202A2104F025
:10152000AFFE05484FF4807202800DB1034B1D7071
:101530003EBD00BF0008014026000020030000203F
:1015400013B5044610481149026800238A428DF8F9
:10155000073001D1002015E01C200D2101220DF1E2
:10156000070304F0C9FD0028F4D09DF807302A2BAA
:1015700001D01A2BEED10648064A07492060626066
:101580000B7001201CBD00BF60010020001BB700D4
:10159000B514000849140008D305002013B5022231
:1015A00004461B2101AB682004F0A6FD9DF8042031
:1015B0009DF8053043EA022000F54E5110314FF4FA
:1015C0008C7291FBF2F3233323801CBD1FB50446BC
:1015D0001D2106226B46682004F08EFD9DF8002038
:1015E0009DF8013043EA022001B2042391FBF3F29B
:1015F0009DF802009DF80310ADF8082041EA002292
:1016000010B290FBF3F19DF805209DF80400ADF8B1
:101610000A1042EA0021064A08B290FBF3F3214681
:1016200002A81278ADF80C3001F0ACFF1FBD00BF6E
:101630000500002010B50446192005F0C0F9682007
:101640001521002204F01CFE10B9032005F054FA05
:101650000D4B16211A78682042F0180204F010FE93
:1016600017210022682004F00BFE3D210122682092
:1016700004F006FE68203E21012204F001FE0CB1B8
:101680000248047010BD00BF0400002005000020C7
:1016900038B5054619200C4605F091F9682015214A
:1016A000002204F0EDFD18B3124B13481349144AFD
:1016B000622C2B606860A960EA60124B0FD004D8DE
:1016C0000A2C12D0142C0CD10DE0BC2C04D0B4F593
:1016D000807F06D1002009E00120187038BD02206B
:1016E00004E0032002E0042000E00520187001203F
:1016F00038BD00BF35160008CD1500089D1500083F
:101700001844923104000020074B197821B10129B7
:1017100006D14FF4805201E04FF40062034B1A806F
:1017200008B1034908707047D40500202600002046
:10173000060000201FB50446432106226B466820A0
:1017400004F0DAFC9DF800209DF8013043EA022005
:1017500001B2042391FBF3F29DF802009DF80310FF
:10176000ADF8082041EA002210B290FBF3F19DF899
:1017700005209DF80400ADF80A1042EA0021064A4F
:1017800008B290FBF3F3214602A81278ADF80C30B2
:1017900001F0F8FE1FBD00BF080000201FB5044681
:1017A0003B2106226B46682004F0A6FC9DF8002031
:1017B0009DF801309DF8021043EA02209DF80320B5
:1017C000ADF8080042EA01239DF804009DF80510D9
:1017D000ADF80A30054B41EA0022ADF80C2002A812
:1017E00021461A7801F0CEFE1FBD00BF0600002082
:1017F00013B5224A4FF4005304460220ADF80430DA
:101800008DF8070013681E48042183428DF80610E6
:1018100001D11C4803E01C498B4203D11B4801A99C
:1018200004F096FD6B218022682004F029FD05203C
:1018300005F0C5F819210022682004F021FD6B2174
:101840000322682004F01CFD37210222682004F0E6
:1018500017FD0F4A1A211278682004F011FD1B2190
:101860001822682004F00CFD68201C21102204F0CE
:1018700007FD0CB1074B1C701CBD00BF60010020B0
:1018800000127A00000C0140001BB700001001405C
:1018900007000020080000202DE9FF410646232014
:1018A0000D46144605F08BF86820752101220DF1D4
:1018B000070304F021FC00286DD09DF80780B8F1E3
:1018C000680F67D106210A4602AB404604F014FCBB
:1018D0009DF80B309DF80D7003F0010107F0010039
:1018E0004A0042EA80079DF8090000F001031F4307
:1018F00007D0012F294801D1002318E0022F0CD175
:1019000014E00C21012240460DF1070304F0F4FB22
:101910009DF8071011F00F0203D1052005F0ECF837
:1019200006E0042A1D4801D1077001E0012303707D
:101930001A481B4903781B4A31607260002B14BFA0
:101940006E216F21184A1948194B142C31742A60E2
:101950006860EB60174915D004D8052C16D00A2C06
:101960000ED111E0BC2C08D0B4F5807F03D0622CDE
:1019700006D102220BE0002209E0012008700AE0F3
:10198000032204E0042202E0052200E006220A709D
:10199000012000E0002004B0BDE8F081D405002063
:1019A000091700089D170008F117000835170008EF
:1019B00019449231070000202DE9F041057890B0DC
:1019C00000350646334818BF01250BF02BFB0024D9
:1019D0003148A542314B0CBF2146802106904FF47F
:1019E00000500CBF4FF001084FF002084FF4807216
:1019F00005930A9120234FF480670E9005A925488E
:101A00000B920D930C970794CDF8208009940F94B6
:101A10000BF080FB1F4801210BF0A9FB4FF4602164
:101A2000012702911E48694600948DF804508DF8F4
:101A3000057003948DF810800AF09AFC1848042170
:101A40003A4603230AF0E5FC2DB11548317802220D
:101A500003230AF0DEFC124801210AF0B6FC10480C
:101A600001210AF0A9FC0E480AF0B8FC0C480AF063
:101A7000BAFC0028FAD10A480AF0B9FC08480AF072
:101A8000BBFC0028FAD1064801210AF0B9FC10B0CD
:101A9000BDE8F08108000240D60500204C2401403A
:101AA00000240140024B33F8100080B2704700BFA1
:101AB000D6050020334B2DE9F0411C88324B5A8962
:101AC0001E89A51A7543B3F91240B3F91420EF1318
:101AD000BE18E50295FBF6F43F19A7F57A6202FB02
:101AE00002F4B3F90480B3F902C00A257D43DF6133
:101AF00002FB0CFCB3F90E7002FB08F2B3F90C8088
:101B00002413674304FB08F4241404EB6232941C8E
:101B1000A210DC88083502F5004262432E114FEA1C
:101B2000EC24B3F92050B3F9003004EBE72404EBC4
:101B3000830303FA05F39C1C144BD20B1B68A3EB25
:101B4000A4044CF2503343FA05F3634303D45C001E
:101B5000B4FBF2F302E0B3FBF2F253001A12524369
:101B600040F6DE3462430A4C5C43241404EB224208
:101B700002F6CF6203EB221300B1036001B10E60E5
:101B8000BDE8F0810A060020E005002004060020E0
:101B900043E3FFFF104B07B5187818B90F490A88BF
:101BA000531C0B80F621032201AB772004F0A4FA2A
:101BB0009DF805109DF804000A02094942EA004018
:101BC0009DF80630B1F920201843C2F1080320FA2D
:101BD00003F0044908600EBDDA050020DC05002092
:101BE000E0050020040600200B4B07B5187818B953
:101BF0000A490A88531C0B80F621022201AB772088
:101C000004F07AFA9DF804009DF80510044B41EAAF
:101C100000221A800EBD00BFDA050020DC0500207E
:101C20000A060020064B074893F820200021920165
:101C30003432017002F0FC027720F42104F020BB62
:101C4000E0050020DA050020034B00221A707720FF
:101C5000F4212E2204F014BBDA05002010B54FF455
:101C600080400AF007FB0128044605D14FF480406C
:101C70000AF010FB014B1C7010BD00BFDA050020FC
:101C80002DE9F0476B4B05461A686B488CB08242D1
:101C900000F0CA80DFF8C0A19AF80080B8F1000F08
:101CA00040F0C480654F102102264FF400598DF892
:101CB0000A10384602A94FF480448DF80B60ADF845
:101CC000089004F045FB0423384602A98DF80A3039
:101CD000ADF8084004F03CFB0E213046C7F81090E8
:101CE00004F072FB0126082204A88DF81520049444
:101CF0008DF814808DF816600AF080FA28200F21E4
:101D00008DF80C0003A88DF80D108DF80E108DF8CD
:101D10000F600AF0D5FB142004F051FE7720D0218B
:101D200032460DF1070304F0E7F99DF80730444C03
:101D30000322552BE375228418BFC7F8149073D182
:101D4000D12132460DF10703772004F0D5F99DF833
:101D50000700162200F00F01030921766376AA21FD
:101D600006AB772004F0C8F99DF818209DF81900FB
:101D70009DF81B3040EA02219DF81A20218043EA99
:101D800002209DF81C109DF81D20608042EA01236E
:101D90009DF81E009DF81F10A38041EA00229DF8C7
:101DA00021309DF82000E28043EA00219DF82220A6
:101DB0009DF82300218140EA02239DF824109DF81C
:101DC0002520638142EA01209DF827309DF82610E6
:101DD000A08143EA01229DF828009DF82910E281A4
:101DE00041EA00239DF82A209DF82B00238240EA37
:101DF00002219DF82D309DF82C20618243EA0220BB
:101E0000104B41F2707146F67812A0828AF8006099
:101E10000D4829806A806B600C490D4A0D4BA86003
:101E2000E9602A616B6101E0002000E001200CB054
:101E3000BDE8F08760010020001BB70000100140E2
:101E4000E0050020491C0008E91B0008251C0008CB
:101E5000951B0008B51A0008080600202DE9F04F70
:101E60004E4E4F4B85B0778903911968328984466D
:101E700038020F1A87FB0201C00940EA4162CB1108
:101E8000F188B48887FB01012404002514EB0208C3
:101E900045EB0309000A40EA01620B12B18974881C
:101EA00087FB0101E403002514EB020A45EB030B59
:101EB000C00D40EA41224FF4FA60CB150021801892
:101EC00041EB0301CDE90001B0F5FA6F71F10001BA
:101ED00047DAA2FB024502FB03F605EB4607B80012
:101EE00040EA9471A0002646241847EB01056910CA
:101EF0004FEA3400A408B8EB000869EB0109A91007
:101F000044EA8570BAEB000A6BEB010B25484FF0F1
:101F1000FF31DDE9004584428D4122DA40F6AC50C4
:101F20000021801841EB03014143A0FB00236FF027
:101F3000060003EB4103544200FB0344A2FB0001F3
:101F400018EB0008214449EB01090B24A2FB040112
:101F500004FB031149104FEA3000BAEB000A6BEBA7
:101F6000010B114A1368A3FB0A0103FB0B11400D7F
:101F700040EAC1224B15B2EB080263EB0903D20B16
:101F800042EA4343BCF1000F01D0CCF80030039883
:101F900008B10099016005B0BDE8F08F140600207B
:101FA0001006002024FAFFFF0C06002007B50021D0
:101FB000032201AB772004F09FF89DF805009DF8FF
:101FC000043001029DF8062041EA034010430EBD93
:101FD00008B5FFF7EBFF014B186008BD0C060020A9
:101FE00008B5FFF7E3FF014B186008BD100600209D
:101FF00077204821012204F043B97720582101229B
:1020000004F03EB9454B73B51A6804464448824211
:102010000FD010258DF80650424D02214FF4005686
:102020008DF80710284601A9ADF8046004F090F976
:102030006E610A2004F0C3FC7720A02101220DF17B
:10204000030304F059F8002866D01E2101227720EE
:1020500004F016F94FF42F6004F0A6FC0025A5F15A
:1020600060030026D9B20222772001AB8DF804600C
:102070008DF8056004F040F89DF804209DF80500F7
:10208000294B40EA0221E9520235102DE7D1DA89C5
:1020900002F47F4502F00F00DD8132460123224920
:1020A000515A0232002918BF0023102AF7D113BB5E
:1020B0001A4612F0010F1C494FEA620604D011F8CB
:1020C00016104B40082104E031F8161083EA112362
:1020D000F8E713F4004F18BF83F4C0535B000139D5
:1020E000F7D10132102AE4D10F49C3F3033305437A
:1020F0009842CD8101D000200EE00C4A42F21070CF
:102100002080608062600A480A490B4B0B4A2061BC
:10211000A160E360626101207CBD00BF600100201E
:10212000001BB7000010014014060020FB1F000830
:10213000D11F0008E11F0008F11F00085D1E000804
:10214000F8B5134B05469B890E461446ECB116B103
:1021500016F8017B00E0FF270D4802210AF002F982
:102160000028F9D00A4839460AF0F7F80848012152
:102170000AF0F8F80028F9D005480AF0F0F8C0B2E3
:102180000DB105F8010B013CE0E70120F8BD00BFEF
:10219000003800402DE9F047012188B04FF480401D
:1021A0000AF03CFE374C01214FF480400AF04EFE0D
:1021B00003214FF420401823ADF800008DF80310E0
:1021C000204669468DF802304FF0040804F0C0F84C
:1021D0002D4E4FF4804220466946ADF800204FF462
:1021E00080554FF0100A8DF8028004F0B1F869466E
:1021F0002046ADF800508DF802A004F0A9F8304652
:102200000AF04EF807214FF4007000230222ADF8C7
:102210001600ADF81C104FF00109304603A94FF429
:102220008277ADF80C30ADF81030ADF81A30ADF85B
:102230001220ADF80E70ADF814901F46ADF818A03E
:102240000AF060F8304649460AF07BF89F238DF883
:1022500004308DF805708DF806708DF807700DEB61
:1022600008014246656102A8FFF76AFF25619DF8F3
:102270000900B0F1EF014A4252EB010008B0BDE89D
:10228000F08700BF000C01400038004037B5002443
:1022900002AB054603F8014D1E200A21012203F07E
:1022A0002BFF50B19DF80730482B03D125B10348CF
:1022B000057001E0204600E001203EBD180000202E
:1022C00030B585B00622054603216B461E2003F07B
:1022D00013FF9DF801309DF800001A4C43EA0021DD
:1022E00008B2FEF79BFC2168FEF7ECFCFEF7B0FE9F
:1022F0009DF80220ADF808009DF8030040EA022393
:1023000018B2FEF78BFCA168FEF7DCFCFEF7A0FE1E
:102310009DF805209DF80410ADF80C0042EA01205C
:1023200000B2FEF77BFC6168FEF7CCFCFEF790FE86
:10233000054BADF80A00294602A81A7801F022F9E7
:1023400005B030BD0C000020180000202DE9FF4131
:10235000634B644A186890420DD104274FF48055AE
:102360000226ADF804508DF807608DF806705E48BF
:102370000DEB070108E05D49884207D104A94FF43D
:1023800080445B4821F80C4D03F0E2FF322004F05A
:1023900016FB002111221E2003F072FF0121602292
:1023A0001E2003F06DFF642004F009FB02A8FFF774
:1023B00087FF00240A2527462646012202211E20E7
:1023C00003F05EFF322004F0FAFA02A8FFF778FF6C
:1023D000BDF90800BDF90A20BDF90C30241882426D
:1023E000B8BF1046F6189842B8BF034613F5805F91
:1023F000174409DD3C49013DC86880F01002CA60FD
:10240000DBD14FF0010801E04FF000081E20002151
:10241000122203F035FF0A25022101221E2003F0BB
:102420002FFF322004F0CBFA02A8FFF749FFBDF9D5
:102430000800BDF90A10BDF90C30241A8142B8BF5A
:102440000846F61A9842B8BF034613F5805FC1EB01
:10245000070707DD2448013DC26882F01001C16012
:10246000DAD101E04FF000082046FEF7D7FB014625
:102470002048FEF7DBFC204D20F000432B6038465F
:10248000FEF7CCFB01461B48FEF7D0FC20F00040D5
:1024900068603046FEF7C2FB01461848FEF7C6FCEE
:1024A00020F00042AA60002170221E2003F0E8FE06
:1024B000012120221E2003F0E3FE1E200221002223
:1024C00003F0DEFE642004F07AFAB8F1000F04D1C4
:1024D0004FF07E5129606960A960BDE8FF8100BFAF
:1024E0006001002000127A00000C0140001BB700C0
:1024F0000010014000406F460C00002001C05E4605
:102500007FB5274C0E4623789BB9264A7A21B2F92B
:1025100000000222C0F1B4038DF8041093FBF2F125
:102520008DF8051001AB6D20FF2103F047FE01235C
:1025300034E0012B1DD179258DF804500A2592FB3A
:10254000F5F00021B4225A3001F032FC8DF805007C
:1025500096FBF5F00021B4225A3001F029FC01ABC2
:102560008DF80600FF216D20032203F027FE0223D1
:1025700014E0022B13D10122002814BF10460020C2
:1025800064218DF804108DF805208DF8060001AB4C
:102590006D20FF21032203F011FE002323707FBD75
:1025A00024060020F21D00200E4B0F4A9868118867
:1025B00010B501420D4C03D004F0D6F920600BE0B9
:1025C00004F0D2F92368984206D9094AC01A126861
:1025D0003B2190FBF1F31360064A1068BDE8104000
:1025E00009F058BE000C01402C06002030060020E7
:1025F0003C06002038060020FFF7D6BFFFF7D4BF07
:1026000030B52F4B85B02F4A50B1012816D12E4C32
:102610002E4D0221188028701180216007200BE0C8
:102620004FF4807119804FF400731380274D264AB0
:10263000092413602C701720254908702048214D6B
:10264000038802221024234801A98DF80720ADF841
:1026500004308DF8064003F07BFE29880423ADF892
:1026600004101C480DEB03018DF8063003F070FEDA
:10267000164A154D1178012003F0A6FE286809F0CE
:1026800009FE2868002102908DF80D4002A801245F
:102690008DF80C108DF80E4009F0B0FD0C4B1A7837
:1026A00002F01F0304FA03F450B20B4A410942F846
:1026B000214004F073F909493C38086005B030BD89
:1026C000400600202C060020380600203506002099
:1026D00034060020000C014000E100E02806002044
:1026E00038B5044604F05AF9084B19683C31884261
:1026F0000BD31860064D07482A880460064C0B204F
:10270000226104F051F92B88636138BD280600204E
:10271000400600203C060020000C0140074BA1F5BC
:102720007A7153F82000838802684B434FF47A7023
:1027300093FBF0F18BB21380704700BF4407002079
:10274000024B53F8200002681180704744070020B4
:102750002DE9F04FDFF828814FEA001558F80540C1
:102760008E468BB008EB05071146834692462046FD
:102770007246019300F0C0FCB96807F108024FF0FF
:10278000020C18237868ADF8141005A98DF81630DE
:102790008DF817C00392CDF808C003F0D9FD039857
:1027A000364E077906A80AF080F870220198DDF805
:1027B00008C0ADF81820012100234FF4807206EB09
:1027C0000509ADF81A10ADF81C30ADF81E00ADF8D3
:1027D00020C0ADF824200C2F2BD8DFE807F0072A03
:1027E0002A2A102A2A2A192A2A2A2200204606A939
:1027F00009F054FF204608210AF08CF819E0204621
:1028000006A909F08FFF204608210AF08BF810E096
:10281000204606A909F0CAFF204608210AF08CF8D4
:1028200007E0204606A90AF003F8204608210AF02E
:102830008BF808EB0B118B7B1BB1204601210AF0B2
:1028400052F8204601210AF042F80C2F10D8DFE898
:1028500007F0070F0F0F090F0F0F0B0F0F0F0D00D2
:10286000343404E0383402E03C3400E04034745145
:10287000A9F804A048460BB0BDE8F08F5806002028
:10288000140F01081B4A1C4813881180C91A89B209
:1028900040F68C2291420380184B02D900221A7014
:1028A0007047A1F2EF2080B240F2DA52904218D87D
:1028B0001B78072B15D81248032B20F81310114A48
:1028C00009D811480088884205D2012101FA03F392
:1028D00010780343137012780F2A02D1094B00219C
:1028E00019700648094B0278511C017000201880AD
:1028F000704700BF420600203A070020540600201F
:10290000440600203C0700201A000020EE070020AB
:102910007FB5044601A80D46164609F0D0FF0020F9
:102920000123ADF80A00ADF80C0001A92046ADF86E
:102930000450ADF80660ADF808300AF041F87FBDEC
:102940002DE9F743DFF858800501144E05EB080424
:10295000A3688946761928210746B2716068022269
:102960008DF8061001A9ADF804308DF8072003F0AA
:10297000EFFC55F80800217B0022FFF7C9FF204635
:1029800001224FF6FF7100F0D9FB204639464A4636
:1029900000F094FB3046BDE8FE8300BF58060020DF
:1029A000140F010810B5134B00011B18DA795AB93E
:1029B00001221981DA71104B02221918097B18586B
:1029C000BDE81040FFF7A4BF1C8959810B4A091BC1
:1029D0009C7989B222F8141000249981DC71064B8D
:1029E00022461918097B1858FFF792FF0448048003
:1029F00010BD00BF58060020140F01084406002037
:102A0000EE0700202DE9F0410446028A484B807908
:102A100061781A80002814BF0225002501B1013514
:102A2000444F57F8257000257A5DFF2A02F00F0009
:102A300002F0F00309D122893F484049B2F5FA7FFC
:102A4000016071D93E4B03606EE0A17811B1811E27
:102A5000012965D9E17811B1011F032960D9E17914
:102A600009B181425CD012F0300F03D02278002AE5
:102A700008BF0023217931B1A27922B9A0F1080160
:102A8000012998BF802362792AB1A17919B9021F5F
:102A9000032A98BF802303F01001CAB23AB1002282
:102AA0002849FFF74DFF284B08221A7038E003F041
:102AB0002001CAB242B1244E24493278FFF740FFC8
:102AC0003078411C31702BE003F04001CAB292B162
:102AD00023891F4AB3F5FA7F94BF012108214A4395
:102AE0001C4EB2FBF3F39AB2A38996F80080FFF76D
:102AF0002FFE194B0EE01B0612D563891449174EA1
:102B000091FBF3F292B2E389012196F80080FFF77E
:102B10001FFE134B43F8280008F1010886F80080D7
:102B200001350E2D80D186E70020BDE8F08100BF81
:102B30001A000020DC0E0108400700204127000891
:102B40001D2700088528000838070020A52900084F
:102B500040420F0039070020440700203D070020B5
:102B60007407002008B5044B1A78824202D9034B3F
:102B70001A68904708BD00BF3907002040070020B1
:102B8000044B1A78824204D9034B53F820000268A0
:102B9000118070473D07002074070020014B33F877
:102BA0001000704744060020704701717047426A68
:102BB000806A131A594251EB03007047037913F0EE
:102BC00001010BD0026AC3699A4205D09CBFC0685C
:102BD0001218D01AC0B270470020704708467047DC
:102BE000037910B513F0010104460ED0FFF7E6FF9C
:102BF00060B1E3696269E168D05C4A1E934201D228
:102C0000013300E00023E36110BD084610BD0379E5
:102C10009A070AD5436A8269D154416A03694A1CFA
:102C2000B2FBF3F103FB11224262704790F842328B
:102C30001BB1D1F1010138BF0021D0F83401426845
:102C4000836809B1136170475361704707B5034644
:102C500099684822ADF804100223406801A98DF854
:102C600006208DF8073003F073FB0EBD58B50E4BF0
:102C7000044618680E460346B3FBF2F1B1F5803FF7
:102C800003D3012BF8D95B08F6E7084A89B2B0FBF9
:102C9000F2F3DAB2204600F051FA054A20463146F6
:102CA000BDE8584000F00ABA6401002040420F001D
:102CB000253000087FB5044601A80D46164609F0E8
:102CC000FEFD00200123ADF80A00ADF80C0001A9BB
:102CD0002046ADF80450ADF80660ADF8083009F0B4
:102CE0006FFE7FBD38B504460D46002A0CBF022298
:102CF0000022217B0068FFF7DDFF034A20462946BA
:102D0000BDE8384000F0DAB9B92E000807B503462F
:102D100099681022ADF804100223406801A98DF8CB
:102D200006208DF8073003F013FB0EBD00F13403CD
:102D30004FF48072436100F59C710023C26003620E
:102D4000C361816102618362436270472DE9F04192
:102D50001D46194B0E46032103600171044690463F
:102D60000127FFF7E3FF002084F83C0284F83902D2
:102D7000A4F84402A4F8460284F83872D4F8340166
:102D800084F84252FFF7C2FF206BFFF75FFF39461E
:102D90002046FFF74BFF322003F011FED4F8340138
:102DA00031464246FFF762FF206B31462A46BDE8B6
:102DB000F041FFF797BF00BFFC0E010810B5084AAD
:102DC000044608480B4602631032C0F83421002143
:102DD0002246FFF7BBFF044B01201C60187110BD99
:102DE000540F01081C1300209407002003460749D4
:102DF0000748084AC0F8781212681031C0F87C13EE
:102E000000F512700121FFF7A1BF00BF740F010888
:102E10001C13002094070020C268036A511E8B42D5
:102E200001D3002300E001330362704710B590F82E
:102E30003C220446AAB9836A416A994225D0806936
:102E40002169C05C01338B42A36228BFA2624200A9
:102E50000A2342F4007084F83D32A4F83E020123B4
:102E600011E090F93D3273B1B0F83E124A08A0F873
:102E70003E2201F00101FFF7D9FE94F83D02431E06
:102E800084F83D3210BD84F83C3210BD90F83B32DE
:102E900010B583B990F83A3290F8392293420AD2A9
:102EA000012101FA03F1B0F8404201332143A0F8B7
:102EB0004012DBB2F2E710BD2D4B10B54FF4127487
:102EC00004FB00342079C10751D594F8381221B39E
:102ED000236B0021186809F041FD94F83C1221B1E0
:102EE000B4F84402421CA4F84422236B94F8422212
:102EF0001868197B002A14BF02220022FFF7DAFEAD
:102F00000020012184F83B1284F8390284F83A0247
:102F1000A4F8400284F8380210BD94F83B22204601
:102F2000012A04BF94F8392284F83A22FFF7AEFF51
:102F300094F83B02236B58B9012094F8422284F89C
:102F40003B021868197B002A14BF022200220AE003
:102F5000002184F83B1294F842221868197B002A59
:102F60000CBF02220022BDE81040FFF7A3BE10BD37
:102F70001C13002090F83B1200230122012980F845
:102F8000393280F838220CD180F83B32036B90F84C
:102F90004222197B1868002A0CBF02220022FFF788
:102FA00089BE704702790346D20713D5B0F8402294
:102FB00002F4007189B209B9D10705D4B3F8460209
:102FC000421CA3F8462270474169036A5208CA545A
:102FD000FFF722BF704710B590F838320446002B37
:102FE0001ED190F839124A1CD3B2092B80F839321D
:102FF00003D1BDE81040FFF749BF0A2B10D190F86C
:103000003B0228B9B4F8401241F00102A4F8402272
:103010002046FFF7C7FF2046BDE81040FFF7AABFD4
:1030200010BD0000064B10B54FF4127404FB0034C1
:103030002046FFF7FBFE2046BDE81040FFF7CBBF60
:103040001C13002030B500240E4D55F82450854245
:1030500002D00134E4B2F7E7A400E4B200200A4D44
:103060002D5C8D4202D0451CE8B2F8E70019C0B2D1
:103070000F2805D8054C04EB001083600171027322
:1030800030BD00BFF40F010804100108AC17002088
:103090000C2912D8DFE801F00711111109111111E3
:1030A0000B1111110D00022104E0042102E008219E
:1030B00000E01021012209F024BC704738B5044615
:1030C0000D461346217B00682A46FFF7BBFF2068A8
:1030D000217BBDE83840FFF7DBBF07B58DF8040062
:1030E000012000238DF806008DF8070001A88DF857
:1030F000053009F0E5F90EBD7FB5044601A80D467F
:10310000164609F0C9FB0B4B0B485E4301680023D0
:10311000B1FBF6F2013D561E204601A9ADF808505C
:10312000ADF80460ADF80A30ADF8063009F06CFA7D
:103130007FBD00BF40420F006401002010B504466F
:103140000068FFF7D9FF2068012109F0C0FB607B10
:10315000BDE81040FFF7C1BF00230C4A52F82320FE
:10316000824202D05A1CD3B2F7E79B00D8B20023A8
:10317000074AD25C8A4202D05A1CD3B2F8E7181828
:10318000044BC1B203EB0110704700BFF40F0108FC
:1031900004100108AC17002070B5044600262E4B21
:1031A000F55C95B90221204609F0B3FC01284FD106
:1031B0002046022109F0B8FC29462046FFF7CCFF43
:1031C0000546204609F098FC3DE0042D12D120462A
:1031D000294609F09EFC01283AD12046294609F0EB
:1031E000A3FC29462046FFF7B7FF0546204609F015
:1031F00086FC28E0082D12D12046294609F089FCDA
:10320000012825D12046294609F08EFC2946204672
:10321000FFF7A2FF0546204609F074FC13E00C2DD1
:1032200016D11021204609F074FC012810D1204647
:10323000102109F079FC29462046FFF78DFF05464D
:10324000204609F062FCAA6801460AB1287B904733
:103250000136042EA3D170BD041001080148FFF708
:103260009BBF00BF002C01404FF08040FFF794BF90
:103270000148FFF791BF00BF000400400148FFF77D
:103280008BBF00BF000800401D481E490268006057
:103290008A4200F01F80002100F004B81A4B5B58EE
:1032A0004350043119481A4B42189A42FFF4F6AFC2
:1032B000184A00F003B8002342F8043B164B9A4228
:1032C000FFF4F9AF08F08CFE0CF0F0FC00F0C8FF42
:1032D000FFF7FEBF114E124830601248016821F01E
:1032E00070610160410201600F4C182020600F499D
:1032F0000F4808600F48D0F800D040680047000031
:10330000F04F0020EFBEADDEE035010800000020E8
:10331000B4050020B40500201C1F00201810024036
:103320000900000004000140140C0140000C0140A1
:103330004434434400F0FF1FFFF7FEBF014B186801
:1033400003F05CB80C1F00200149002000F054BEBF
:103350003D33000810B5FDF761FC0A49FDF7B2FCEA
:103360000949FDF763FD094B044618680078FDF72D
:1033700055FC01462046FDF7A5FCFDF78FFE80B207
:1033800010BD00BF3333534000F07F45B00700202D
:1033900038B50D4C00202578FEF784FB0B4A05F06C
:1033A000070322F813000135002325701846D15A6F
:1033B00002334018102B80B2F9D1C008FFF7CAFFC2
:1033C000034A107038BD00BF9C0700209E070020F4
:1033D000AC180020074B084A19781088884207D398
:1033E000064B1A68907888428CBF002001207047F5
:1033F00000207047AC180020AE180020B007002055
:10340000124B70B51860202400250020FEF74AFBFF
:103410002D180A2003F0D3FA013CF6D1C5F34F1062
:10342000FFF798FF094902230A6851784D00661991
:10343000B04203D30133062B0C44F8D104489278F0
:103440000370534303490B8070BD00BFB0070020D9
:103450001C000020AE1800202DE9F04F0446008823
:1034600085B048B9B4F9023043B9B4F90420D2F1B7
:10347000010138BF002102E0002100E0014611F007
:10348000010377D13D4D00B22B7000F0E5FC0646FC
:10349000B4F9020000F0E0FC0546B4F9040000F0C5
:1034A000DBFC0446304609F085FE0746304609F04D
:1034B000F5FE8046284609F07DFE0646284609F0BE
:1034C000EDFE0546204609F075FE8246204609F0CD
:1034D000E5FE394681465046FDF7F4FB3946834602
:1034E0004846FDF7EFFB514601904046FDF7EAFBE9
:1034F000494602904046FDF7E5FB314603905046B1
:10350000FDF7E0FB1E4C4946206006F10040FDF748
:10351000D9FB29466060A5600298FDF7D3FB014600
:103520000198FDF7C7FA2946E0600398FDF7CAFB4A
:1035300001465846FDF7BCFA3146206108F10040CB
:10354000FDF7C0FB294660615846FDF7BBFB01460D
:103550000398FDF7ADFA2946A0610198FDF7B2FB8B
:1035600001460298FDF7A6FA3946E0613046FDF7BC
:10357000A9FB206205B0BDE8F08F00BF1D00002050
:10358000B4070020013A2DE9F8430C46072A30D849
:10359000DFE802F004080F14191E2226018821809A
:1035A000428803E043880B8002885242628082880E
:1035B0001EE00388594221804288F6E74388594239
:1035C00021800288F2E703885942218041880CE07B
:1035D00042880A80018808E003880B80428803E063
:1035E000438859422180028851426180808842424A
:1035F000A28030480278002A5AD1B4F90000FDF7C1
:103600000DFB8046B4F90200FDF708FB0746B4F94C
:103610000400FDF703FB284D064629684046FDF7E8
:1036200051FBE96881463846FDF74CFB01464846A8
:10363000FDF740FAA96981463046FDF743FB014694
:103640004846FDF737FA09F0E9FD696820804046F1
:10365000FDF738FB296981463846FDF733FB014603
:103660004846FDF727FAE96981463046FDF72AFB0F
:1036700001464846FDF71EFA09F0D0FDA9686080B2
:103680004046FDF71FFB696980463846FDF71AFB87
:1036900001464046FDF70EFA296A07463046FDF717
:1036A00011FB01463846FDF705FA09F0B7FDA08089
:1036B000BDE8F8831D000020B4070020F8B5174CC2
:1036C00006462378274673B903F068F9144D2A6833
:1036D0003232904207D30120207003F01FF903F02B
:1036E0005DF92860F8BD3878B0B103F057F90C4C9B
:1036F0002168731898420FD3084A0020107003F015
:103700000DF903F04BF920600648017809B14B1E12
:103710000370054801220270F8BD00BFD8070020E1
:10372000E0070020DA070020DB07002037B58DF81E
:10373000051022498DF807300B788DF8040002A897
:103740008DF80620C21812F8044C0D46443CE0B235
:103750000A282CD81A49022B31F8104003D814B18A
:103760002046FFF7ABFF2B78022B0BD9154D2D68A8
:1037700003F014F9021B954204D21049124B0020A9
:1037800008701870114802780146012A00D094B9D7
:103790000A4B1878022801D8421C1A7000200870C1
:1037A0000B49087003B0BDE8304003F0B7B83224CD
:1037B000022BD5D9D7E703B030BD00BFDD0700200D
:1037C00008100108E0070020DA070020DB070020CE
:1037D000D807002070B5394B04465A7B384802B1EF
:1037E000012202704FF4007000F036F9F0B1354953
:1037F0004B78181C18BF012000F0D0FC38B1324DB6
:103800000120287000F0D6FC08B102222A7000F0D6
:10381000B3FC28B12B494B7813B92B4A0220107006
:1038200000F0A0FC10B1284B00211970202005F0F9
:1038300019FE60B121482549827A0AB9C37A23B1B9
:103840002048C27A0AB9012300E000230B701E4908
:103850000878022802D14C204E211DE0012807D112
:103860004D2153204C220B46BDE87040FFF75EBF50
:10387000164A1378012B03D1532001464E2206E04D
:103880000F490878012804D15320014602464D23F0
:10389000EAE724B153204D210A464423E4E70C4AC9
:1038A000137823B13220BDE87040FFF707BF094904
:1038B00020460C70BDE8704003F030B8981E002020
:1038C000D9070020871E0020DE070020DC0700202B
:1038D000DA070020D80700200E4B1A78402A16D1AC
:1038E0005888B0F5667F12D11979BE290FD193F8A7
:1038F00095230020EF2A0CD113F8011B064A4840FB
:103900009342F9D1D0F1010038BF00207047002068
:103910007047704700F8010898FB010838B5FFF7B9
:10392000DBFF10B90A2003F0E7F8164C16492046D1
:103930004FF466720CF004FA94F89433022B02D917
:10394000002084F8940394F89413CC2202FB0143E2
:103950000E4D03F5987128460CF0F2F905F11F00A1
:1039600005F036FE05F11F00B4F8D010B4F8D220EF
:1039700005F048FE287801F07FF9BDE8384004F0F2
:1039800051BD00BF7C19002000F80108B0180020CC
:103990002C4B70B5402206464FF466701A70588062
:1039A000BE25EF2200201D7183F8952383F896032E
:1039B00049B193F89413CC2202FB0133224903F559
:1039C00098700CF0BDF900210D461E4A885C01314B
:1039D000B1F5667F85EA0005F7D182F89653002598
:1039E00009F02EF9342009F03FF9184809F092F94E
:1039F000042811D1154C164B2046E15809F060F906
:103A0000042805D0013509F027F9032DE8D103E09A
:103A1000104A04349442EED109F01EF9032D02D06D
:103A2000FFF75AFF10B90A2003F066F8FFF776FF98
:103A300036B10F2014210122BDE8704008F0AABA67
:103A400070BD00BF7C190020B018002000F80108EC
:103A50007C21FE1798FB0108034B996808420CBFB4
:103A600000200120704700BF7C190020024B9A689B
:103A700010439860704700BF7C1900202DE9F34780
:103A80000446FFF729FF10B1002C00F07081B94AFD
:103A9000B94D10685168B94C6B4603C34FF4667258
:103AA000002128460CF0FAF9CC22002120460CF027
:103AB000F5F940200321287002206971FFF7D6FF35
:103AC000FA22A5F8F2202A236E22A5F8EE304FF450
:103AD000FA7085F804212B2340F24C42A5F8F60039
:103AE00085F80531212002F54873202185F806016B
:103AF000A5F8163140F27E404FF47A7300274FF05C
:103B000001094FF4167685F8F410A5F8142140F257
:103B1000DC5100F52F72A5F8D00003F5CB70A5F8A5
:103B2000F060A5F81211A5F8D22085F89473A5F8D5
:103B3000F870A5F8FA70A5F8FC7085F8E27085F8C1
:103B4000E37085F8E470A5F8E670A5F8E870A5F8CC
:103B5000EA7085F8ED7085F8EC9085F8077185F8C6
:103B60002C7185F82D7185F82E7185F8107185F806
:103B7000187185F8197185F81A91A5F8D430A5F84F
:103B8000D6006C30A5F8D8004FF4C870A5F8DE0058
:103B90004FF41650322340F2B452C5F8240140F6D7
:103BA000AC50A5F8DA20A5F8DC301A46A5F8E030CC
:103BB000A8814FF4E1331E20C5F82031E072522372
:103BC0002073552085F82A31E07017230B204FF021
:103BD00028086375A37560712D2314204FF0080E1B
:103BE00063732271A07184F810E085F81C7185F868
:103BF0001D7185F8287185F8297185F81B7127706A
:103C000084F8018084F80280E775A7732776E7734C
:103C10006776A37660745020E076E1845A20042110
:103C200020722375E077412384F82E1054485549BB
:103C30004FF00E0A84F82030534B84F807A04FF061
:103C4000640C4FF00A0A4FF0780E84F8212060636C
:103C50001522E1634D4805F5847184F83120A36392
:103C600084F812A084F81CC084F8098084F80AE063
:103C700084F81E9084F8237084F8247084F82570EA
:103C800084F822706785A785278584F82F8084F8BB
:103C9000308084F8409005F0F3FC4FF44872C8205F
:103CA0004FF4966340F2D9313E4684F86C7084F844
:103CB0006D7084F86E8084F86F9084F87270A4F848
:103CC000702084F8B4A084F8B500A4F8B630A4F845
:103CD000B8104FF47F724FF4FA601DF80710A4F883
:103CE0007420A0F5FA73FF220137A4F87600A4F837
:103CF000783084F87A1084F87B200834082FE8D1D3
:103D00001E4C0120C823142184F8BA0084F8BB009B
:103D100084F8BC00A4F8BE3084F8C01084F8C20057
:103D20001E2264204FF49673282184F8C120A4F841
:103D3000C400A4F8C630A4F8C81000240E4A00231A
:103D4000A0181034C02C0361F8D100241049CC22F3
:103D500060180A49CC340BF0F3FFB4F5197FF5D1A4
:103D60000020014602B0BDE8F047FFF711BE02B0E7
:103D7000BDE8F087940E01087C190020B0180020DF
:103D80009A99193F3D0A773FF6287C3F1E1001089B
:103D9000AC1A0020024B9A6822EA00009860704733
:103DA0007C190020014B9868704700BF7C190020E7
:103DB000884203DB8242B4BF114601460846704781
:103DC0000023036170472DE9F0410669044601367E
:103DD000012E0D46066105D10023616021608360DC
:103DE000BDE8F081D0F8008008464146FCF760FE4F
:103DF00007463046FCF712FF01463846FDF716F835
:103E000001464046FCF756FE0646606031462846AD
:103E1000FCF74EFE01463846FCF754FFA168FCF75C
:103E200049FE2660E060A060BDE8F08110B5044660
:103E30000069012807DD0138FCF7F0FE0146E06863
:103E4000FCF7F4FF10BD002010BD08B5FFF7EEFF32
:103E5000BDE8084009F044BC08B5FCF7D5FA04A356
:103E6000D3E90023FCF736FBFCF7CEFD08BD00BF0D
:103E7000399D52A246DF913F2DE9F041069C06464E
:103E80000F46002B0CBF4FF020084FF030082046A3
:103E900010F8013B0BB9154603E0002AFBDD013A9F
:103EA000F6E7002D04DD30464146B847013DF8E70E
:103EB00014F8011B11B13046B847F9E7BDE8F081AD
:103EC0002DE9F04389B006460F4603921C46039A3B
:103ED000134613F8011B0393002900F08A8025295B
:103EE00001D0304683E0002004905578911C302D9D
:103EF000039105D19578033203924FF0010800E059
:103F00008046A5F13003D8B2092806D8284603A96F
:103F10000A2204AB00F00CF905466C2D05D103997B
:103F2000012211F8015B039100E00022642D2FD0E3
:103F300010D8582D3AD006D8002D5AD0252DC6D1EC
:103F40003046294653E0632DC1D130462178251DE6
:103F5000B8474AE0752D0DD0782D27D0732DB6D1F6
:103F6000251D2468304600943946049A0023FFF743
:103F700083FF3AE0251D20680A2122B1002205AB0B
:103F800000F060F802E005AB00F08CF82C4623E06E
:103F900005AD04F104092068294612B100F077F854
:103FA00001E000F0A4F84C46009517E004F1040984
:103FB0002068102142B1B5F15804634253EB04026A
:103FC00005AB00F03FF806E0B5F158035A425A41FC
:103FD00005AB00F067F84C4605A80090304639461E
:103FE000049A4346FFF748FF71E72C466FE7B8474E
:103FF0006DE709B0BDE8F083024B19600249086023
:10400000704700BFE4070020E80700200FB407B5A1
:10401000094904AB0868094953F8042B096801935E
:10402000FFF74EFF064B186802F007FA0028F9D098
:10403000BDE80E4004B07047E8070020E407002008
:104040000C1F0020F0B50124B0FBF4F58D4201D324
:104050004C43F9E70026C4B1B0FBF4F504FB1500AE
:10406000B4FBF1F41EB9002D01DC002CF4D1092DB4
:10407000EFB204DD002A0CBF5725372500E03025BC
:10408000ED1903F8015B0136E5E71C70F0BD00286F
:104090000B4603DA2D22404203F8012B0A210022AD
:1040A000FFF7D0BFF0B50124B0FBF4F58D4201D38A
:1040B0004C43F9E70026C4B1B0FBF4F504FB15004E
:1040C000B4FBF1F41EB9002D01DC002CF4D1092D54
:1040D000EFB204DD002A0CBF5725372500E030255C
:1040E000ED1903F8015B0136E5E71C70F0BD00280F
:1040F0000B4603DA2D22404203F8012B0A2100224D
:10410000FFF7D0BFA0F13003DAB2092A01D8184670
:104110007047A0F16101052901D857387047A0F117
:104120004103052B01D8373870474FF0FF307047F7
:104130002DE9F8430D6804460F469046994600263F
:104140002046FFF7DFFF002806DB404504DC08FBC4
:10415000060615F8014BF3E73D602046C9F80060FC
:10416000BDE8F883034BB3F90000D0F1010038BF7C
:1041700000207047EE070020064B0749B3F9000006
:1041800091F8B430052253439842D4BF0020012057
:10419000704700BFEE070020B018002010B504469D
:1041A000FFF7EAFF002814BF2046002000F00100BE
:1041B00010BD00000749084B91F8B420B3F9000086
:1041C00091F8B530D118052251438842D4BF002060
:1041D00001207047B0180020EE07002008B505F058
:1041E00061F9024B00221A7008BD00BF871E002033
:1041F00010B54FF40070FFF72FFC18B3FFF7BCFFAA
:10420000E0B1114B5C78201C18BF0120FFF7C6FFFE
:1042100070B10E480E4BB0F812210E49B3F8B6003B
:104220000A804A808A80C8800B490A88531C0B8008
:10423000FFF7C0FF00B90CB9FFF7D0FF07480188AE
:104240004A1C028010BD00BF871E00207C19002080
:10425000B0180020C81E0020EC070020EE07002048
:1042600030B587B002F0B6FBFFF76EF80020FFF71D
:1042700005FCFFF753FB814A92F8073133B1012B5C
:1042800001D0092B02D18DF8003004E000208DF818
:10429000000082F807016846FDF78EFB7848FFF7BB
:1042A000DBF80E2005F0E8F803F0E4FA73494C79E6
:1042B0000E2C01D0082C01D1012500E000254FF47F
:1042C00080708DF80A50FFF7C7FB18B90820FFF778
:1042D000C3FB00E0012000F0010240208DF8062021
:1042E000FFF7BAFB8DF807000120FFF7B5FB8DF84B
:1042F00005000820FFF7B0FB80F001038DF80430C3
:1043000003F008FF8DF808005E485C4D90F8BC1083
:10431000B5F8DE204FF47A70B5F8E030C1F38004D0
:10432000ADF810004FF480408DF80940ADF80C2036
:10433000ADF80E30FFF790FB18B1B5F8DA10ADF814
:104340001010BDF80C40B4F5FA7F02D90022ADF888
:1043500010204C48B5F8123195F80751B0F8B81054
:10436000012DADF81230ADF8141004D0092D01D193
:10437000072500E0002501A88DF80B50FEF742FB51
:10438000414805F0AFF84FF48070FFF765FB40B18E
:104390000820FFF761FB20B9384C94F81D0104F0A8
:1043A00093F80120FFF758FB30B14FF48060FFF71E
:1043B00053FB08B101F062FC344B102208205A6113
:1043C0000A251861314C013DE16881F01003E3607A
:1043D000E26882F00800E060192002F0F0FA0120A3
:1043E00002F09CFA192002F0EAFA002002F096FA94
:1043F00015F0FF05E6D1082110232161236101F0AA
:1044000075FB02F029FC0220FFF726FB10B12048C3
:10441000FEF7F6FF1F4805F0F5FE4020FFF71CFBF6
:1044200050B1164CD4F8240194F82811FEF7C6FCBC
:1044300094F82901FEF7DAFC4FF40060FFF70CFB5B
:1044400010B1154805F0C2FB02F08EFA134A106055
:104450000A484579052D03D1114B4FF4C8711980D5
:10446000104A114D114B4FF47A74C8200121148069
:104470002880597300F00EFCFCE700BF7C19002077
:10448000621A0020B0180020841A0020000C01409D
:10449000801A00209C1A00200C1F002020080020F9
:1044A00090080020E6090020E4090020871E002073
:1044B00008B5034BB3F9D40003F0F8FAFEE700BFE8
:1044C0007C1900202DE9F04F794B0024B3F902A0AC
:1044D000B3F9000087B0BAF1000FB8BFCAF1000A03
:1044E0000028B8BF40428245B8BF82462546A04654
:1044F00027460594A14626466E49CA7812B90B791B
:10450000002B40D0022E3ED06B4B6C486849B0F86F
:10451000F620685EE95EDFF8B4B101EB400051427D
:10452000FFF746FC664A05EB0B0335F902C0B3F909
:104530002A10CCEB00009BF8082000EB010902FBDD
:1045400009F09BF81C30642190FBF1F005226FF01C
:10455000040159435A43CDF81090FFF729FC594BF9
:10456000DDF810C0E258584981460CEB020042F2D7
:1045700010720493FFF71CFC04999BF812306050F2
:104580005843001305904B49CA781AB10B790BB9FF
:10459000022E30D1464F4D48EF5F5021794306EB54
:1045A000000B9BF801204A4BDFF83C8191FBF2F0B5
:1045B000E95E54F80820401A801846494FF47A52B0
:1045C0000493FFF7F5FB049B48F80400E95E00291B
:1045D000B8BF4942B1F5207F02DD002048F8040051
:1045E00058F804207D239BF80B1092FBF3FE01FB8F
:1045F0000EFC4FEAAC182F480279A2B1022E12D05D
:104600000AFB07F1CAF5FA7303FB09104FF4FA71BC
:1046100090FBF1F20AFB08F0DDF814B003FB0B038A
:1046200093FBF1F308E0C3780BB1022E02D14346AD
:104630003A4601E0059B4A462549DFF8B0C0695A71
:1046400016F80CB008B20BFB00FB6FF04F0C9BFB95
:10465000FCFB9344204ACDF804B035F902C0A952BE
:10466000CCEB00001D4ADFF888C0029054F80C1013
:10467000A0584018029903904018A15844F80C1013
:104680000299A150164A0434B15C202201FB00F0CB
:1046900090FBF2F15B1A134A9B44013625F802B0F5
:1046A0000235032E7FF428AF07B0BDE8F08F00BFBE
:1046B000441D0020871E0020760800207C19002061
:1046C000940D002080080020F0D8FFFFB0180020D3
:1046D000980D002080C1FFFF020800206008002024
:1046E000921D00204C1D0020F4070020951D002085
:1046F000380800202DE9F74F002425462646A2461B
:10470000474BDA780AB91879C8B1022E19D0454B4F
:1047100045484649B0F8F6206F5EE85E514200EB2E
:104720004700FFF745FB424A424F35F902A0EB191B
:10473000CAEB0001B3F92A0001EB000A0BE0022EDC
:1047400009D13C49394B91F82470B3F904201B3747
:1047500057437B1116E03249364ACF7877B9334850
:1047600092F823702B5E1B375F4309793B1149B1E7
:10477000927C02FB0AF703EB272303E0137A03FB87
:104780000AF003112C48DFF8C8B0295EBBF800001E
:104790005F1A284B784306EB030898F80120DFF8EE
:1047A000B4907A4398F80B104FEAE21C54F80920B1
:1047B000C31201FB0320214944F809004FF4001201
:1047C000CDF804C0FFF7F4FA1D4B4FF6FF72E15825
:1047D000E750791ABBF8007044F809003B09B2FBB6
:1047E000F3F74F43174A184B54F80290E158BF11A2
:1047F000A750494498F81520C9194A43DDF804C068
:1048000012490CEB603044F80390013600EB222390
:104810006B5204340235032E7FF472AFBDE8FE8F75
:10482000871E0020760800207C190020441D0020EF
:10483000940D0020B0180020980D00200000E0FF2B
:104840005008002028080020100800204C1D0020DF
:104850005C080020F40700200B4B0C481A8852B962
:10486000817841B142786AB9012141700848094B09
:1048700002881A807047437823B90220FF21012261
:1048800007F088BB704700BFE6090020871E0020A4
:10489000F21D0020901D00202DE9F04FA24BA34AED
:1048A000B3F90600D18C85B088420FDBB0F5FA6F02
:1048B00092F8254007DA451A6C43A1F5FA6694FB95
:1048C000F6F4643403E0C4F1640400E06424984A1C
:1048D000964BB2F8127192F9EC2093F823100097DE
:1048E000574293F86C50019193F86D60B9B293F808
:1048F00024300291002103930A468B4FDDF800809B
:1049000031F907C040F2E637C8EB0C0303F2F31E9F
:10491000BE4503D8002BB8BF5B4201E04FF4FA73E9
:10492000022ADFF818822CD025B1AB42CCBFC5EBF0
:10493000030300236427DFF82CA293FBF7FE6FF03C
:10494000630B3AF81E900BFB0E3B0EF1010E3AF989
:104950001EA00FFA89FECEEB0A0E0EFB0BFE9EFB8D
:10496000F7FEF14428F80190DDF8048003FB08FE0F
:10497000704B9EFBF3F3DB199BB2634393FBF7F79A
:1049800012E026B1B342CCBFC6EB03030023029F63
:104990005F43A8F80470039F002BB8BF5B427B43C2
:1049A000644F93FBF7F76437604B02EB030E9EF8FE
:1049B0000190642307FB09F898FBF3F9DFF8A8815D
:1049C00002F808909EF80B909EF815E007FB09F896
:1049D00007FB0EF798FBF3F9DFF8908197FBF3F3F1
:1049E00002F80890DDF80080534FC445D35503DA30
:1049F000524BCF5A7F42CF5201320231032A7FF409
:104A00007CAF4B4C4FF4FA62B4F81411FFF7D0F9B5
:104A1000B4F814614FF47A75801B4543C6F5FA6308
:104A2000B5FBF3F56421464895FBF1F36FF063069F
:104A300030F8132006FB0355013330F9130013B28D
:104A4000C01A45433F4B3D4C95FBF1F1587A8A180B
:104A5000E280002838D03C4F3C4D3E882988721AAD
:104A600010B2FFF7F9F9074608F0A4FB06463846EE
:104A700008F014FC0546B4F90200FCF7CFF807462D
:104A8000B4F90000FCF7CAF831468046FCF71AF981
:104A9000294681463846FCF715F901464846FCF799
:104AA00007F8FCF7D5FA314620803846FCF70AF9BA
:104AB000294606464046FCF705F901463046FBF715
:104AC000F9FFFCF7C5FA60800220FEF7C5FF90B140
:104AD0001F4806220378591CCBB20370B3FBF2F0D7
:104AE00002FB103111F0FF0F05D1FEF751FCFEF76C
:104AF00071FC184B1870174A1078003018BF01204D
:104B0000FEF768FE14490B881BB9144A108828B9AF
:104B10002EE0022004F0A6FC0028F6D0104BDA6844
:104B200082F00801D96030E0C81E0020B0180020D3
:104B30007C1900200CFEFFFF921D0020441D002068
:104B4000B01E0020871E0020F21D0020901D0020B6
:104B5000340800205E08002090080020E6090020AC
:104B6000000C0140EC1E0020951D0020881D002037
:104B7000364B997811B1364A082010615B7813B131
:104B800033480821416104F0FDFF8020FEF764FFF7
:104B9000B0B13048304B02681968501A00280FDB5A
:104BA00002F5434250321A60284B2C4A5978081CAF
:104BB00018BF0120B2F90210B2F90020FDF7A0FCE5
:104BC0002448274A01681368C81A002810DB1F4BC5
:104BD000587B58B998701E4B01F5F421D86880F0C5
:104BE0000800D86001F59073136001E0012199700D
:104BF00005F014FB1B4A107830B94FF40060FEF743
:104C00002BFF08B105F006F8202004F02BFCA0B122
:104C10001049154B0A681868111A00290DDB134852
:104C20000178042909D902F5123202F5F8701860EA
:104C3000074BD96881F01002DA600D4883680BB128
:104C40000C48984705B0BDE8F08F00BF871E0020D4
:104C5000000C014088080020F0070020940D00207F
:104C60004C080020841200200C0800208E1D00201B
:104C7000DC1D0020241D00200128034B14BF034A23
:104C8000034A1A60704700BF20000020C544000896
:104C9000F546000870B50820FEF7DEFE90B19F4B88
:104CA00093F8100103280CD8DFE800F00202050891
:104CB00004F016FF06E004F071FD03E004F024FEAA
:104CC00000E000209649974A0B681168591A00299C
:104CD00002DA002800F0E88203F59C449248203470
:104CE0009249146004F01CFC4FF48040FEF7B4FEBF
:104CF00020B18F4D297809B904F0D4FB874A92F886
:104D00001B01B0B18B4CC31C34F913504FF47A72B1
:104D10000021A5F57A70FFF74BF8FBF77FFF864976
:104D2000FCF784F88549FBF7CDFFFCF7B7F9844918
:104D30000880FFF75DFA794AB2F81401B2F816411B
:104D4000002213467B4D9B08515F8142C4BF63F034
:104D50007F03DBB2A142B8BF43F040030232082A0E
:104D6000F0D17848784A047805469C4204D11078FE
:104D7000F92803D8411C00E0002111704FF4804055
:104D80002B70FEF769FE68B1644D6A4BB5F81211DD
:104D9000B5F8DC20B3F90640881A844202DD8B188E
:104DA0009C420CDB4FF48040FEF756FEF8B9614C94
:104DB0005A49B4F90650B1F81421954217DA634DF7
:104DC0006348644CB5F8421000230360436083607D
:104DD0002360636059B1564A5F4B1078002800F099
:104DE000C7831C78002C00F0C383FFF735FD5649BC
:104DF0000A78142A40F0D58057484478ECB1534CD7
:104E0000B4F842202AB94F4D29785F2901D104F026
:104E100049FB424890F81831002B00F0C2804B4CFF
:104E2000B4F84220002A40F0BC80464D29787D2904
:104E300040F0B78004F036FBB3E0424D2B78572B9F
:104E400018D1464C4FF47A724FF480702280FEF7EE
:104E500003FE08B103F094FA042004F003FB10B140
:104E60003F490A250D80082004F0FCFAD8B93D4BD3
:104E7000188018E00420FEF7EFFDA0B129785A2928
:104E800011D1394802781AB10470384B012009E079
:104E9000374C384B257885F00101217009B102208B
:104EA00000E003201870274802785D2A00F067832D
:104EB0005B2A00F066835E2A00F065832348B0F821
:104EC000422032B91F4C25786F2D02D1FFF7C4FC68
:104ED00015E012491B4B91F8180118B112B91A7854
:104EE0007E2AF3D01C78972C04D1234B4FF4C87042
:104EF000188004E0A72C02D1174901258D73114AAF
:104F00001478BB2C03D1114CA18D8D1C04E0B72C5F
:104F100034D10E4CA28D951EA5853BE07C19002056
:104F2000880800208C080020841A0020AE1E002073
:104F3000981E0020C81E002000007A4400C07F4454
:104F40008C1D0020240800207A080020B0180020C2
:104F5000F407002080080020871E0020E6090020BA
:104F6000E4090020F21D002000080020360800207F
:104F700025080020DA07002090080020BE2C03D16D
:104F8000774D6B8D981C04E0BD2C0AD1744D698D52
:104F9000881E688501200146FEF7FAFC714B00204F
:104FA00018700420FEF758FD00282CD06E4B18789E
:104FB00088B16E4C627872B16D4D6E48B5F90610CD
:104FC000B0F81441A14206DD6B4A15781DB96B4952
:104FD000322008801D70684B5C7C54B1684B1D7892
:104FE0002DB9684A107810B9644C3221218001240F
:104FF00008E0644D2A7832B15C48417819B9624BB7
:10500000297001241C700023604C1A4634F8020FEA
:1050100040F2135501B2A942CCBF0025012505FA83
:1050200003F5A0F21550B0F5C77F8CBF002001201A
:105030002A435D1C00FA05F0024340F2A46081425D
:10504000D4BF00210121981C01FA00F103330A4367
:105050000C2B92B2DAD100234148474900EB4300C0
:10506000B0F8420002420CBF002001205854013326
:10507000152BF1D14A7822B1022004F0F3F928B9B6
:105080000DE0FFF779F80028F6D108E0374AD37829
:1050900043B93F4901200B604B60D07002E03348B8
:1050A0000021C170344A314B917839B1187900210F
:1050B000D97020B9364A01211060506019712E4B09
:1050C0002A49187808B901220A70C878314B10B9FA
:1050D00026490A7912B11021596101E010201861A6
:1050E000042004F0BFF910B3234B2048DA7882B1D2
:1050F00082797AB9284B0121817118682749284B98
:105100000860D8882749284B088028481A60026020
:1051100000E082714FF40050FEF79EFC38B1164A51
:105120001249107910B1CB7B0BB90120C873022052
:1051300004F098F920B1104A0C4B517931B93BE099
:10514000082004F08FF90028F5D145E05879A0BB7C
:10515000174901225A710888164B18802DE000BFAC
:10516000B01800207A08002025080020871E0020A3
:10517000C81E00207C190020981E0020480800202E
:105180007E0800200008002036080020CE1E0020E7
:1051900080080020000C0140181E00201C1E00206A
:1051A000441D002008080020AC0D0020EC0D00205C
:1051B000F21D0020F01D002059718749874B8A7924
:1051C000084612B15A7A0AB901225A72C17919B144
:1051D0008348844B02881A80202004F043F9002879
:1051E00052D07E4BD97A1846002948D07E4A117891
:1051F000042944D9784A917A79B1DA79002A43D1DD
:105200007A480121D9711A72794B011D1A7003F085
:10521000C3F9784A0220107036E0D07AD97118B3F9
:105220007549764AB1F90000B2F8C8200028B8BF25
:105230004042904218DAB1F902100029B8BF494241
:10524000914211DA187AF8B901241C72684B6C4942
:1052500018706C480A684B68011D0260436003F0D7
:105260009BF9644804700FE061485C4B01780022B0
:105270001A7249B90122027003F0A6F804E0002373
:10528000C37103725B4803705349544B087B00B1F0
:1052900001205D4A98725179082901D00E2944D124
:1052A0004E4B0020587240E058480368042B3CD80D
:1052B000DFE803F0030C17222E0001220260082011
:1052C00004F0D0F810B100F0E1FA70BB4F49086863
:1052D000431C04200B6004F0C5F810B100F08EFAF6
:1052E00018BB4A490A68501C0860042004F0BAF848
:1052F00010B102F0C5F8C0B9444B4FF48070196882
:105300004A1C1A60FEF7A8FB10B103F0DDF90CE0AF
:105310003E4B00201860102004F0A4F808B100F003
:10532000BBFC4FF40050FEF797FB01F01DFB384A21
:10533000354910608A89374B22B11968411A002912
:10534000C0F231818018186001F09EFEFFF7A4FAC8
:1053500001F00AFB304B2E4A19681060421A2F499F
:10536000186008200A8004F07DF800285CD02248EC
:10537000818801F145039AB28A2A194B284A51D8EB
:105380001648407900284DD018881388C21A92B266
:1053900093B218B2B330BCBF02F5B4739BB21A48D3
:1053A0001AB2B32A90F8EC200C48C8BFA3F5B47326
:1053B000407BC8BF9BB2002836D052B25042434314
:1053C0000E4A1BB2507A6FF01D0243430A4893FB0A
:1053D000F2F3C918818027E0981E0020871E002064
:1053E000F21D0020901D00208E1D0020541D002065
:1053F000240000201C080020441D0020B0180020BC
:10540000701D0020341D00207C190020440800205D
:105410008808002070080020200800205C08002078
:10542000F01D002019881180042004F01BF80028CA
:1054300077D05D4B9A79002A73D0187C5B4B00289B
:1054400066D15B495B4C91F86F2032B3DE882488CB
:1054500091F86E2035B221B26B1A002BB8BF5B42B7
:105460009342554B0CDD554CB6B2206001208D4265
:10547000187001DD524292B24C4B9119D98050E024
:105480001A7822B14E494F4A0968187011604E4887
:10549000464903681C19CC8043E0D888238805B2AC
:1054A0001CB22C1B91F86E10002CB8BF64428C42C9
:1054B00013DD464A16888519E91A4FF4FA600CB2D2
:1054C00094FBF0F100FB11443E4D14802E683A4AE3
:1054D000761801202E60107009E03749087830B145
:1054E000374C384824680A700460384C22803649AA
:1054F000374A0C68B2F8D010E3182C4C98B2E08010
:10550000963100B2B2F8D220FEF752FCE08008E0FB
:105510002F492D4891F91A210068598800FB021281
:105520005A80234890F8722052B11F49CB780BB9AA
:10553000087928B11D4B274AD88811880A18DA80C3
:10554000202003F08FFF40B1174BD97909B9187AA1
:1055500018B11A7B0AB103F0FFFE1F4B1968884788
:1055600002F0B6FA02F032FABDE8704002F08ABAF0
:105570005D78002D3FF43BAC03F094FF37E4012449
:1055800002E0022400E00324E5B2114B0020691E72
:1055900083F894130146FEF7FBF9022028212A46DE
:1055A00006F0F8FC8AE470BD871E0020441D002030
:1055B000B01800200808002035080020AC0D00209D
:1055C000181E00201C1E0020EC0D00206C0800207E
:1055D0007C1900209E0D002020000020F8B5614BB2
:1055E000188800283BD000231A46B0F5C87F5E49D2
:1055F00001D100248C505D4C8E581F5F5A4DF61916
:105600008E50002119535A4C04321E190233062BB6
:10561000A6F8F810E9D101281DD12A684FF4C87303
:1056200002F1C80292FBF3F2A4F8F8206A68C832CB
:1056300092FBF3F2A4F8FA20AA68C83292FBF3F3C3
:105640004C4A12889B1A4C4AA4F8FC30518591852B
:105650000146FEF79DF9434801884B1E0380042054
:10566000FEF7FAF900286BD0444A1288322A11D189
:105670003F4C434DB4F8F860B4F8FA00B4F8FC10AD
:105680002E806880A9803C4D3E4B6C8DAE8D1C8079
:105690005E8001E0002A32D000231946322A3A48BF
:1056A00001D100254550314D44585E5FA619465042
:1056B0002F4800245C531D1802330431062B264664
:1056C000A5F8F840EAD1012A16D1304B30491A70BA
:1056D000304B0C7002211970294B1988A0F8F81072
:1056E00059889B88A0F8FA102649A0F8FC30224B74
:1056F0000888498858859985204B013A1A802648A0
:105700000178E9B1002303701F48194A0468322167
:1057100094FBF1F4A2F8F8404468806894FBF1F43B
:1057200090FBF1F11348A2F8FA400088091AA2F898
:10573000FC100120104A014653859385FEF728F995
:105740000A4B0B4A1888B2F8F810401A1880B2F8C1
:10575000FA105888B2F8FC20401A99885880881AA4
:105760009880F8BD90080020AC080020101E002092
:105770007C19002026000020B018002048080020D6
:1057800092080020980800209C08002000080020B3
:105790007E080020DA0700203608002008B5044BF8
:1057A000044859688847BDE80840FFF717BF00BFA5
:1057B000A81D0020101E002030B50B4B0B481968A7
:1057C00090F831400A4D4A1CA24208BF0022094805
:1057D0002C681A6040F82140074950F822000D68F3
:1057E0006419241A0C6030BDB8080020B0180020DD
:1057F000A80D0020BC080020DC0D002070B5154B62
:10580000154D18682A68811A002921DB134E28607B
:105810003368134C7BB120698047616888472288D0
:105820002B681049D018286062690F489047002102
:105830003160022070BDA0688047E2689047FFF7A2
:10584000BBFF2B6861880120CA1830602A6070BDD8
:10585000002070BD880800207C09002080090020FD
:10586000BC1D0020780D0020A80D002038B5054C87
:1058700010256561FCF76AFD034B012225611A7052
:1058800038BD00BF000C014092090020F8B53C4B28
:105890003C4D18682A68811A00296EDB00F5C33474
:1058A000A0342C60384C394E2046FCF709FDB37B00
:1058B000BBB12D68364F37483749384A3D60258897
:1058C0000023A0F8FE300D801580A0F80031658817
:1058D000A0F80231A0881F464D80558088809080B6
:1058E000B3732F4B197881B1274B2A4A1888B2F825
:1058F000FE10401A1880B2F800115888B2F8022140
:10590000401A99885880881A9880214A1368002B79
:1059100031D01C4908682349C31A8B4216D8224C3F
:105920000023E26882F00800E06017495A5A1A49D9
:1059300010B25C5E8442C8BF5A5218495C5E844211
:10594000B8BF5A520233062BEFD114E00023136084
:1059500011481249185E595E0E4A411802209A18E1
:105960001B1891FBF0F1062BA2F8FE10F0D10120DC
:105970000146FEF70DF80120F8BD0020F8BD00BF7C
:105980008808002088090020D41D0020871E0020E0
:10599000840900207C190020940900208C09002033
:1059A000920900207FC3C901000C01402DE9F84F86
:1059B000414B188800286ED00024254626463E49D3
:1059C0000A88B2F57A7F08D13C4B3D490027142064
:1059D000EF5000FB0610FEF7F3F9DFF8F0A0374FA9
:1059E0003AF90400EA59DFF8D8901318EB51FBF7A5
:1059F00015F94FF0140B0BFB069B01464FF0000806
:105A00005846FEF7E0F924F80A80DFF8ACA02D48EC
:105A1000BAF8001024F80080012933D15846FEF767
:105A200014FA294A834692F8F400E0B1FBF7F6F83D
:105A300001465846FBF702FBA8B14FF47A7148467D
:105A4000AAF80010FEF7BCF909F11400FEF7B8F946
:105A500009F12800FEF7B4F9C7F80880C7F80480F8
:105A6000C7F800800EE0154B4FF47A72E858154BDA
:105A700000F5FA7191FBF2F0E0520F210A200122A9
:105A800006F088FA013604350234032E97D10A480D
:105A90000288531E03800D4B0A4A18881188401A49
:105AA0001880518858889288401A99885880881A96
:105AB0009880BDE8F88F00BFE60900209C0900200F
:105AC000A8090020BC0D00207C190020F81D002032
:105AD00008B5044B044859688847BDE80840FFF7FB
:105AE00065BF00BFDC1D0020F81D00202DE9F3413B
:105AF000594C5A485A49B4F8EE20FBF7CDFE98B9F4
:105B00005748B4F8EE10FBF76DFC08B100270CE025
:105B10005348B4F8EE10FBF7BBFD07460028F5D15B
:105B2000032000F0E9FF00E001274B4B93F8ED0064
:105B300005283ED8DFE800F007071B2A36030220BD
:105B400003F0A2FC35E000218DF804104FF44872F8
:105B500001A84249ADF80620FBF762FB10B1414BAA
:105B600001241C703C4890F8ED10012921D06FB140
:105B7000394D3A48B5F8EE203949FBF78DFE95F8D6
:105B8000ED300222374C9342227012D03348FBF79B
:105B9000D7FC38B1304A032092F8ED4031498442B5
:105BA000087006D02D48FBF7ABFB10B12D4B04203D
:105BB00018702C490A784AB9274C94F8ED0010B1B6
:105BC00084F8ED20B1E7022003F05EFC2648FCF7E4
:105BD00019FA30B92448FCF753F810B9042003F03F
:105BE00053FC022003F03EFC1B4F20B11B4B97F8E7
:105BF000E300196888471A4A97F8E2001468A0473A
:105C000097F8E400FCF742FB10B9082003F03CFCD5
:105C10001648174C078D082003F024FCC0B13FB292
:105C2000642697FBF6F52846FAF7F8FF06FB157190
:105C3000804608B2FAF7F2FF0E49FBF743F8014637
:105C40004046FAF737FF0C49FBF73CF8206001E0CB
:105C500000232360BDE8FC817C190020A81D0020E2
:105C6000DC1D0020A8080020BC1D0020B01800206A
:105C70008C0D00208988883C0000204108B5012057
:105C8000FCF7BEFC102003F0F7FB024B00221A6069
:105C900008BD00BFF41D00200148FCF721BD00BF76
:105CA000F41D00202DE9F84F9C4C2068838A9BB29C
:105CB00013F0010239D0018821F400631A04110C99
:105CC0000180012107F08CF9954A964B117800204C
:105CD0001870D9B1944803781BB9944A1178FF29F8
:105CE00014D10123037092480278022A06D18B490D
:105CF0000B68188882B242F4006119808D4B874886
:105D000019780068012207F085F92FE18948834B53
:105D100001780022186807F07DF9844A1178FF297C
:105D200000F02481FF207F4BDEE003F00201C9B2C6
:105D300000293DD0BFF35F8F7D4D2E78012E354673
:105D400016D177490B789BB177490B7883B111460F
:105D500007F046F9BFF35F8F20683146038B07F0E9
:105D600033F9754A206816704FF480613246FBE0C3
:105D7000038BBFF35F8F6E490A78022A09D1684B03
:105D80001A7832B1684B1A781AB1002107F028F955
:105D9000E5E00978032907D1614B1A7822B16249FD
:105DA0000B78002B40F0DD804FF480610122DBE0B6
:105DB00003F00406F6B2002E71D0594BDFF878815B
:105DC0001A78012688F80060574B002A4DD01A78BF
:105DD000002A4AD0564D2F78524D022F574F29D9BD
:105DE00007F0FEF8206895F80090D7F800A007F0BB
:105DF0000EF94FFA89FB0AF80B0009EB0600314651
:105E00002870206807F0E0F8206888F800603F6894
:105E100095F8008007F0FBF84FFA88F907F80900B9
:105E2000B04420684FF48061324685F8008007F066
:105E3000E3F82BE0314607F0C7F820682E78D7F852
:105E4000008007F0E4F84FFA86F9731C08F809009F
:105E5000D9B220684FFA81F83F68297007F0D7F867
:105E6000033607F808002E7010E01B78012113B9E3
:105E7000334A13782BB107F0A7F82A480278511C4F
:105E800003E007F095F8284801210170234A1168C2
:105E90000B8803F4807082B2002AF9D166E003F027
:105EA00040010F461F4D09B3244B2F78D3F80080D3
:105EB00007F0ADF84FFA87F908F80900781CC1B26D
:105EC00029701B4D4FB22A780337BA4205D120689A
:105ED0004FF48061324607F08FF8124B28781A7819
:105EE00051B2884242D1501C18703FE01B063DD58C
:105EF0002B785EB2721C27D0124901330A682B70CE
:105F0000915D07F082F80A4895F9002001789142E6
:105F10002CD120684FF480613A4625E0000A002029
:105F2000FE090020FC090020FD090020EB090020EB
:105F3000EC090020050A0020EA090020F0090020F1
:105F4000F4090020F8090020154A2970117807F09B
:105F50005CF81448017811B9134B1A7832B9134818
:105F600000684FF48061002207F046F80E4A104B9B
:105F7000117893F900004A1C90420ED10D4B0E4946
:105F8000187800220A7028B1084908684FF4407157
:105F900007F032F8094B00221A70BDE8F88F00BFF5
:105FA000EB090020FE090020EC090020000A002077
:105FB000FC090020EA090020FD090020040A002055
:105FC000FFF770BEFFF76EBEF0B5484C89B04FF4D6
:105FD00040651C2307460226204602A9ADF808505A
:105FE0008DF80A308DF80B6000F0B2F940481421AA
:105FF00007608DF80E10204603A9ADF80C508DF8FF
:106000000F6000F0A5F925610825384CA2685205FB
:1060100003D40A2000F0C8FCF7E74FF480660A209A
:10602000666100F0C1FC6F1E0A20266100F0BCFC16
:1060300017F0FF05E9D14FF4006767610A2000F00F
:10604000B3FC66610A2000F0AFFC26610A2000F074
:10605000ABFC022027611C218DF80F002046244C48
:106060004FF440638DF80E1003A9ADF80C3000F02A
:106070006FF9206806F0FEFE04A806F07FFF206896
:106080002A464FF4407106F0B7FF1A484FF4804398
:106090004BF6FF72049001212068ADF81C30ADF87A
:1060A0001620ADF8145006F077FF04A9206806F01A
:1060B000FBFE4FF4A06006F0F9F92221012201A8AD
:1060C0008DF804108DF805508DF806508DF80720D6
:1060D00006F0F6F9212301A82E468DF804308DF83C
:1060E000055006F0EDF909B0F0BD00BF000C01400D
:1060F000000A0020801A060010B54000244CC0B2EF
:1061000020702448244C017000212170234C012070
:106110002070234C2360234C2360234B1A70234AA6
:1061200010702348017023490868838803F40072C3
:1061300091B2A1B9038803F4807291B241B9038886
:1061400003F4007291B20029F9D1012106F030FF69
:1061500018484FF440710068012206F04DFF47F2E5
:106160003053124A117811B1013BFAD100E053B912
:1061700011490A88501C83B20B800E490868FFF74A
:1061800023FF002010BD0A4B187880F0010010BDDD
:10619000050A0020EB090020F4090020FE09002078
:1061A000F0090020F8090020EC090020040A002072
:1061B000F5090020000A0020E809002010B5400081
:1061C000244CC0B220702448244C01702449012082
:1061D000087000212170234C2360234C2360234B43
:1061E0001A70234A10702348017023490868838875
:1061F00003F4007291B2A1B9038803F4807291B2E2
:1062000041B9038803F4007291B20029F9D1012148
:1062100006F0CEFE18484FF440710068012206F0E7
:10622000EBFE47F23053124A117811B1013BFAD11B
:1062300000E053B911490A88501C83B20B800E4903
:106240000868FFF7C1FE002010BD0A4B187880F0E7
:10625000010010BD050A0020EB090020FE09002006
:10626000F4090020F8090020F0090020EC090020C2
:10627000040A0020F5090020000A0020E809002097
:1062800007B502AB03F8012D0122FFF797FF0EBD02
:10629000274B37B51868818A8AB20192019B13F4A3
:1062A000706F02D0234A01211170019B13F4E06F3B
:1062B00031D04FF480610022038B06F09DFE0198DF
:1062C000810528D41A4D2868018801F4007293B220
:1062D0000BBB048804F480718CB29CB1028802F478
:1062E000807399B20029F9D1012106F06DFE1048A2
:1062F0000068028802F4007399B20029F9D1FFF70F
:1063000063FE08E0012106F05FFE28684FF440714B
:10631000224606F071FE06480268938A23F47061F3
:106320000804030C0449938200220A703EBD00BF9A
:10633000000A0020F5090020040A0020FFF7A8BF8A
:10634000FFF7A6BF014B188880B27047E80900200C
:106350002DE9F0410F88002347FA03F2D2072DD52B
:106360008A7803F00705DC08AD0012F0100F18BFA3
:1063700091F803C002F00F0618BF46EA0C064FF072
:106380000F0C0CFA05FC06FA05F550F82480282AB3
:1063900028EA0C0C45EA0C0540F8245006D10122ED
:1063A00002FA03F2C46824EA020206E0482A05D190
:1063B000012202FA03F2C4682243C2600133102BA7
:1063C000CAD1BDE8F081000001F0030230B59200AF
:1063D0000F2404FA02F400FA02F0074B8908023194
:1063E00053F8215025EA040443F8214053F8214092
:1063F000044343F8214030BD0000014008B5036864
:106400001A68904708BD38B505460C4614F8011BBC
:1064100019B12846FFF7F2FFF8E738BD08B5036861
:106420005968884708BD08B503689968884708BD5A
:1064300008B50368DA68904708BD08B503681969AC
:10644000884708BD08B503685A69904708BD70477A
:10645000036B13B15A68006C01E0026AC069101A3C
:1064600018BF01207047436B13B190F84400704788
:10647000826A406A111A4B4253EB01007047836AEB
:106480008169426BC918D160416A994203D9CB1A1C
:106490005360816204E00169CB1A5360002282627A
:1064A000002180F84410406B012106F060BE30B539
:1064B0000446007985B000230D460091C107ADF870
:1064C0000430ADF80630ADF80830ADF80C30ADF85A
:1064D0000A3002D50422ADF80A20820705D5BDF89E
:1064E0000A1041F00803ADF80A30A06C694606F0C6
:1064F0001FFBA56005B030BD026B034610B54069B7
:1065000042B11A6CD9688C1A013A18BF1146005D65
:10651000196410BD196ADA68405C0131B1FBF2F40C
:1065200002FB1411196210BD10B5426A8469A154AE
:10653000416A02690131B1FBF2F402FB1411426BB2
:10654000416232B11368DB070BD4BDE81040FFF79E
:1065500096BF806C40F227710122BDE8104006F022
:106560004BBB10BD214B13B5986021480C465861B8
:106570002048214A2149186314381A6099614FF460
:106580008072586301214FF48040DA601A6106F08E
:1065900039FC4FF4007102231822ADF80010A10756
:1065A0008DF803308DF8022003D515486946FFF7B2
:1065B000CFFE48234FF48060E207ADF800008DF86D
:1065C000023003D50E486946FFF7C2FE01220E21B4
:1065D00001A88DF804108DF805208DF806208DF89F
:1065E000072005F06DFF01481CBD00BFC80C00204E
:1065F000C60B00205800024028100108460A00205F
:10660000000801401F4B13B51F4A98600C468020BC
:106610004021D86019611D481D491A601D4A9861C2
:1066200099644FF4003001215A6106F0F7FB022310
:10663000042218208DF80330A307ADF800208DF850
:10664000020003D514486946FFF782FE082148235B
:10665000E007ADF800108DF8023003D50E4869460A
:10666000FFF776FE012026228DF8050002218DF825
:10667000070001A88DF804208DF8061005F020FF12
:1066800000481CBD140D002028100108060A002037
:1066900000440040460B0020000801402DE9F04175
:1066A0001E46584B90B0984205468846174604D17E
:1066B00010463146FFF756FF07E053480024854255
:1066C00004D110463146FFF79DFF0446002106F035
:1066D00004022671A7600197A5642162E161A162AD
:1066E0006162C4F82C80ADF8081002F0FF0732B1E7
:1066F0004FF40053ADF80A304FF4806701E0ADF875
:106700000A700020ADF80C7016F00107ADF810000B
:1067100002D1ADF80E7002E00421ADF80E1006F0C3
:10672000020606F0FF082EB1BDF80E2042F0080365
:10673000ADF80E30284601A906F0FAF901212846E5
:1067400006F04EFA05A806F005FD0023281D4FF4BB
:106750008051802205900E910F9309930B930A921A
:106760000C9317B3206BD0B16269E16807932023C3
:106770000D930692089106F055FC206B05A906F0D2
:10678000C9FC206B012106F0F2FC284640210122C1
:1067900006F04CFA206B06F0FFFC206405E028466A
:1067A00040F22551012206F027FAB8F1000F24D05B
:1067B000606BE0B1266910210896002607910D96BE
:1067C00006F030FC606B05A906F0A4FC0122606BAA
:1067D000022106F0D7FC606B314606F0DBFC606BF3
:1067E000802146600122284606F020FA05E028466E
:1067F00040F22771012206F0FFF9204610B0BDE8F3
:10680000F08100BF003801400044004010B50B4C3F
:106810004FF4005006F0C4FC0021606B06F0A7FCAA
:10682000626AA36A9A4204D02046BDE81040FFF78E
:1068300026BE012084F8440010BD00BFC80C002013
:106840000D4B986C028802F080018AB29AB19A6A64
:10685000596A8A420AD09969895C01328180196932
:10686000B2FBF1F001FB10229A62704740F22771EF
:10687000002206F0C1B97047C80C00201C4B10B5AF
:106880009A6C1488A4B204F0200188B290B1D96A3D
:1068900019B1938898B288470CE09288D9695869F1
:1068A000D2B24254D869DA68411CB1FBF2F002FB63
:1068B0001011D96104F08004A4B2C4B10C4B9A6ADF
:1068C000586A82420BD09869996C805C013288804A
:1068D0001969B2FBF1F001FB10229A6210BD986CAD
:1068E00040F227710022BDE8104006F085B910BDC6
:1068F000140D0020034B4FF4805208B15A617047C9
:106900001A61704700080140034B4FF4805208B1F0
:106910001A6170475A6170470008014008B5024B80
:106920001968884708BD00BF600D0020054B064868
:106930001A68064982420CBF054A064A00200A60CE
:10694000FFF7ECBF60010020001BB700600D0020C6
:1069500009690008F5680008024B1A68501C1860A5
:10696000704700BF640D002010B5094A094913683B
:106970008C6810688342F8D1074A106811684FF498
:106980007A725043001BB0FBF1F102FB031010BD03
:10699000640D002010E000E0680D0020014B186835
:1069A000704700BF640D002038B50446FFF7DCFFD8
:1069B0000546FFF7D9FF401BA042FAD338BD10B5FA
:1069C00004462CB14FF47A70FFF7EEFF013CF8E774
:1069D00010BD000030B53A4D8DB006AC0FCD0FC4E0
:1069E00095E8030084E8030005F05AFB35480121CF
:1069F00006F014FA44F61D20012106F003FA0120E6
:106A00000146314D06F0F2F9002406F02BFA4FF65C
:106A1000FF732E486946ADF800308DF80240FFF74D
:106A200097FC28466946FFF793FC29486946FFF71B
:106A30008FFC2848426842F000714160FFF776FF02
:106A4000082310202B6128612546234A234B116817
:106A500006A8994205D102199179142901D1102370
:106A6000937100EBC502111D00590135FFF770FC51
:106A70000834032DE9D101A806F06AF901991848F4
:106A8000184AB1FBF0F31848136001684FF47A73A9
:106A9000B1FBF3F2501E154B154AF021586082F8F5
:106AA000231000200721986019601248FFF78CFA24
:106AB000FBF770FB6420FFF782FF0DB030BD00BF15
:106AC0009C0E010807004000000C01400008014036
:106AD000001001400000014060010020001BB700D1
:106AE00040420F00680D00206401002010E000E02B
:106AF00000ED00E00058004010B540F2DB146043A8
:106B00000D4B102208215A61841E19610A48C3687E
:106B100083F01002C260C16881F00803C3602046A0
:106B2000FFF74DFF0120FFF7F9FE1920FFF747FFA0
:106B30000020FFF7F3FEE9E7000C014010B1034A23
:106B4000034B1A6003480449C8607047EFBEADDECE
:106B5000F04F00200400FA0500ED00E00000000006
:106B60002DE9F84F384E04463768384606F022FBC8
:106B70000546384606F092FB76688046304606F0B9
:106B800019FB8346304606F089FBD4F8049006468C
:106B900029464846FAF796F8A7688246414638469D
:106BA000FAF790F801465046F9F782FF21688246CD
:106BB0005846FAF787F8414604464846FAF782F8FD
:106BC0003146FAF77FF801462046F9F773FF314660
:106BD00004463846FAF776F82946FAF773F801467C
:106BE0002046F9F767FF0146504606F0E3FB1749D8
:106BF000FAF768F8F9F71AFC11A3D3E90023F9F7BB
:106C000093FD134B044618680D46F9F70FFC024636
:106C10000B4620462946F9F7ABFA00220D4BF9F74F
:106C200083FDF9F7F1FE06F0F9FA81B20A0444BFD8
:106C300000F5B47189B208B2BDE8F88FAFF30080F7
:106C4000182D4454FB210940CC0D00200000E144E4
:106C50008C0D00200000244010B51D4C2088F9F751
:106C6000DDFF1C49FAF72EF806F0D8FA1A4B188007
:106C70002088F9F7D3FF01461848FAF7D7F81849E2
:106C8000FAF7D4F8174908601748B0F87000F9F718
:106C9000C5FF01461548FAF7C9F8F9F7C7FB0AA37B
:106CA000D3E90023F9F716FCF9F7AEFE104A10609D
:106CB000082002F0D7FB18B1BDE81040FEF7D6BDA2
:106CC00010BD00BFAFF300803B597E90A9E7814023
:106CD00026000020C903683FC80D00200AE81C41B7
:106CE00000401C460C1E0020B0180020000061442B
:106CF000281E0020AFF300802DE9F0410446006813
:106D00000D460146F9F7DEFFD4F8048006464146F9
:106D10004046F9F7D7FF01463046F9F7CBFEA768A2
:106D2000064639463846F9F7CDFF01463046F9F7B1
:106D3000C1FE06F0D5FC00210646FAF757F970B9F6
:106D400020683146FAF772F8314628606068FAF731
:106D50006DF831466860A068FAF768F8A860BDE889
:106D6000F0812DE9F04F0C68836889B0D0F800A05D
:106D7000D0F804800646204603938B4606F01AFAA4
:106D80000746204606F08AFADBF804408146204692
:106D900006F010FA0546204606F080FADBF80820D7
:106DA00004461046019206F005FA8346019806F063
:106DB00075FA394602905846F9F784FF394604902F
:106DC0000298F9F77FFF594605904846F9F77AFF90
:106DD000029906904846F9F775FF294607905846EC
:106DE000F9F770FF01465046F9F76CFF21468346DC
:106DF0000698F9F767FF01460598F9F75BFE01462B
:106E00004046F9F75FFF01465846F9F753FE214621
:106E100083460498F9F756FF01460798F9F748FEAC
:106E200001460398F9F74EFF01465846F9F742FE2E
:106E30003060029905F10040F9F744FF01465046E1
:106E4000F9F740FF214683460798F9F73BFF0146D3
:106E50000498F9F72DFE01464046F9F733FF014645
:106E60005846F9F727FE214683460598F9F72AFF89
:106E700001460698F9F71EFE01460398F9F722FF2E
:106E800001465846F9F716FE214670605046F9F75C
:106E900019FF2946044609F10040F9F713FF01469E
:106EA0004046F9F70FFF01462046F9F703FE394641
:106EB00004462846F9F706FF01460398F9F702FF52
:106EC00001462046F9F7F6FDB06009B0BDE8F08F45
:106ED0001FB50B684A6889680193039101A9029262
:106EE000FFF73FFF05B000BD80EAE073A3EBE0735E
:106EF0008B4206DB002801DD401A704702D04018A3
:106F000070470020704700002DE9F041524B86B0D9
:106F10001A685B6802F1004203F1004301934F4B92
:106F20000646B3F900000092F9F778FE00F1004040
:106F3000F9F77CFA46A3D3E90023F9F7CBFAF9F77E
:106F400063FD474C0290B4F90000F9F767FE039027
:106F5000B4F90200F9F762FE0490B4F90400F9F7FD
:106F60005DFE6946059003A8FFF7FBFE3D4B93F8D5
:106F70004030012B16D13C48417869B93B4C402543
:106F8000226892FBF5F7D01BF9F748FE0599F9F74F
:106F900091FDFAF75DF82060344B4021186890FBB2
:106FA000F1F001E0324B1888F9F738FE01460598F8
:106FB000F9F77EFD05903046F9F72CFE2D4907467E
:106FC000F9F778FD01463846F9F730FF2A4D0746B4
:106FD0002C6805982146F9F76BFD01463846F9F70C
:106FE00071FE01462046F9F765FD244C28601D4DD1
:106FF00007460398D4F8008006F010F995F8301091
:10700000FFF772FF08EB000204982260D4F80480B6
:1070100006F004F995F83010FFF766FF08EB00035F
:1070200038466360D4F8088006F0F8F895F82F1019
:10703000FFF75AFF1249134B0A684044A0601868D2
:10704000B6180E60411C196006B0BDE8F08100BFA3
:10705000399D52A246DF913FCC0D0020F21D002049
:10706000201E0020B0180020871E0020A00D002048
:10707000260000203661823CD40D0020001E002036
:10708000E80D0020C40D00202DE9F04F87B0FEF779
:107090001FFD022002F0E6F9002800F0A781FEF7AC
:1070A0007DFBFFF761FCAA4C05462768C71B3846E5
:1070B000F9F7B0FDA749C968F9F704FE8346A64869
:1070C000256090F82E8000252C462E46A34A105F9E
:1070D000F9F7A4FD5946F9F7F5FD03AB5851B8F19E
:1070E000000F27D04046F9F799FD01464FF07E503A
:1070F000F9F79CFEDFF8A492824651464FF07E508D
:10710000F9F7D6FC55F80910F9F7DCFD9449034668
:10711000085F0193F9F782FD5146F9F7D3FD014667
:107120000198F9F7C7FC49F80500F9F791FF8D4A76
:10713000105303E08A498B4A605AA052894B0435A8
:10714000E15E0234062C01FB0166BFD1864A642051
:10715000138846435B43854803A996FBF3F6FFF784
:10716000B7FE082002F07EF920B1814803A9FFF79D
:10717000AFFE07E07F4803A9FFF7AAFE7D4801465E
:10718000FFF7BAFD493EB1B23B2904D9082002F00D
:1071900069F948BB50E0784CB4F8F000F9F73AFDD3
:1071A0004FF07E518046F9F785FC01464FF07E5046
:1071B000F9F73CFE002406466C4D404655F8141085
:1071C000F9F780FD81466748005FF9F727FD014622
:1071D0004846F9F76FFC3146F9F774FD45F814009D
:1071E0000234062CE8D1D1E7634A0024B2F8F20059
:1071F000F9F710FD4FF07E518046F9F75BFC014630
:107200004FF07E50F9F712FE0646594D404655F8AC
:107210001410F9F757FD594B8146185FF9F7FEFC3A
:1072200001464846F9F746FC3146F9F74BFD45F86B
:1072300014000234062CE8D151494C4DB1F900003C
:10724000F9F7ECFCAC68014620460126F9F7F6FE9A
:1072500000B906464B4821464673686806F0AAF80E
:10726000494C2A682060686802F100460146F9F737
:1072700029FDD5F80880054641464046F9F722FD2C
:1072800001462846F9F716FC06F02AFA0146304670
:1072900006F090F860602068F9F7C8F82AA3D3E9EF
:1072A0000023F9F717F9F9F7AFFB05F0B7FF374DF2
:1072B00028806068F9F7BAF823A3D3E90023F9F727
:1072C00009F9F9F7A1FB05F0A9FF6880082002F091
:1072D000C9F82F4C08B1264800E02648FFF740FCCB
:1072E0001D4D20803846FFF70FFE95F87230002BB9
:1072F00000F080801D4908688C684F680146F9F7E6
:10730000E1FC394606463846F9F7DCFC01463046D2
:10731000F9F7D0FB214606462046F9F7D3FC014693
:107320003046F9F7C7FB06F0DBF901462046F9F7CE
:107330007DFD18490446F9F76DFE88B3164A002012
:10734000108057E0AFF300803B597E90A9E7814061
:107350007C0D0020DC1D0020B0180020F81D00204E
:10736000101E0020201E0020260000202C1E0020C1
:10737000B00D0020280000207C190020D41D002022
:10738000C80D0020871E0020CC0D0020940D002089
:10739000F21D00208FC2753C9E0D0020800D002044
:1073A000204605F0B7FF264B1968F9F78BFC05F06E
:1073B00035FFB0F5617FA8BF4FF46170F9F724F88D
:1073C0001DA3D3E90023F9F7AFF9F9F71DFB05F089
:1073D00065FF044695F87200F9F720FC2146F9F79D
:1073E00071FC05F01BFF174B188003E0164B18804B
:1073F00058809880154B5979154B012907D01548AD
:107400001A8859889B8802804180838011E0124944
:10741000B3F90420B1F9000002EB4000032290FB15
:10742000F2F080B20B4A088019885B889080118046
:10743000538007B0BDE8F08FA2EB0FE5DD16964054
:10744000281E00209E0D0020101E00207C19002008
:10745000F81D0020980D0020CA0D0020AFF3008019
:10746000044A054805490023136053609360036094
:107470000B607047001E0020C40D0020E80D0020A6
:107480002DE9F04F85B0FFF76FFABA4B46F2A7121D
:107490001F68C71B9742029740F2A881B64C18603C
:1074A000208868B3B54DB64E95F83130B54A31688D
:1074B00010685F1E082391FBF3F5491BB0FBF7F73B
:1074C0007A18326092FBF3F0F9F7A8FBAE49F9F7AE
:1074D000ADFCAE4905F070FF01464FF07E50F9F764
:1074E000E7FAAB49F9F7EEFBF9F7B2FDA94E2588AB
:1074F000A94FAA4B3060691E0020386018602180B7
:107500009E4CA04894F831200768561EB7FBF6F051
:10751000F9F780FB9C49F9F789FC9C4905F04CFF81
:1075200001464FF07E50F9F7C3FA9949F9F7CAFBC3
:1075300005F074FE9A4F656B80463868F9F76EFB6C
:107540002946F9F7BFFB934B06461968C1EB0800C3
:10755000F9F764FB294681464FF07E50F9F7A8FA07
:1075600001464846F9F7AEFB01463046F9F7A2FA64
:1075700005F054FE024638608A488B4E006800923F
:10758000F9F748FB89490546F9F79CFB8346B06843
:10759000F9F744FB864B06461868F9F73FFB0146AE
:1075A0003046F9F743FC834906460968F9F78AFB38
:1075B0002946F9F787FB4FF07C510390F9F782FBDE
:1075C0005946F9F77FFB744D8446D5F8008059463B
:1075D0004046D4F83CA0CDF804C0F9F773FBDDF8C1
:1075E00004B0DFF8B89101465846F9F763FAD9F8C4
:1075F0000010F9F75FFA5146F9F764FB009A8346E9
:107600001046F9F70BFB514603464FF07E500093AE
:10761000F9F74EFA01460098F9F754FB014658462F
:10762000F9F748FAC9F80000F9F712FDDFF8AC9154
:107630000399C9F800004046F9F73CFADFF8A08149
:107640002860FFF70DFFD7F800A0D8F80070C7EB4F
:107650000A00F9F7E3FA5849F9F734FB8346029830
:10766000F9F7D8FA01465846F9F7E0FBF9F7F0FCCC
:107670004FF496725149C8F800A0FCF799FB0A2113
:10768000FFF732FCA76B296882463846F9F71AFBE8
:1076900080465046F9F7C2FA394682464FF07E508E
:1076A000F9F706FA01465046F9F70CFB0146404649
:1076B000F9F700FA286005F0B1FD05210546FFF74E
:1076C00013FC3F493F4AD9F80030086010683E4932
:1076D000C01A4FF4FA72FCF76BFB0A21FFF704FCA7
:1076E0002779802178434FF4967290FBF1F033496B
:1076F000FCF75EFBC5EB0008A57A202008FB05F22D
:107700002E4992FBF0F04FF49672FCF751FB237D6B
:107710002E4F08FB03F12E4D3B680822286091FB99
:10772000F2F0C0182B494FF448323860FCF740FBA8
:107730002A6838604FF4806790FBF7F18F18A07FBC
:107740002F60F9F76BFA244C804621683046F9F730
:10775000B1F901464046F9F7B5FA4FF07251F9F721
:10776000B1FAF9F775FC6FF095019622FCF720FB52
:10777000381A37E0900D0020E4090020B0180020EE
:10778000F00D0020DC0D002080E6C547B1DC423E54
:10779000D048874A700D0020E40D00206C0D0020B9
:1077A000A40D0020E80D0020001E0020BD37863506
:1077B000C40D00200C1E002000247449D4FEFFFFDD
:1077C000E00D00201C1E00200CFEFFFFAC0D002071
:1077D000EC0D002000E0FCFF740D0020181E0020BE
:1077E000D80D002028602660012000E0002005B0B0
:1077F000BDE8F08F10B5054C00202188FBF7C0F9DB
:1078000061880120BDE81040FBF7BAB934000020C0
:107810000A4A02EBC00393F87B10FF2904D019B188
:10782000074830F8110007E00728DABF02EBC00074
:10783000B0F8780040F2DC5000B27047B018002079
:10784000C81E002010B500244FF48040FCF704F956
:10785000064B10B1B3F8DA0001E0B3F8D400044AE3
:10786000A0520234182CEFD110BD00BF7C190020AB
:10787000501E0020F8B53B4D3B4E6B793B4C06EB60
:10788000C300417820202160FCF7E6F8324608B1B9
:10789000012626606B79162B1CD10024314E002165
:1078A000A6193069F9F7A2FB28B14FF48040FCF724
:1078B000D3F850BB23E02E4B06F110001D190FC862
:1078C00085E80F002B4910340A78531CC02C0B702C
:1078D000E4D1EAE7274F12F8336002EBC3003E70B1
:1078E0004768002FE1D00024B442DEDA204D2101A8
:1078F0006D187A180FCA013485E80F00F4E71948AB
:107900001D4B4179082923D124E01A4E3678012EE7
:10791000F5D91A4C00251034B542F0DA54F8100CA1
:107920004FF07C51F9F7CEF94FF07C5144F8100C30
:1079300054F8140CF9F7C6F94FF07C5144F8140CC4
:1079400054F80C0CF9F7BEF9013544F80C0CE2E7D9
:107950000E2901D1012200E000221A74BDE8F8408E
:10796000FFF770BF7C190020B0110108F80D00204E
:10797000FC0D0020F40D0020871E0020040E0020C6
:10798000F0B50023461C0E4A002198181033C02B76
:107990000161F8D10B4F07EBC6035F6807B9F0BD73
:1079A0000024084A12F83600844208DA064D210104
:1079B0004D197B180FCB013485E80F00F1E7F0BDBE
:1079C0007C190020B01101088C190020284B10B53B
:1079D000186800284AD027494A79531E142B3DD8ED
:1079E000DFE803F00B3C3C24403C3C1C3C3C3C3C72
:1079F0003C2C3C3C3C3C3C242C001F4890F8BB10E9
:107A000031B11E4B00205989BDE81040FBF7B8B8D2
:107A10001B4A50780028F4D10146F5E7174C0020A6
:107A2000E188FBF7ADF801202189EDE7134C002038
:107A30002189FBF7A5F801206189E5E70F4C0020BB
:107A4000E188FBF79DF801202189FBF799F80220D6
:107A50006189FBF795F80320A189D5E72020FBF782
:107A6000FBFF18B1BDE81040FFF7C4BE10BD00BF5A
:107A7000F80D00207C190020B018002034000020F0
:107A8000871E002010B50024064B1878A04208D9A4
:107A90000549204631F814100134FBF763F8E4B2CD
:107AA000F2E710BDF40D0020381E0020064B1A78B6
:107AB0000023D9B2914204D2044921F813000133C2
:107AC000F7E7FFF7DFBF00BFF40D0020381E0020EE
:107AD0002DE9F84FB24B187803280FD9B149B24CB1
:107AE000B1F904206FF06305002AB8BF5242A91A09
:107AF000B4F904006432FCF75BF9A080A84A167858
:107B0000012E1DD8A94EAA4C75796A1E142A00F2BE
:107B1000F981DFE812F0C200F701F7018400D50017
:107B2000F701F7017101F701F701F701F701F7011B
:107B3000F100F701F701F701F701F7015E00C70156
:107B40009B48994B90F9BA90964FB3F90440C9F10C
:107B50000001B7F806A004FB01F95F88B3F80080C4
:107B6000944C00251034B542CCD20FFA8AF0F9F7C4
:107B700055F854F8101CF9F7A5F8834638B2F9F710
:107B80004DF854F8081CF9F79DF801465846F8F7E7
:107B900091FF83460FFA88F0F9F740F854F80C1C6F
:107BA000F9F790F801465846F8F784FF83464846AF
:107BB000F9F734F854F8041CF9F784F801465846EC
:107BC000F8F778FFF9F744FA7B4B23F815000135F5
:107BD000C8E794F89A20744D12F0010F6B880CBF1F
:107BE00001264FF0FF365E43744CB7B20420278164
:107BF000FFF70EFE29886E4D381895F8A2302081C7
:107C000013F0010F0CBF01224FF0FF324A43052051
:107C100096B26681FFF7FCFD3718678172E194F830
:107C20009A50614805F002084FFA88F6002E0CBF02
:107C300001214FF0FF3115F0010F45880CBF0122E3
:107C40004FF0FF326A438688042001FB06F497B2A6
:107C5000FFF7DEFD1FFA84F808EB00035448F9181B
:107C600090F8A270554C07F0020253B22181002B0C
:107C70000CBF01214FF0FF314E4317F0010F0CBF35
:107C800001204FF0FF3045430520FFF7C1FDB6B29C
:107C9000ADB23718EA19628134E1434994F8A24041
:107CA0008E8814F0010F0CBF01234FF0FF33052025
:107CB0005E43FFF7ADFDB5B2404F2818788121E152
:107CC0000020FFF7A5FD3E4F94F97A30B7F9026026
:107CD0003A4D7343322693FBF6F140182880012079
:107CE000FFF796FDB7F9002094F98240544394FBC6
:107CF000F6F3C7186F8005E1324C607820B9B6F80A
:107D0000D4202E4BDA810AE02649B6F8D220B1F908
:107D10000600B6F8D010FCF74BF8284DE881274E46
:107D2000254CF7892780214F97F8190130B3204D52
:107D30000220FFF76DFDB5F98410B5F98620FCF738
:107D400037F8214BB7F812111A880C1A16B220B264
:107D5000864203DA97F81961B41803E003DD97F857
:107D60001971D41B1C8095F98A50B3F90030642234
:107D70006B43124F93FBF2F00918B980114C0F4D71
:107D8000A67A56B1074B1A880324EA802A8198887C
:107D900068815988A981094D18E0034BF3E700BFBA
:107DA000F40D0020441D00204C1D00207C190020F3
:107DB000B0180020FC0D0020381E002034000020E8
:107DC000940D0020871E0020F60D0020AA4FB5F963
:107DD000062007EBC40696F97A3064205A4392FBDA
:107DE000F0F7EF802046FFF713FD01343918E980E2
:107DF0000235072CEAD185E0A04B5A7822B9B6F8B3
:107E0000D4709F49CF810AE09E48B6F8D010B6F8EA
:107E1000D220B0F90600FBF7CBFF994EF081964EC9
:107E2000974B964A96F89270974DDC89907A17F0A6
:107E3000010F2C800CBF01254FF0FF3508B191498F
:107E400000E09249488807F00204454396F89A609A
:107E5000098862B2002A0CBF01274FF0FF3716F0E5
:107E6000010F0CBF01244FF0FF3407FB01556043A5
:107E700006F0020257B2DD80002F0CBF01254FF043
:107E8000FF3505FB010018810320FFF7C1FC7C4E84
:107E9000F388C1180420F180FFF7BAFC3489021975
:107EA00032812FE0794F0324BF88734B03EBC4006A
:107EB00090F87A60C4F1060306F002014DB2002D7D
:107EC0000CBF01224FF0FF327A437049580831F855
:107ED000105016F0010F0CBF01264FF0FF3606FBC5
:107EE0000522674D96B225F814602046FFF790FCF6
:107EF000331825F814300134072CD6D1614F62496C
:107F0000F88808802020FBF7A7FD002841D000203A
:107F1000FFF77EFC5A4C054620800120FFF778FCD5
:107F20005B4A6080137AA3B3534F5A4A97F8BC1048
:107F300001F00206F3B2CBB1B2F9003097F982102A
:107F400097F97A70B2F9022059437B4253433226A3
:107F500091FBF6F16FF0310789B293FBF7F28F18BE
:107F60007D1993FBF6F625808E1910E097F97A10AB
:107F7000B2F9026097F982704E43B2F900203221C3
:107F8000574396FBF1F3ED18258097FBF1F6801926
:107F90006080414C384D04F11006B4F90200B5F987
:107FA0007410B5F97620FBF703FF24F8020F0835AB
:107FB000B442F2D1304991F8BC3003F00402D7B298
:107FC0002FB93148354B07881C7801221CE0344D0D
:107FD00068790E280AD0082808D0324C04EBC0017A
:107FE0004B78002B14BF0225002500E00425002457
:107FF0002D4F621907EB4401D0B209890134FAF719
:10800000BFFD042CF4D1DCE7A24209D21E483FB2E6
:1080100030F912100132B942A8BF0F46BFB2F3E7E0
:108020000024A0461D4A1178884567D21C4D3BB2FA
:10803000B5F8D200834204DD134DC21B615B5018BA
:1080400060534FF48040FBF707FD0F4D70B3164BA4
:1080500040F2DC51B3F90620114B8A42285FC7BFBA
:10806000B3F8D810B3F8D220B3F8D410B3F8D620B0
:10807000FBF79EFE285336E0B0180020871E002034
:1080800034000020441D0020381E00204C1D00201C
:10809000981E0020940D002032000020F40D0020D6
:1080A0007C190020B0110108C81E0020144E285F62
:1080B000B6F8D010B6F8D220FBF77AFE114BB6F81E
:1080C0001411B3F9062005EB04098A4228530ADA91
:1080D0001020FBF7C1FC10B9B6F8D00001E0B6F8EB
:1080E000D400A9F80000084A507818B90749084B8D
:1080F000625AE25208F10108023493E7BDE8F88FB2
:108100007C190020C81E0020871E0020501E002061
:10811000381E0020024B1868003018BF012070473D
:10812000F80D002044F25063984203DDA0F50C40A6
:10813000A038704703498842BCBF00F50C40A0300E
:10814000704700BFB0B9FFFF10B5F8F767FD002119
:108150000446F8F773FF08B1204601E004F100403F
:108160000549F8F763FE0549F8F7ACFD05F022F87C
:10817000034B186010BD00BF8096184B35FA8E3C3B
:108180004400002010B5044C002320702361FEF74A
:1081900005FC606110BD00BF6C1E0020F8B51D46D7
:1081A00014460E46F8F73AFD6968F8F78BFD31463C
:1081B000F8F788FD2168F8F77DFC2060F8F748FFA4
:1081C000ED68074605F10040F8F742FF06462846ED
:1081D000F8F73EFF314602463846FBF7E9FDF8F76F
:1081E0001DFD2060F8F734FFF8BD0000F8B5101A47
:1081F0000C461F46F8F712FD0546381BF8F70EFD32
:10820000174B079E1968F8F75DFD29460446284676
:10821000F8F758FD214607462046F8F753FD01467A
:108220003846F8F747FC05F05BFA0E49F8F74AFDC7
:10823000F8F734FF06990860214605F1004005F083
:10824000B9F80949F8F73EFD0849F8F733FCF8F7A3
:10825000FFFE0028BCBF00F50C40A0303060F8BD28
:10826000440000202C7D8E3FA00CB34500A00C469E
:1082700010B50446002003460D49CA5CA2B12E2A5F
:1082800004D1013394B1C91800220A55084A0A21C1
:10829000D25C4843A2F13001092901D83038801856
:1082A0000E2B02D80133E7E710BD002010BD00BF40
:1082B00002100020F8B52D4B93F81C0110B10128D5
:1082C00050D10AE02A4B2B4A58782B4B02EB001175
:1082D00049685868FEF7ACF841E0274D6868FEF73A
:1082E000ACF800283ED0224C2178264601291ED128
:1082F000FEF754FB06466069321A632A35D92169B4
:10830000042912D81B4F686807EB01135968FEF760
:108310008FF8607807EB0017B9686868FEF773F8A4
:1083200022696661511C21611CE0022018E022696B
:108330003AB964780F4B686803EB04114968FEF79B
:1083400077F833690A4C8B2B09D80C4A0A48D15C60
:108350004068FEF753F821694B1C236102E00320BB
:10836000FFF710FF024A00205060F8BD7C19002082
:108370006C1E0020D01601080C1F002042160108B8
:1083800010B50B4CE37A8BB10A48017804290DD95A
:10839000094A0A4B1068516818605960FFF7D4FE0B
:1083A0000748084B028801211A80217310BD00BFC5
:1083B000871E00208E1D0020701D0020541D0020EF
:1083C000F21D0020760F0020002370B51C460F48D8
:1083D00000211952142060430D4A0E4E0E4D995241
:1083E00000223250595335180C4E6960AA60325041
:1083F00035180B4E01346960AA6002333518022C1F
:1084000032506960AA60E2D170BD00BF281D002013
:1084100076080020340F00202C1D0020E80E0020DC
:10842000B80F002070B5204C204D6079F8F7F2FBB2
:108430001F49F8F7FBFC2860E07BF8F7EBFB1C49D1
:10844000F8F7F4FC1B4E6860EE60A079F8F7E2FBE9
:108450001949F8F7EBFC194D2860207CF8F7DAFB96
:108460001349F8F7E3FC6860A07EF8F7D3FB1449E2
:10847000F8F7DCFCEE60A860E079F8F7CBFB0E497A
:10848000F8F7D4FC0F4D2860607CF8F7C3FB08496F
:10849000F8F7CCFC6860E07EF8F7BCFB0849F8F719
:1084A000C5FCEE60A86070BDB0180020600F002011
:1084B0000000C8420000FA4400002041940F002050
:1084C00000007A44240F002070B5124C05460020AD
:1084D000FFF758FE6570FEF761FA0F4BA06093F846
:1084E0001C0100266660B0420CBF01240324FFF784
:1084F00099FF0A49234601EB05156A683146084889
:10850000FEF7CCF8074A50600120BDE87040FFF745
:1085100039BE00BF6C1E00207C190020D016010857
:10852000004400400C1F0020F8B5184B18780328B1
:1085300028D11749082210240A610C61154C606883
:10854000FDF76CFF58B1124D08266E616068276810
:10855000FDF769FF01463846FDF750FF2E610D4CCF
:108560002068FDF75BFF0028E8D0094D102694E84D
:1085700081006E61FDF757FF01463846FDF73EFF6B
:108580002E61DBE74FF0FF30F8BD00BF6C1E00200E
:10859000000C01400C1F0020F7B50368164C174D66
:1085A00023600968164E61600068FFF7CDFD94E80E
:1085B0000C0014480196009095E80300FFF716FEA2
:1085C0006B68114A61683668C81A1660F8F726FBAE
:1085D0000E4A0F4F1168F8F775FBF8F739FD296857
:1085E000786020680B4A431A0B483B60B0F8C4100F
:1085F0000A4B16601980FEBD7C0F0020701D002004
:10860000E40F0020F00F0020780F0020440000202D
:1086100020100020F80F0020B01800201E100020AD
:10862000264BF0B51D68024600F11001167814467D
:10863000AB195B78013203F00403DBB263B18A4209
:10864000F4D10020F0BD13B10A225343DBB210F87D
:10865000011B30395B18DBB2211A0229F3DC00213F
:10866000844209D911B10A225143C9B210F8012B31
:10867000303A8918C9B2F3E72E2E11D10134042003
:1086800000220A2672432678AF197F7807F0040784
:10869000FFB217B1303A921901340138F1D100E03C
:1086A0000022074C6420614300FB021106240548A8
:1086B000B1FBF4F200FB0320F0BD00BF80010020FD
:1086C00040420F00809698002DE9F04F9A4B91B0F0
:1086D0005868C0B9994C21784A1E032A00F20286D4
:1086E000DFE812F0C605C605DF05C9056068FDF7BD
:1086F0009AFE9349044691F81C31012B00F0DF806B
:1087000008D3022B06D08C4C6068FDF787FE00284A
:10871000ECD1DFE7242C07D18A4B8B4A8B4C00210C
:10872000197011702170C5E02C2C02D02A2C40F059
:108730008280854D834A2978854B157800205854CE
:10874000844AB5B918781570472868D159785029E6
:1087500065D19878472840F0B385D978472940F00B
:10876000AF851B79412B40F0AB850120107000F0E4
:10877000A7BD117801293AD1022D05D11846FFF77E
:108780004FFF754908604AE0032D07D11978532936
:1087900045D1714802685342036040E0042D05D181
:1087A0001846FFF73DFF6C4B586038E0052D07D1A8
:1087B0001B78572B33D168494A68504248602EE0F5
:1087C000062D07D119786548302994BF0021012171
:1087D000C17224E0072D04D1FFF74AFD604A1070F2
:1087E0001DE0092D1BD1FFF743FD5E4B16E002296A
:1087F00015D1072D0CD10120FFF73AFD41F21842A7
:1088000050434FF47A71584BB0FBF1F0188006E0FA
:10881000082D04D10120FFF72BFD544B1880494B44
:108820004949013500202A2C1D70087039D1504863
:10883000012404703EE00D2C4D4A01D00A2C26D1B3
:108840001478FCB1424C21786478A1F13000C3B2B5
:10885000092B84BFA1F13703DBB2A4F1300003F090
:108860000F02C3B21101092B84BFA4F13703DBB29D
:10887000364C03F00F0289182078CBB2C21A51424D
:1088800051EB02043A4B002018707CB912E02E49DB
:108890000B780E2B03D82E48C45401330B7012787A
:1088A00042B92A4B1A7854401C7003E0294A1078C8
:1088B000012800D00020C00700F1338123E72D4BB1
:1088C0000022197808293FF61EAFDFE801F00A05FB
:1088D0001119275F7C96A000622801D1022105E0D2
:1088E0001A70B52C7FF40FAF1C78611C19700AE761
:1088F0002149224A03261E7008701070204B0BE09D
:108900001E4E0421197032781D4BA1181878CAB276
:10891000101818701B4B32701C70F4E6052119708A
:10892000164B174E1A783078A118CAB2101830704A
:10893000154E1A703480E6E60C1F00206C1E0020D5
:108940007C1900201D100020F40F00208C0F002047
:1089500002100020B00F0020701D0020871E002094
:108960008E1D0020261D0020301D00207C080020C8
:10897000720F0020740F002000100020700F0020E4
:10898000710F0020E40E0020220F00206C49062603
:108990001E700A786B4BA6181878F2B2101818706F
:1089A000694B0A70198801EB0424A6B2B6F5007F62
:1089B00001D81E8003E000221A80644B1A70002444
:1089C000634B00F052BC5E495E4E0A783078A318C3
:1089D000DAB2101830705E4E0A7033885A4AC72BCC
:1089E00098BF5C49108898BFCC545C1CA1B28842E7
:1089F00031807FF488AE072107E0514A08261E70B7
:108A0000137883423FF47FAE0021504B6EE74D4E0A
:108A10001A70337883427FF476AE4F4C2078062864
:108A20003BD005D8022813D003287FF46CAE23E096
:108A3000122847D030287FF466AE464A474C167954
:108A4000444A102E88BF102626702178002347E064
:108A5000404C434E6368A06821697360414B4FF4FA
:108A60007A723060404C91FBF2F618783F492680CC
:108A7000C87201223E4923E036494A7912F00100CA
:108A800004D00E79F41E634253EB0400354908709C
:108A9000002839D1354AD07236E02E4EF47A14F0DF
:108AA000010104D0B07AC21E534253EB02012D4E95
:108AB000317009B92D4CE17226482E4990F82F20CB
:108AC0000A7021E023482C498669426942F21074F9
:108AD0002A4B96FBF4F00A80188001222849EFE720
:108AE0000C328B4210DA12F8046C264812F8034C50
:108AF0001E54254E25489C5512F8014C16781C54DE
:108B0000234C1E550133EBE719490A78002A3FF43C
:108B1000FAAD1B4B1E78002E3FF4F5AD00240C700F
:108B20001C701C4CA068E060FDF738FFA06020209E
:108B300000F0A2FC18490A78012A2FD100232EE068
:108B4000700F0020710F0020220F0020740F0020F2
:108B50005C0F00202C100020E40E00208F1D002050
:108B6000701D00201C100020261D0020871E0020E4
:108B7000730F00208E1D0020301D00207C08002077
:108B800001100020141D00205E1D0020781D002013
:108B9000981D00206C1E00207408002001237E4CCC
:108BA0000B70E07A00283FF4AEAD7C490A78042AC5
:108BB0007FF6A9AD677807B92773257B15B90FB183
:108BC000FFF7DEFB764E05213378764F5C1C94FB75
:108BD000F1F001FB10423270734E97F800C0734DF4
:108BE00006EB82020023724C72491F59DFF810E233
:108BF0007148724E5F5097FBFEF1195006FB0170F1
:108C0000DFF8009203EB040A42F2107490FBF4F7D1
:108C10001668BCB253F809701060C6EB07084044F0
:108C2000052643F8090090FBF6F00EFB01016448AD
:108C3000BCF1010F25F8024F195005D1023CB4F5E3
:108C4000797F98BFCAF8001004331432082BCAD1B8
:108C5000FDF7A4FE5B4D5C4C2A68801AF7F7DAFF3B
:108C60005A49F8F7E3F82060FDF798FE2860256878
:108C70004FF07E512846F8F7C3F908B94FF07E55FA
:108C800025600CA90DAC4A48514B0194009103C8D2
:108C90000CCBFFF7ABFA0C9A64234E49B2FBF3F00E
:108CA00008800D9A3C4892FBF3F34B4C027B2380E7
:108CB0000AB90A80228049490C78002C36D0424FEC
:108CC0004FF07E503968F8F7B1F8454D384E2B68B3
:108CD00004463068C01AF7F7A1FF2146F7F7F2FF04
:108CE000F8F7B6F9726869683E4D0746501AF7F70B
:108CF00095FF2968F7F7E6FF2146F7F7E3FFF8F756
:108D0000A7F904B238480225B0F902303FB2E218A0
:108D100092FBF5F1B0F900208BB2B918334C91FBFE
:108D2000F5F291B263802180438001802B4B0120BA
:108D30001F4C1870184B6168294A20681C7A5160D2
:108D400010601CB9DA79002A3FF4DDAC284E294DB9
:108D5000294C01960095164F94E80C00FFF746FA4F
:108D600061687868254E081AF7F758FF1D4B196897
:108D7000F7F7A8FFF8F76CF970600A48226890F9D5
:108D800000303C68012BC4EB020131603CD0022B67
:108D90007FF4B9ACF2E000BF871E00208E1D0020DA
:108DA000281000201C080020BC0E00208C0F002082
:108DB000701D002014100020A80F0020806967FF9C
:108DC000180F0020140F0020A40F002000007A4488
:108DD000541D0020521D00205C1D0020100F00209B
:108DE000840F002044000020FC0F0020B20F002060
:108DF000E40F0020F00F00207C0F00202010002046
:108E000080969800E80F0020002634463546DFF8AB
:108E100074B28B4F5BF82580DFF864924046F7F719
:108E2000FDFE3968F7F74EFFF8F712F934F809102C
:108E3000844B421A90B2E05207B2CDF80890DFF8A6
:108E4000489238460397F7F7E9FED9F80010F7F78C
:108E500039FFF8F7FDF881B27B48142202FB0507C1
:108E6000DFF800A2039B089103EB0800DAF800107A
:108E70004B463A46FFF792F90899DFF810820A1834
:108E80005BF82500DAF800B024F80820089058466E
:108E9000F7F7CCFAD7F808A0CDE904015046F7F768
:108EA000C5FA6A4BCDE9060193F8C000F7F7B2FEA8
:108EB000F7F7BCFA60A3D3E90023F7F70BFB0246F0
:108EC0000B4600206249F7F72FFCDDE90423F7F792
:108ED0004FF90B460246DDE90401F7F725FC089A35
:108EE000CDE9040179680135501AF7F797FE594624
:108EF000F7F79CFF5146F7F7DBFDF7F797FA0246C5
:108F00000B46DDE90401F7F7E5FA0B460246DDE919
:108F10000601F7F72DF9F7F777FD089938617960C1
:108F2000B860D9F80810F7F7CDFEF8F791F849497D
:108F30004FF4FA62FAF73CFFDDF808C034F8081085
:108F400034F80C20313293B2622B98BF00204018C5
:108F500082B224F8082010B23F4940F6B832FAF73E
:108F600027FF394B28F8040099593C480234315006
:108F70001436022D7FF44BAFFFF7C5BB2F68334D7E
:108F8000374CB5F9C6807E08B04528BFB046258865
:108F90001FFA88F80FFA88F229B28A420BDD3148AD
:108FA00031490068F7F78EFEF8F752F843191FFAB7
:108FB00083F8A4F800802D4E2D4D34682A68A61A37
:108FC0003046FFF7AFF80028D8BF404241F2931176
:108FD0008842CCBF00200120002859D03046F7F746
:108FE0001DFE2449F7F76EFE04F058F90546384691
:108FF000F7F710FE01462846F7F764FEF8F728F861
:109000001D4B1549188040F6B83200B2FAF7D0FE71
:10901000201848F6A044A04203DDA0F50C40A0387B
:1090200004E00028BCBF00F50C40A030134A1060DB
:1090300030E000BFAFF30080182D4454FB211940ED
:10904000600F0020E00F0020E80E0020B018002084
:109050000000F03F30F8FFFF48F4FFFFB80F00209A
:109060001E100020A40F00200000C842E40F0020C2
:10907000F80F0020D3023739200F0020780F00208E
:10908000B20F002020100020940F00202C1D002083
:10909000994F3C60984E002531682C46C1F50C5024
:1090A0002830F7F7BBFD9549F7F70CFE074604F0AB
:1090B00081F80F90384604F0F1F82F460E900FFA21
:1090C00088F0F7F7ABFD0EAB53F82710F7F7FAFD72
:1090D00006468B48DFF86CA2005FF7F79FFD01465C
:1090E0003046F7F7E5FCF7F7B3FF864924F80A00A6
:1090F0004FF47A7200B2FAF75BFE82B211B2DFF877
:10910000489224F80A2008460391F7F787FDD9F81A
:109110000010F7F7D7FDF7F79BFF83B27A481426C4
:1091200006FB0706DFF824B2039ADBF8001006936B
:1091300010464B463246FFF731F8DBF800C034F9F1
:109140000A1009906046D6F808A00891CDF808C02A
:10915000F7F76CF9CDE904015046F7F767F9DFF846
:10916000F0B1CDE90A019BF8C000F7F753FDF7F71E
:109170005DF95FA3D3E90023F7F7ACF902460B468C
:1091800000206249F7F7D0FADDE90423F6F7F0FF93
:1091900002460B46DDE90401F7F7C6FA089BCDE964
:1091A000040170680137181AF7F738FDDDF808C0B8
:1091B0006146F7F73BFE5146F7F77AFCF7F736F9C9
:1091C00002460B46DDE90401F7F784F902460B4637
:1091D000DDE90A01F6F7CCFFF7F716FC089A099BC0
:1091E00072603061B060069ED9F80810F618F7F783
:1091F00069FDF7F72DFF3018454E81B2A15308B233
:1092000040F6B8324349FAF7D3FD3F4A3053424B58
:10921000A8580234E8501435022F58467FF44FAF57
:1092200090F8C21031B1344A642413683B4A93FB6E
:10923000F4F111803A4BB0F8BE001C6884420ED99C
:10924000384939480A68036842F21074D01AFEF7A8
:1092500069FF0028B8BF4042A0427FF754AA3348B4
:10926000334A012104882D4B11701C80FFF74BBA43
:10927000FFF720F836E062686078531C411CCAB2E0
:1092800063600523B2FBF3F003FB10216170FDF76F
:1092900085FB284AA06028480023C3721370012070
:1092A0000BE0FDF77BFBA36840F6C411C01A8842AF
:1092B00018D9202000F0E8F80420FEF763FF11E041
:1092C0001E498A78522A7FF4AAAACB784D2B7FF4C4
:1092D000A6AA087943287FF4A2AA194A022111708C
:1092E000FFF79DBA11B0BDE8F08F00BFAFF300806B
:1092F000182D4454FB211940780F0020D302373930
:10930000B20F002018FCFFFFB80F00200000F03F54
:109310002C1D002048F4FFFFE80E0020F01D002067
:10932000F00F0020E40F0020F80F0020760F00203F
:109330001C0800208E1D0020871E00200210002027
:10934000B00F0020E00F0020240F0020A40F002009
:10935000B0180020AFF300803B4B2DE9F047B3F984
:109360000000F7F75BFC3949F7F7ACFC044603F063
:1093700095FF0646204603F01DFFDFF8E490054602
:1093800099F8C180324FB8F1000F29D0314CB7F9AC
:109390000200B4F802A00FFA8AF1401AFEF7C2FEEA
:1093A000C8F100014246FAF703FDB4F80080B7F9AE
:1093B00000700FFA88F300EB0A02F81A6280FEF7D9
:1093C000B1FE99F8C1205142FAF7F2FC404487B24D
:1093D0002780B4F90200F7F721FC804638B206E096
:1093E000B7F90200F7F71AFC8046B7F90000F7F763
:1093F00015FC294607464046F7F764FC314681468E
:109400003846F7F75FFC01464846F7F751FB12492B
:10941000F7F70CFDF7F71CFE104C31462080404654
:10942000F7F750FC294606463846F7F74BFC01464D
:109430003046F7F73FFB0849F7F7F8FCF7F708FE67
:109440006080BDE8F08700BFF21D002035FA8E3C39
:109450002C1D0020281D002000002041760800203F
:10946000B0180020034B196808420CBF00200120EF
:10947000704700BFF4100020024B1A6810431860B8
:10948000704700BFF4100020024B1A6822EA000067
:1094900018607047F4100020014B1868704700BF37
:1094A000F4100020024B5A780AB10020587070471F
:1094B000871E0020037A032B0FD8DFE803F0020297
:1094C000060A0649064A00F0D5BA0449044A00F0E3
:1094D0003BB90249024A00F0FDB97047AE1E0020B8
:1094E0003C11002010B5002304466189094A9952B5
:1094F0000233242BF9D10820FAF7AEFA20B1204626
:10950000BDE81040FFF7D6BF03480449BDE810404E
:1095100000F0D8B8C81E0020AE1E00203C1100206C
:109520002DE9F843074608208846FAF795FA70B106
:109530000024224A414613683846E2B2984720493F
:1095400021F814000134082CF3D1BDE8F8831D4A3A
:109550001D4D1378591CCCB204F00306147005EBB2
:1095600046090446064615484146036832463846D1
:10957000984729F824002A886988AB885018EA8817
:10958000C118881803B2991C042291FBF2F00C4A0E
:109590000E4BA15EE052CB1E984201DA811CA15213
:1095A000135FD91C884201DD023810530136F6B230
:1095B00002340835082ED6D1BDE8F8833C110020CE
:1095C000C81E0020F8100020FA10002040110020D2
:1095D00010B544780078002303FB03F11939614387
:1095E00001F6C4115943414340F6C41291FBF2F114
:1095F000034A22F813100133072BEDD110BD00BF31
:10960000EC1E00202DE9F04F85784FF00A0C0CFB82
:1096100005FCC778C5F164086E425FFA88F8C7F1A7
:109620006409B6B2002330B2002804DCB8BF2C466F
:1096300002DB012400E0444600FB00FB64430BFB1B
:1096400007FB9BFBF4F44C4444434FF00A0B94FBA0
:10965000FBF00CEB000420B2C1EB020A00FB0AF4A1
:109660004FF47A7094FBF0F404480C191C52023346
:109670005E44182BB6B2D6D1BDE8F08FB01E0020E4
:10968000F8B505460F46441E14F8011F49B1054EB2
:10969000304606F0BFFC0028F6D0861B631BBB5586
:1096A000F2E7F8BD2017010810B50446805CF9F711
:1096B00075FAA0F2EE2291B240F2DC53994288BFD3
:1096C000608910BD024B0B6008210170704700BF1C
:1096D000A9960008825C044B53F82200410801F56A
:1096E000777290B2704700BF5C11002038B5044615
:1096F000FDF73AF9104B40F6C4111A68821A8A42F3
:109700001A460E4B01D9002119701B7810600BB955
:109710000F2C10D10A4800210170084A4BB1094DA5
:10972000182B1D4405F8014C03D10123037011705F
:1097300038BD0133137038BD541100205011002082
:10974000581100207C110020408938B50D4B0D4682
:10975000A0F5777114464A001A605A609A60DA6080
:109760001A615A619A61DA6107490848084A052373
:10977000FCF794FF0749C8600CB107482060082235
:109780002A7038BD5C110020ED96000800440040AE
:10979000A08601000C1F0020D5960008274970B54F
:1097A0000878002849D0264B987DC0F3C0000028D7
:1097B00041D1244A10805D781C78234A05F00706C1
:1097C00044EA062414609C7804F03F06760146EAD9
:1097D000D5055560DE78B50045EA94151C7904F08E
:1097E000010645EA862595605D7905F00F06F601CC
:1097F00046EA5404D4609C7904F07F06360146EAB8
:1098000015151561DE79750045EAD4141D7A05F049
:10981000030644EA462454615C7A04F01F06B6014C
:1098200046EA950595619B7A0870DB0043EA54147B
:10983000D461012070BD0020087070BD5811002057
:109840007C110020EE0700205C110020825C034B9D
:1098500053F82200C0F3CF00704700BFB4110020BE
:1098600010B50446FDF780F8154B1A68811AB1F55A
:109870007A6F1A46134B01D90021197010601878BD
:1098800020B9A82C1AD1104B187006E0022802D17A
:109890000E4A147001E0142801D80D490C540B49EC
:1098A0000130C3B20878074A4100481D8342137053
:1098B00004D100230449137001220A7010BD00BFB7
:1098C000AC110020D4110020B0110020B1110020F3
:1098D0009511002038B5084801230D461446074964
:1098E0004FF4E132FCF7DAFE054BD8600CB10548C5
:1098F00020600821297038BD0044004061980008AC
:109900000C1F00204D980008134A10B513780BB9AE
:10991000002010BD1149002010704A78012AF7D1AB
:109920000F4B18800F480178082901D908220270CE
:1099300001780D4A0023D8B2023288420AD212F8C6
:10994000010C12F8024C40EA0424084840F8234075
:109950000133F0E7012010BDB01100209511002067
:10996000EE070020B111002098110020B411002052
:10997000124B012210B51A700446FCF7F5FF104A8D
:109980000146106811600B1A0E4841F288318B4273
:1099900003600D4B01D900221A7018780B49E4B20C
:1099A0000F280C5406D10A490A4B012000220870E6
:1099B0001A8010BD044A431C137010BDDD11002035
:1099C000D8110020E0110020DE110020FA1E002036
:1099D000DC110020EE0700201F4B2DE9F0431B781F
:1099E00023B31E4C1E4D277891F800C095F80080D7
:1099F00002231C4C03F10109E65C46FA07F606F067
:109A00000F05EEB266450BD20B2E09D8E65C14F8B2
:109A1000094006EA080604EB0626134C44F82560C4
:109A20000233102BE5D10C4B00241C7009789142B5
:109A300002D90E4B197811B94089BDE8F0830C4B5F
:109A4000825C1978084B53F8220001B1400800F5F8
:109A5000777188B2BDE8F083DC110020D5110020B9
:109A6000E4110020FA1E0020E8110020DD11002082
:109A7000D611002010B5037A14465BB1012B13D127
:109A8000104A03201070104A072010700F4803700E
:109A90000C2308E00B4A022010700B4A03201070C0
:109AA0000A48037007230B7009490A484FF4E13252
:109AB0000123FCF7F3FD0849C8600CB1074A226096
:109AC00010BD00BFD5110020E4110020D6110020E8
:109AD00071990008004400400C1F0020D99900082B
:109AE000014B1878704700BFDC11002008B54FF417
:109AF0000060F9F7B1FF08B9002008BD4020F9F770
:109B0000ABFF094B20B993F82D21501E0128F3D942
:109B100093F82C01012805D1034991F82D31002B30
:109B2000EAD008BD012008BD7C190020084B93F83D
:109B30002D215AB993F82E0110B9064A537801E045
:109B400005490B7D181C18BF012070470120704784
:109B50007C190020871E0020981E002010B5084B9D
:109B600093F82C211C460AB900F0ACF894F82C01AB
:109B7000012803D1BDE8104000F062BA10BD00BF5B
:109B80007C19002038B50E4B1878C0B1FFF7CEFF16
:109B90000C4904460A78824211D060B10A4D95F80A
:109BA0002C310BB900F098F895F82C01012804D15C
:109BB00000F03EFA01E0FFF7D1FF02490C7038BD1A
:109BC00019120020181200207C19002038B5044614
:109BD0004020F9F741FF0B4D08B985F82D01FFF73B
:109BE00085FF094B187095F82D01012801D1074810
:109BF00003E002280CBF06482068A060BDE838409A
:109C0000FFF7C0BF7C190020191200201C13002090
:109C1000641500200B4B10B5187888B1FFF786FF4C
:109C200070B1094991F82C210C460AB900F06CF882
:109C300094F82C31012B03D1BDE8104000F008BA94
:109C400010BD00BF191200207C19002038B5064C49
:109C500005465E21A068FCF7D1FBA0682946BDE857
:109C60003840FCF7CBBB00BF0C1F0020024B5E212D
:109C70009868FCF7C3BB00BF0C1F002010B50A4C4E
:109C80005E280146A06805D15D21FCF7B7FBA068FE
:109C90003E2105E05D2903D1FCF7B0FBA0683D2122
:109CA000BDE81040FCF7AABB0C1F002010B504460D
:109CB000C0B2FFF7E3FFC4F30720BDE81040FFF791
:109CC000DDBF0000034B93F82D0108B900F092BAF4
:109CD000704700BF7C190020044B93F82D0118B980
:109CE0004FF4165000F078BA704700BF7C1900207E
:109CF00008B5044B9868FCF791FBD0F1010038BF20
:109D0000002008BD0C1F00202DE9F041FFF7F0FFF7
:109D1000002800F04081FCF741FEA04B1A68811A30
:109D20007C2940F2388118609D480478651C0570D4
:109D3000002404F12406F0B2FFF788FF994B33F9B1
:109D40001400F6F76BFF984A05461088F6F766FF91
:109D500001462846F7F76AF89449F6F7B3FFF7F794
:109D600077F9013400B2FFF7A1FF032CE1D13020D5
:109D7000FFF76CFF8E49B1F90000FFF797FFFFF77F
:109D800075FF8748067816F0030629D1894D102003
:109D9000FFF75CFF2B68642493FBF4F210B2FFF72B
:109DA00085FF2120FFF752FF296891FBF4F004FBA7
:109DB000101484EAE473A3EBE47318B2FFF776FFA0
:109DC0001420FFF743FF7C4AB2F90000FFF76EFF53
:109DD0001C20FFF73BFF3046FFF768FFFFF746FF09
:109DE0006F490878430740F0B080744D0220FFF7B8
:109DF0002DFFB5F900300A2593FBF5F0FFF756FF6C
:109E00000220F9F729FE002847D06D4F6D4E3878B3
:109E1000347840F63401B4FBF0F26B4C4A432188AD
:109E20002A2391FBF0F800FB1810B2FBF3F24FEA83
:109E3000001399B241EA022C1FFA8CFEC2F30322EE
:109E40004EEA02080620FFF701FF0FFA88F0FFF73D
:109E50002DFF20883F78431C9AB292FBF7F107FB55
:109E60001120367820806E247443152394FBF3F47C
:109E70003A206427FFF7EAFEB4FBF7F63046FFF717
:109E800015FF3B20FFF7E2FE07FB164291B24C1D87
:109E900094FBF5F000B2FFF709FF2020FFF7E2FA8C
:109EA000002850D0494C1320FFF7D0FE2568484FBA
:109EB000002DB8BF6D4295FBF7F630B2FFF7F6FE06
:109EC0001B20FFF7C3FE23680A26002BB8BF5B42A6
:109ED00093FBF6F142F2107591FBF5F205FB1210BF
:109EE00000B2FFF7E3FE2320FFF7B0FE2368002B4C
:109EF000ACBF4E205320FFF7D9FE1220FFF7A6FE7D
:109F000061680029B8BF494291FBF7F210B2FFF730
:109F1000CDFE1A20FFF79AFE60680028B8BF4042C5
:109F200090FBF6F696FBF5F305FB136108B2FFF71D
:109F3000BDFE2220FFF78AFE6268002AACBF4520E2
:109F40005720FFF7B3FEFFF791FE15480378282B43
:109F500021D100240470FCF721FD4FF47A753C24D4
:109F6000B0FBF5F61720FFF771FEB6FBF4F5B5FB75
:109F7000F4F104FB1152100200B2FFF797FE182013
:109F8000FFF764FE04FB156318B2FFF78FFEBDE810
:109F9000F041FFF76BBEBDE8F08100BF201200204A
:109FA0001A120020201E00202600002000007A4403
:109FB000E00D0020A40D0020F21D0020241D002033
:109FC0001C000020AC1800201C120020701D002076
:109FD000A0860100154B2DE9F04180460F46986898
:109FE0000221FCF72FFA00242646781E84420F4DEA
:109FF0000DDA18F80410A8688E190134FCF7FEF980
:10A000004FF47A70B6B2FCF7CFFCE4B2EDE7F1B2F0
:10A01000A868FCF7F3F94FF47A70FCF7C5FCA86860
:10A020000121BDE8F041FCF70DBA00BF0C1F002074
:10A03000024B01219868FCF705BA00BF0C1F0020F5
:10A04000024B03219868FCF7FDB900BF0C1F0020EC
:10A05000F8B5544CA068FCF7E1F9002800F0A080A6
:10A06000A068FCF7E0F905460520FCF7A8FC8A2D5E
:10A0700021D08E2DEDD14C4C00212E22204605F012
:10A080000DFF4A4A7C2323701378E0207D21E07085
:10A0900084F82C1014204FF4FA71A377237548220A
:10A0A00078232076607661836570628484F824303A
:10A0B00020462E2171E02020FFF7D4F90028C8D0D7
:10A0C0003B4C00212C22204605F0E8FEA021E17047
:10A0D000384B39497C207D22207084F82B20187859
:10A0E000CA7A6570A076002A52D0344934480F6885
:10A0F0006625FE0F97FBF0FC6672324E5FFA8CFC11
:10A1000006FB0C7284F8295006256A4342F210734C
:10A11000B2FBF3FE03FB1E274968277391FBF0F0A7
:10A120003F0AC0B26773CF0F06FB00116943B1FB52
:10A13000F3F5642203FB1513E9B202FB0010010AD8
:10A14000E0732148217401885FFA8EFE63741B0A54
:10A1500002FB0CECA374B1FBF2F224235A4390B23D
:10A160001A4A010A1388E0712172180A18492075E9
:10A1700018480A8801884FEA1C2EE374130A84F8F1
:10A180000AC084F80BE0A7736275A375217702E01B
:10A19000202384F8293006482C21FFF71BFF58E7BD
:10A1A000F8BD00BF0C1F002050120020AC1800208A
:10A1B000241200208E1D0020871E0020701D00200C
:10A1C000A08601006079FEFF301D0020521D002096
:10A1D000261D00205C1D002008B50246032303480D
:10A1E0000021FCF75BFA024B186008BD0038014003
:10A1F0000C1F0020024B18680068FFF7EDBF00BF7E
:10A200008012002008B5044B1860FFF7F3FFBDE88B
:10A21000084001F0EFB800BF80120020034B18780F
:10A2200008B100F0F1BE01F05FB900BF8412002058
:10A23000232801D100F0E8BE044B19688A7A8242D3
:10A2400002D10120FCF77ABC704700BF80120020C9
:10A2500070B50646B6FBF2F40846154614B1204622
:10A26000FFF7F6FF05FB1464024B195D00F8011BB4
:10A2700070BD00BFA41801082DE9F0410278034623
:10A280000130202AFAD0092AF8D02D2A02D103461B
:10A29000414D04E02B2A08BF03464FF07E551E4671
:10A2A0000024334616F8010BA0F13007F9B2092952
:10A2B0000DD83A492046F6F705FD04463846F6F72C
:10A2C000ADFC01462046F6F7F5FB0446E9E72E28EB
:10A2D00017D1324F334616F8010B3038C2B2092A73
:10A2E0000FD8F6F79BFC3946F6F7A0FD014620464D
:10A2F000F6F7E0FB294904463846F6F7E3FC074643
:10A30000E8E71878652801D0452839D15E782D2EE8
:10A3100002D19F1C012605E02B2E01D05F1C00E01E
:10A320009F1C00267B1E002713F8012F303AD1B264
:10A33000092903D80A2000FB0727F5E7B7F59A7F1C
:10A3400028BF4FF49A77B8464FF07E51B8F1070F07
:10A3500007D908461249F6F7B5FCA8F108080146E6
:10A36000F4E707F0070737B108460C49F6F7AAFCEF
:10A37000013F0146F7E72EB12046F6F757FD04E00E
:10A380004FF07E512046F6F79DFC01462846F6F731
:10A3900099FCBDE8F08100BF000080BF00002041B3
:10A3A00020BCBE4C10B5441E14F8011F21B1034B54
:10A3B0001868FCF723F8F7E710BD00BF0C1F00205A
:10A3C0000148FFF7EFBF00BFC918010810B50748E3
:10A3D000FFF7E8FF0024064B06481A19E1585268B7
:10A3E0000C34F9F713FEC02CF5D110BDF718010895
:10A3F000C81701080D19010870B5FCF7CFFA244CF5
:10A40000244B4FF47A71B0FBF1F11A78224823788B
:10A41000F9F7FCFDFFF740F805462048204902689F
:10A420002048B2FBF1F1F9F7F1FD00241E4B53F87F
:10A43000241051B1012000FA04F0284202D01B4838
:10A44000F9F7E4FD0134E4B2F0E70220FFF70AF87F
:10A4500068B1174A174B1178174853F82110F9F7CC
:10A46000D5FD1648017C11B11548F9F7CFFD154C03
:10A470001548FFF797FF2488FBF764FF024613484F
:10A4800021464FF46673BDE87040F9F7BFBD00BFC9
:10A490001C000020AC1800201519010864010020E0
:10A4A00040420F0053190108DC2601087119010808
:10A4B000A80800208818010875190108A81D0020A7
:10A4C0007F1901085C080020341C01088319010869
:10A4D00038B50C680546204605F078FE0246286827
:10A4E0002146BDE8384005F0A1BE000008B5094886
:10A4F000FFF758FF01210020F9F74AFA0648FFF755
:10A5000051FF0A20FCF75BFA0020BDE80840FCF789
:10A5100015BB00BFB5190108BF1901087FB5044676
:10A5200005F054FE082825D100231F49E25C086885
:10A5300085186E7806F00301022908BF203AE2541C
:10A540000133082BF1D10025665D1848314605F02E
:10A5500061FD28B101356019314605F05BFD18B188
:10A560001348FFF71FFF1DE0082DEDD120461149CC
:10A57000FFF786F81048FFF715FF00230F4A04A9DC
:10A58000981890F808218818084A995C0133082B1C
:10A5900000F80C1CF2D100208DF80C0001A908482D
:10A5A000F9F734FD7FBD00BF8001002020170108AE
:10A5B000CE190108841A0020EE1901087C19002028
:10A5C0001019010808B5FDF7AFFF01300CBF0348B3
:10A5D0000348BDE80840FFF7E5BE00BF031A0108C5
:10A5E000291A01082DE9F041054605F0EFFD044662
:10A5F000F9F7D8FB064694B92A48FFF7D3FE2A4953
:10A6000051F8241049B1012202FA04F2324202D078
:10A610002648F9F7FBFC0134F1E7254821E02846FC
:10A620002449224605F002FE58B92348FFF7BAFE36
:10A63000224C54F8041F0029EFD01C48F9F7E6FC1F
:10A64000F7E72B782D2B04D10135013C4FF00108A1
:10A6500001E04FF000080026134850F8267027B993
:10A660001748BDE8F041FFF79DBE2846394622460F
:10A6700005F0DCFDA0B9012000FA06F0B8F1000FEA
:10A6800003D0F9F787FB0F4802E0F9F7EFF90E481E
:10A69000FFF788FE0D483946BDE8F041F9F7B6BC32
:10A6A0000136D9E7471A01082C170108711901086A
:10A6B000341C0108E62401085A1A01082817010869
:10A6C0006F1A0108891A0108931A01081019010864
:10A6D00010B504460848FFF765FE084A08480949CE
:10A6E0000023036013700B70FDF7ACF82046BDE843
:10A6F0001040FFF7FBBE00BF9C1A01088512002026
:10A70000B81200208412002008B50848FFF74AFE5E
:10A710000120F9F7B3F90648FFF744FE0A20FCF7D9
:10A720004EF90020BDE80840FCF708BAB41A010849
:10A73000C1190108F8B5074605F048FD044638B9C7
:10A740001A491B4B4A791B48511E53F8211028E027
:10A7500038461949224605F069FD60B91748FFF7E8
:10A7600021FE174C54F8041F19B11648F9F74EFC96
:10A77000F8E7154805E000250D4B53F8256026B98C
:10A780001248BDE8F840FFF70DBE38463146224674
:10A7900005F04CFD01350028EED1044831464571E5
:10A7A0000B48BDE8F840F9F731BC00BF7C19002028
:10A7B0006C170108CF1A0108E6240108E31A010802
:10A7C0006817010871190108341C0108F61A0108FC
:10A7D0000E1B010810B50446204605F0F7FC10F0EA
:10A7E000FF0F07D10B490C4891F89413BDE81040B6
:10A7F000F9F70CBC204605F007FA022808D8054BEB
:10A80000064C83F8940300200146F9F7C1F8E3E70A
:10A8100010BD00BF7C190020201B0108441E010848
:10A8200070B5044605F0D2FC08B9204830E0204657
:10A830001F4906F043F900242646254678B12CB17D
:10A84000012C06D105F0E0F9064602E005F0DCF93E
:10A85000054600201649013406F030F9EEE70B2DCD
:10A8600005D914480C21BDE87040F9F7CFBB012C85
:10A8700008DC114A114832F915202946BDE870401C
:10A88000F9F7C4BBA6F57A73B3F57A7F04D90C48FF
:10A89000BDE87040F9F7BABB0A4829463246F9F7D5
:10A8A000B5FB054820F8156070BD00BF361B0108D8
:10A8B0000E1E0108701B0108501E0020961B010887
:10A8C000AE1B0108D01B010838B5054605F07EFC1B
:10A8D000C0B268B904461249124801EB4402B2F80A
:10A8E000422021460134F9F791FB152CF3D138BDF4
:10A8F000284605F089F9142804460BDC2021284657
:10A9000005F088FB05F080F9054B03EB4404A4F83F
:10A91000420038BD04481521BDE83840F9F776BB40
:10A92000B0180020E91B0108F51B0108931E222B1B
:10A9300088BF0A22031E10B50C4603DA2D2001F849
:10A94000010B5842FFF784FC00210170204610BD26
:10A9500030B587B005460C4603A800210C2205F04F
:10A960009DFA28460021F6F769FB20B128462949BF
:10A97000F6F7A0F803E028462649F6F799F82649A5
:10A98000F6F7A0F9F6F764FB054685EAE570A0EB5B
:10A99000E5700A226946FFF7C9FF002D01DB20237D
:10A9A00000E02D2368468DF80C3005F00FFC0128DF
:10A9B00007D130228DF80D208DF80E208DF80F2054
:10A9C0000CE0022805D130218DF80D108DF80E1005
:10A9D00004E0032802D130208DF80D00694603A859
:10A9E00005F0F2FA03A805F0F1FBC51EEDB22A4608
:10A9F00003A9204605F088FC00236355204607493B
:10AA000005F0E2FA03A92046491905F0DDFA2046CF
:10AA100007B030BD6F12033A00007A44CC19010828
:10AA200037B5037904460D46052B34D8DFE803F02B
:10AA300003060A0D1114816809782DE0806890F9E9
:10AA4000001029E08368198826E08268B2F90010B6
:10AA500022E0816809681FE0806869460068FFF7A6
:10AA600077FF01461148F9F7D1FAF5B1E068F6F73A
:10AA7000D5F86946FFF76CFF01460D48F9F7C6FAAD
:10AA80002069F6F7CBF86946FFF762FF01460848F0
:10AA9000F9F7BCFA09E000210648F9F7B7FA25B141
:10AAA0000548E1682269F9F7B1FA3EBD7C19010851
:10AAB0007B1901081F1C01081B1C01082DE9F04728
:10AAC000064605F083FB054620B1012819D13378ED
:10AAD0002A2B16D14748FFF765FC0024142666434D
:10AAE000454F4648F159F9F791FAB8192946FFF749
:10AAF00097FF01344248FFF755FC6E2CEED1BDE8BC
:10AB0000F08730463D2105F085FA002857D0441CD7
:10AB1000204605F079F882462046FFF7ADFB002776
:10AB2000054614247C43DFF8D09054F80980404651
:10AB300005F04CFB41460246304605F077FB002805
:10AB400035D14C44E068F6F769F801462846F6F737
:10AB50006BFA002829D02069F6F760F801462846EC
:10AB6000F6F758FA002820D020792279052818BF56
:10AB70005546052A0FD8DFE802F003030606090C44
:10AB8000A1680D7007E0A268158004E0A068056068
:10AB900001E0A1680D6041461A48F9F737FA2046EE
:10ABA0000021BDE8F047FFF73BBF174803E001373E
:10ABB0006E2FB6D11548BDE8F047FFF7F3BB04464A
:10ABC000142565430C4F314655F80780404605F083
:10ABD000FFFD50B109484146F9F718FA78190021EC
:10ABE000FFF71EFF0648F9F711FA01346E2CE7D182
:10ABF000BDE8F087221C0108FC260108011D0108A0
:10AC0000341C0108371C0108421C0108671C01089C
:10AC10002DE9F043584885B0584CF9F7F7F95848F2
:10AC2000FFF752FE6279574B511E574853F82110D7
:10AC3000F9F7ECF920690021F6F7D8F9002858D186
:10AC40000025266900213046F6F7D0F900284CD1BE
:10AC500001354E482946D4F81490D4F81880E76995
:10AC6000F9F7D4F930460021F6F7CAF910B148488F
:10AC7000F9F7CCF969463046FFF76AFE01464548C8
:10AC8000F9F7C4F948460021F6F7BAF910B140487F
:10AC9000F9F7BCF969464846FFF75AFE01463D48B8
:10ACA000F9F7B4F940460021F6F7AAF910B138488F
:10ACB000F9F7ACF969464046FFF74AFE01463548C8
:10ACC000F9F7A4F938460021F6F79AF910B130489F
:10ACD000F9F79CF969463846FFF73AFE01462E48D7
:10ACE000F9F794F910340C2DABD12C48691CF9F705
:10ACF0008DF9F9F757F82A4C064654F8041F19B194
:10AD00002848F9F783F9F8E70D46274850F8251049
:10AD100049B1012202FA05F2324202D02348F9F782
:10AD200075F90135F1E7154B214ACE1896F808411F
:10AD30008B5C04A801310519082905F8103CF2D1F3
:10AD400000241C4869468DF80840F9F75FF914257E
:10AD50006543194E1948A959F9F758F90021701996
:10AD6000FFF75EFE01341648FFF71CFB6E2CEED198
:10AD700005B0BDE8F08300BF841C01087C190020E9
:10AD8000441E01086C170108B41C0108BF1C01080F
:10AD90000E1E01087C19010810190108C71C0108C2
:10ADA00028170108D91C01082C170108E71C010805
:10ADB00020170108F41C0108FC260108FD1C0108ED
:10ADC000341C01082DE9F04389B0044605F0FEF972
:10ADD000C6B2002E6AD17948FFF7E4FA784C2069B0
:10ADE0000021F6F703F938BB013676483146F9F70A
:10ADF0000DF9206904A9FFF7ABFD01467248F9F788
:10AE000005F9606904A9FFF7A3FD01466E48F9F74B
:10AE1000FDF8A06904A9FFF79BFD01466A48F9F710
:10AE2000F5F8E06904A9FFF793FD01466748F9F7D3
:10AE3000EDF810340C2ED2D10025654C2F46A846D3
:10AE40004FF000091034B14514DA404654F8101C94
:10AE5000F5F730FE54F80C1C80462846F5F72AFE1C
:10AE600054F8081C05463846F5F724FE09F1010997
:10AE70000746E7E75748CDF8048002950397FFF7A8
:10AE800091FA002401A82358534923F00040F6F713
:10AE9000D5F85249524A0434002814BF10460846D7
:10AEA000FFF780FA0C2CEDD14E4870E020464E4959
:10AEB000052205F0BBF938B9414B0022C11810300A
:10AEC000C0280A61F8D176E020464849042205F0FE
:10AED000ADF90546204605BB202105F09BF800286A
:10AEE00069D0461C304605F071F92C4607464048AB
:10AEF00050F824500DB93F4849E030462946FAB28F
:10AF000005F094F938B92046FCF73AFD3A4829464D
:10AF1000F9F77CF847E00134E9E704F075FE461ED6
:10AF20000B2E074643DC2046202105F073F805462A
:10AF300040B1451C2846FFF79FF9214B3F01D851EE
:10AF4000012400E004462846202105F063F8054668
:10AF500040B1451C2846FFF78FF91949013401EB30
:10AF6000061250612846202105F054F8054640B1EC
:10AF7000451C2846FFF780F9114B013403EB0611FD
:10AF800088612846202105F045F818B91B48FFF7CD
:10AF900009FA10E00130FFF76FF9094A032C02EBC0
:10AFA0000616F061F2D11648FFF70CFF03E01548D2
:10AFB0000C21F9F72BF809B0BDE8F0830F1D01084B
:10AFC0007C1900203A1D0108401D010810190108D4
:10AFD00090190020441D01080AD7233C0B1D0108CD
:10AFE000071D0108341C0108531D0108591D0108E3
:10AFF0006C170108F61A01085E1D0108711D010891
:10B00000441E0108AB1D0108F0B5694B87B01A78E2
:10B010003AB9012018706748FFF7C4F96648FFF78E
:10B02000C1F9664C2068FBF7F9F9002800F0BD80F3
:10B030002068FBF7F8F909280146614A01D03F284A
:10B0400051D1002517685F4C2E462FB15E4821680C
:10B050003A4605F0EBF810B9254606B926465B4995
:10B060000C348C42F1D3C6B13468D5F800E03B46CD
:10B07000E05C1EF8031081420DD1534A41B92D2BDB
:10B0800006D820244E48D45401330360D15404E040
:10B09000D0540133ECE74A490B60494A14681CB1AB
:10B0A000AE4201D13C4612E04948FFF77BF9AE427F
:10B0B00009D856F80C0BFFF775F9404B09211868B1
:10B0C000FBF79CF9F3E73C48FFF76CF900243C4B95
:10B0D00018688442A5D239493B4A0868115DFBF7DC
:10B0E0008DF90134F3E713682BB9042838D13648B9
:10B0F000FFF7EEFA59E00C2801D136488CE70A290F
:10B1000001D00D2948D12E4D3348FFF74BF92E4C75
:10B110002A6832490023A3540493009103A82949C3
:10B1200010220C23039404F073FD054638B1006827
:10B1300005F04CF80130AA682018904702E0284832
:10B14000FFF730F9002130221F4804F0A7FE18480D
:10B150001B4B027800211960002A7FF45FAF24E0C6
:10B160000C28CAD07F2903D15BE72F2B3FF659AFBC
:10B170001F297FF656AF7E293FF653AF13B920291A
:10B180003FF44FAF104C0E480C4AE15401330360BA
:10B190001068FBF733F944E77F29E6D10A485C1EC3
:10B1A0000021015514600F4839E707B0F0BD00BF1A
:10B1B00084120020D31D01080B1E01080C1F002063
:10B1C000B8120020C817010885120020881801084D
:10B1D000101E0108151E0108341C0108D1A4000826
:10B1E000201E0108411E0108F8B5174E174C184DD6
:10B1F0000746C1B230682170FBF700F922782B783E
:10B20000C7F3072182EA0300287030682170FBF73A
:10B21000F5F821782A78306881EA0203C7F30741FC
:10B220002B702170FBF7EAF82078297880EA010278
:10B23000390E306821702A70FBF7E0F82B782078FF
:10B2400080EA03012970F8BD0C1F0020BD12002008
:10B25000BC120020F8B50D4E0D4D0E4CC1B2074684
:10B2600030682970FBF7CAF82A782378391282EA05
:10B270000300207029703068C9B2FBF7BFF823784B
:10B280002A7882EA03002070F8BD00BF0C1F00205E
:10B29000BF120020BC120020054B10B50446214609
:10B2A0001868FBF7ABF8034802785440047010BDEF
:10B2B0000C1F0020BC120020034B04491A78885C44
:10B2C00001321A70704700BFD9120020DA12002034
:10B2D00010B5FFF7F1FF0446FFF7EEFF04EB002087
:10B2E00080B210BD10B5FFF7F3FF0446FFF7F0FF83
:10B2F00004EB004010BD000038B5044624200D4684
:10B30000FFF7CAFF4D20FFF7C7FF002C0CBF3E2000
:10B310002120FFF7C1FF064B002228461A70FFF7D5
:10B32000BBFF04480078BDE83840FFF7B5BF00BF59
:10B33000BC120020C312002001460020FFF7DCBF32
:10B3400001460120FFF7D8BF014B1878FFF7A4BFD3
:10B35000BC12002070B5054608460E46FFF7ECFF0C
:10B360002C467219D0B2E3B2984204D014F8010B03
:10B37000FFF792FFF5E770BD10B5441E14F8010FFA
:10B3800010B1FFF789FFF9E710BD00002DE9F84380
:10B39000002701240025144B187885421CDA134934
:10B3A000134B15F801800C2202FB0830406804F0B2
:10B3B0000DFF81460CB13F180CE026464E4509DAD8
:10B3C0000B4A0C2101FB08235868805DFFF764FFDE
:10B3D0000136F3E70135DEE724B1F8B2FFF7ACFF41
:10B3E0000024D7E7BDE8F883BE120020C412002075
:10B3F0004800002070B5394DFF211522284604F081
:10B400004DFD002302202B70FEF72CF8012418B10B
:10B4100002206C70A87003240420FEF723F868B1A2
:10B420002E4E03214FF400503155651CF8F714FBE4
:10B4300018B104227255023400E02C460220FEF7B7
:10B4400011F848B1254B05201E190621072518556E
:10B450007170B570033404E00820FEF703F800288B
:10B46000F0D12020F8F7F8FA18B11C4B08221A5531
:10B4700001344FF48070F8F7EFFA30B117480A261C
:10B4800001190B2506554D700234154A134B50799E
:10B49000082801D00E2802D10C261E5501340D219A
:10B4A00004201955651CF8F7D7FA18B10B4811227A
:10B4B0004255A51C0A49132391F82E21074E6C1CF6
:10B4C000101C18BF01207355F8F7C6FA10B11420EC
:10B4D0003055AC1C034B1C7070BD00BFC412002063
:10B4E0007C190020BE120020F8B5B54C2068FAF790
:10B4F00095FF002800F041852068FAF794FFB14AD3
:10B500000346117871B9B0F124014B4253EB0104A9
:10B510001470002CE9D1AC4A51780029E5D1FEF72E
:10B5200087FEE2E7012904D14D280CBF0223002346
:10B5300021E0022904D13C280CBF032300231AE098
:10B5400003290FD140284FF0000401D91470CCE733
:10B550009E489F4903709F480C7004709E4C237056
:10B56000042308E0042908D19B4C9C4821780370EF
:10B570004B40237005231370B7E70529B5D19448D4
:10B58000924C017822788A42934A07D914785C4019
:10B590001470934A535401310170A6E71078984211
:10B5A00040F0E6848D4B19787B2900F0338300F25C
:10B5B000C5806E2900F07D8360D8682900F046833D
:10B5C00025D8652900F0128219D8642940F0CB846F
:10B5D0000720844CFFF7B0FEE620FFF75DFE6079A0
:10B5E000FFF75AFE0020FFF757FE94F819017E4B33
:10B5F0007E4A00280CBF1046184600F067BC66293A
:10B6000000F07282672940F0AE8479481FE36B290D
:10B6100000F02D8323D8692900F01D836A2940F0AA
:10B62000A2841020FFF788FE6748724CC07AFFF7AB
:10B6300033FE71490878FFF72FFE2068FFF7D4FD2D
:10B640006068FFF7D1FD6D4AB2F90000FFF702FE16
:10B650006B4BB3F90000FFF7FDFD6A4A26E36C2946
:10B6600000F017836D2940F07E840620FFF764FE0A
:10B6700065490868FFF7B8FD644A17E3732900F0CD
:10B6800085833CD8702900F04383C0F0238371295F
:10B6900000F05183722940F06684524C1620FFF767
:10B6A0004BFE0020FFF7D6FDB4F9D000FFF7D2FD26
:10B6B000574DB4F9D200FFF7CDFDB4F9D400FFF730
:10B6C000C9FDB5F9B600FFF7C5FD0020FFF7C2FDC3
:10B6D0000020FFF789FDB5F928000A2390FBF3F05D
:10B6E000FFF7B8FD94F80401FFF7D6FD94F80601C2
:10B6F000FFF7D2FD94F80501FFF7CEFD75E376293B
:10B7000000F04F830DD8742900F02D83752940F087
:10B710002A842F20FFF710FE3E48FFF72DFE00F091
:10B7200025BC772900F02283782940F01C84384C0E
:10B730003820FFF701FE04F1400539E2D02900F07E
:10B74000898300F2CA80CA2900F00F816CD8A4292D
:10B7500000F0E88310D8A02940F005840C20FFF702
:10B76000EBFD2D492D4C0868FFF73EFD2C4A106873
:10B77000FFF73AFD2068A9E3C82900F0ED80C92948
:10B7800040F0F183FFF798FD0F4B1A4CD872FFF78A
:10B7900093FD19490870FFF7A5FD2060FFF7A2FD92
:10B7A0006060FFF795FD154A1080FFF791FD144B7F
:10B7B00018801C48017841F002040470E4E000BFE6
:10B7C0000C1F0020C1120020871E0020C012002084
:10B7D000C2120020D9120020BC120020C312002087
:10B7E000DA1200207C1900201C0000801400008068
:10B7F00034000020701D00208E1D0020261D00201A
:10B80000301D00207C080020181E0020E00D0020C4
:10B81000B0180020942F0108E8F7FF1FF0F7FF1F72
:10B82000ECF7FF1F74080020CD2900F01C8322D8FC
:10B83000CB2900F0AB80CC2940F09583FFF73CFD8D
:10B84000C84CE077FFF738FD84F82000FFF734FD9F
:10B8500084F82300FFF730FD84F82400FFF72CFD67
:10B8600084F82500FFF728FD84F82100FFF724FD68
:10B8700084F8220088E0CE2900F0FF82CF2940F032
:10B880007283FFF725FDFFF723FDB74CB54DA4F8F4
:10B89000D000FFF71DFDA4F8D200FFF719FDA4F8B2
:10B8A000D400FFF715FDA5F8B600FFF711FDFFF76F
:10B8B00019FDFFF70DFD0A2358432885FFF7FCFC0F
:10B8C00084F80401FFF7F8FC84F80601FFF7F4FCA4
:10B8D00084F80501FFF7F0FC56E0D52900F0A881B7
:10B8E0000FD8D2296BD0C0F08482D32979D0D42943
:10B8F00040F039839B4C0020FFF71EFD04F140050A
:10B900006AE1F02900F0D5820CD8D6294ED0EF2973
:10B9100040F02983FFF7DCFC924CA085FFF7D8FCB0
:10B92000608531E0FA2900F0B082FE2940F01B83E7
:10B930000820FFF701FD8D4C8D488E4B0168206873
:10B94000B1FBF3F2B0FBF3F34FF47A7101FB023475
:10B95000894AD4800024A4E20024FFF7B9FC874A76
:10B9600010530234102CF8D10EE0854C04F10A0576
:10B97000FFF7A2FC01346070FFF79EFCE072FFF756
:10B980009BFCAC426075F3D1002087E200247D4827
:10B9900001788C42F8D27C4D655DFFF799FC714AC5
:10B9A000013402EB4505A5F84200F0E70024FFF75B
:10B9B0008FFC764A10530234102CF8D1E4E7744C13
:10B9C0006478002CE0D1FFF777FC6749022881F802
:10B9D000940388BF81F8944300200146F7F7D8FF0D
:10B9E000D2E7FFF775FC6B490880CDE76A4D0B2065
:10B9F000FFF7A2FCB5F90000FFF72CFCFAF7A2FC58
:10BA000000B2FFF727FC0220FDF72CFD05460420BD
:10BA1000FDF728FD04460820FDF724FD820042EAD8
:10BA20004401294320208CB2FDF71CFD44EAC000EC
:10BA300084B21020FDF716FD44EA001318B2FFF798
:10BA400009FC534A1079D17884005378907944EAFC
:10BA50004101194341EAC0045179537A44EA411043
:10BA600040EA83144D48C17944EAC113047A417A0B
:10BA700043EA042343EA4124D379117A44EA832434
:10BA8000927A44EAC123417B43EA0234827B44EA4E
:10BA90004133017C43EA8234027944EA0143417C28
:10BAA00043EA0214827C44EA4143C17C43EA824473
:10BAB000007D44EAC142334B42EA00540020197829
:10BAC00003468B420AD2304D01225D5D02FA05F534
:10BAD00025421CBF9A4010430133F2E7224CFFF786
:10BAE00083FB94F8940381E11220FFF725FC2C4995
:10BAF0000C88B4F5806F2B4CB4F9000008D8FFF720
:10BB0000A9FBB4F90200FFF7A5FBB4F904000EE0AD
:10BB1000082590FBF5F0FFF79DFBB4F9020090FBC0
:10BB2000F5F0FFF797FBB4F9043093FBF5F01E4CEA
:10BB3000FFF790FBB4F90000FFF78CFBB4F90200AB
:10BB4000FFF788FBB4F90400184CFFF783FBB4F946
:10BB50000000FFF77FFBB4F90200FFF77BFBB4F9AD
:10BB60000400B0E1B01800207C190020640100201E
:10BB70006001002040420F003C1D0020C81E002034
:10BB8000AF180020BE120020C4120020501E00205A
:10BB9000871E0020F01D00205C080020981E002059
:10BBA00026000020201E0020980D0020D41D00201B
:10BBB000B4F97400FFF74EFBB4F97600FFF74AFBC7
:10BBC000B4F97800FFF746FB94F87A000834FFF7E1
:10BBD00063FBAC42ECD1C9E1FFF77AFBA4F8740037
:10BBE000FFF776FBA4F87600FFF772FBA0F57A72F8
:10BBF000072893B298BF84F87B00B3F57A7F98BF8B
:10BC0000A4F87800FFF758FB84F87A000834AC42B7
:10BC1000E2D1ABE10820FFF78FFB0024AD496218A9
:10BC200092F87B000834FFF737FB402CF6D19DE1FA
:10BC30000020FFF781FB0024FFF73EFBA5496218B7
:10BC40000834402C82F87B00F6D18FE1A248102105
:10BC5000FFF780FB8AE11020FFF76EFB00249F486E
:10BC6000005F0234FFF7F6FA102CF8D17EE10520D0
:10BC7000FFF762FB9A4BB3F90000FFF7EBFA994824
:10BC8000B0F90000FFF7E6FA97490A7802F00100E0
:10BC9000ACE0964C0620FFF74FFBB4F90000FFF72D
:10BCA000D9FAB4F90200FFF7D5FA914AB2F90000C7
:10BCB00009E10720FFF740FB8E480078FFF7ECFA18
:10BCC0000020FFF7C7FA8C4BB3F90000FFF7C2FA68
:10BCD0000020F8E07F4C0720FFF72EFBE07FFFF706
:10BCE000DBFA94F82000FFF7D7FA94F82300FFF767
:10BCF000D3FA94F82400FFF7CFFA94F82500FFF761
:10BD0000CBFA94F82100FFF7C7FA94F822006DE00F
:10BD10001E20FFF711FB794C04F10A05013460780D
:10BD2000FFF7BAFAE07AFFF7B7FA607DFFF7B4FAE7
:10BD3000AC42F3D11AE172490A78540004F0FE00D3
:10BD4000FFF7FAFA00246E4803789C4280F00E81D7
:10BD50006C496048625C013400EB4203B3F9420075
:10BD6000FFF778FAEFE7FFF711FBFFE064490024E3
:10BD70000878FFF7E1FA624A1078844280F0F68092
:10BD8000604B185DFFF788FA0134F4E70820FFF7ED
:10BD9000D3FA0124E0B20134FFF77EFA092CF9D17D
:10BDA000E4E0FFF789FA06461220FFF7C5FA0EB95C
:10BDB000554902E0102E03D154490D684C6801E04A
:10BDC000002425463046FFF767FA2846FFF70CFAAD
:10BDD0002046FFF709FA4E4A1068FFF705FA0020DF
:10BDE000FFF738FA0020FFF735FA0020FFF754FA82
:10BDF000BCE0FFF761FA0546FFF774FA0746FFF764
:10BE000071FA0646FFF76EFA0446FFF761FAFFF78C
:10BE10005FFAFFF751FA65B93B483E4901220760D6
:10BE20004660CD710A73002C3FF4AEAD384B1C60F8
:10BE3000AAE5102D7FF4A8AD3448076046600CB128
:10BE4000334A1460344B314802211970011DFCF74C
:10BE5000A3FB99E52F484378002B7FF495AD012093
:10BE6000F7F70CFE90E52B4C6378002B7FF48CAD3C
:10BE70002A494FF4C870088086E526484178002991
:10BE80007FF482AD012282737EE5224B5C78002C28
:10BE900069D120460121F7F77BFD2046FFF74CFAD8
:10BEA00064E01F48005F0234FFF7D4F9082CF8D192
:10BEB0005CE0084C0420FFF73FFAB4F92C00FFF7D0
:10BEC000C9F9B4F92A00FFF7C5F94FE0FFF78CF97B
:10BED0004CE000BFB0180020381E0020C81E002013
:10BEE000521D00205C1D002074080020940D0020CD
:10BEF000F21D0020AC1800208C1D0020AF1800207F
:10BF0000BE120020C4120020541D0020341D002049
:10BF10001C1E0020871E00201C0800209008002006
:10BF20003C1D0020154C23789800411CC8B2FFF737
:10BF300003FA2078FFF7B0F90024104A13789C42E6
:10BF400014D20F48005DFFF7A7F90E49085DFFF70F
:10BF5000A3F90D4A105DFFF79FF90C4B185DFFF731
:10BF60009BF90134E9E70020FFF7EAF9FFF7ECF964
:10BF7000074B00201870FFF7B8BAF8BD8F1D0020DE
:10BF8000141D00205E1D0020781D0020981D00203B
:10BF9000C11200202DE9F0410746884616460024CC
:10BFA000B44219D00025BD4210D00C4B0135DA68DF
:10BFB000EDB282F00800D8600120FAF7AFFC4046ED
:10BFC000FAF7FDFC0020FAF7A9FCECE73C2001346D
:10BFD000FAF7F5FCE4B2E3E7BDE8F081000C0140BC
:10BFE0000F4B1A6842F00100186059680D4A0A4068
:10BFF0005A60186820F0847121F480321A60186841
:10C0000020F4802119605A684FF41F0122F4FE00C9
:10C0100058609960044B4FF000629A60704700BF0F
:10C02000001002400000FFF800ED00E0164A174B38
:10C03000516801F00C00042803D0082805D01448EA
:10C0400001E014490868186011E051685068C1F3B4
:10C0500083410231C00301D40F4A06E052680D4803
:10C0600012F4003F026818BF520851431960064B92
:10C070000A485A68054BC2F30311415C1A6822FA58
:10C0800001F21A60704700BF0010024064010020F6
:10C0900000127A006001002000093D0050010020DC
:10C0A0001FB500234F494FF4E01000930193029312
:10C0B00003900A6842F480330B60886940F01002F4
:10C0C0008A61484B196801F400300190009A511CB4
:10C0D000009101981A4618B9009BB3F5A06FF0D1F2
:10C0E0001168404811F4003201D0022216E00368C2
:10C0F00043F00101016000923A48026802F0020335
:10C10000019300994A1C0092019B1BB90099B1F55B
:10C11000A06FF1D1006883073CD50122324B029217
:10C12000196841F0100018601A6822F003011960C4
:10C13000186840F002021A60A3F5805359685960EC
:10C14000586858605A6842F48061284A59601068FB
:10C1500020F070411160264826490860586820F494
:10C160007C105860106840F000401060906820F427
:10C1700000409060043A9268100449BF1E4A4FF490
:10C18000E0120A604FF480120392029915480129C7
:10C1900001D10AE0FEE702290BD14268039B42EA83
:10C1A000030141F48032426003E0596841F46012B7
:10C1B0005A60036843F0807101600A480268920186
:10C1C000FBD5436823F003014160426842F002035B
:10C1D0004360416801F00C02082AFAD1FFF726FFFC
:10C1E00005B000BD001002400020024004100140D4
:10C1F00000127A0060010020001BB700837910B59F
:10C20000002B29D01A4B01681C68CA4314401C60DB
:10C210005C6822405A60027902F1804404F582325F
:10C2200014682143116002689C68D1430C409C60F3
:10C23000DC68407921401028D96006D19868104305
:10C240009860D9680A43DA6010BD00F1804303F5B5
:10C25000823319680A4308E00179006801F18042DD
:10C2600002F582331A6822EA00021A6010BD00BF8C
:10C2700000040140064B1A68596910EA010304D012
:10C2800010420CBF0020012070471846704700BFC5
:10C2900000040140014B5861704700BF0004014099
:10C2A00008B5154B98420BD101214FF4805000F096
:10C2B000C1FD4FF480500021BDE8084000F0BABD38
:10C2C0000E49884207D14FF48040012100F0BEFDA5
:10C2D0004FF4804009E00A4A90420BD14FF40040ED
:10C2E000012100F0B3FD4FF400400021BDE80840FB
:10C2F00000F0ACBD08BD00BF003001400038004078
:10C30000003C00400B8810B54C88028823438C8881
:10C3100002F441522343CC8823430C8923434C89A4
:10C3200023438C892343CC89098A23431A4393B23C
:10C330000380828B22F400631A04130C838301822E
:10C3400010BD038819B199B241F0400303E023F016
:10C3500040010A04130C0380704781817047808973
:10C3600080B27047038919420CBF0020012070473A
:10C37000426810B522F470230A6823F4807444EAFA
:10C3800002030C7943EA04224260CB688A6884681D
:10C390001A43084B234013434A7943EA420383601C
:10C3A000097CC26A4B1E22F47002D9B242EA0152E1
:10C3B000C26210BDFDF7F1FF836811B143F00101C6
:10C3C00001E023F0010181607047836811B143F4FB
:10C3D000807101E023F4807181607047836843F0CD
:10C3E0000801816070478068C0F3C00070478368AF
:10C3F00043F00401816070478068C0F3800070479B
:10C40000836811B143F4A00101E023F4A00181602D
:10C410007047092970B54FF003040CD94C43072528
:10C420001E3C05FA04F503FA04F3C66826EA05057E
:10C430002B43C3600BE04C43072505FA04F503FAD0
:10C4400004F3066926EA050545EA03040461062AA1
:10C450004FF005030DD8013A53431F2202FA03F2AD
:10C4600001FA03F1446B24EA020242EA0103436346
:10C4700070BD0C2A0DD853431F22233B02FA03F24E
:10C4800001FA03F1046B24EA020242EA01030363A6
:10C4900070BD53431F22413B02FA03F201FA03F13C
:10C4A000C46A24EA02021143C16270BD40F0BF6059
:10C4B000024B40F40031D960704700BF00ED00E04E
:10C4C000C37810B503B3164CE168CB43C3F3022421
:10C4D0004178C4F1040201FA02F10F2222FA04F2B7
:10C4E0008478037822400A43110103F16043CAB201
:10C4F00003F5614181F800230078012200F01F0359
:10C50000410902FA03F007E00078012200F01F035E
:10C51000410902FA03F02031024B43F8210010BD1B
:10C5200000ED00E000E100E030B5048C24F00105EE
:10C530002C04250C0584048BA5B225F0F3052A43B1
:10C5400042EA0313114A048C9042A4B29DB215D062
:10C5500002F50063984211D0B0F1804F0ED0A3F5E0
:10C56000983290420AD002F58063984206D003F5D3
:10C570008062904218BF24F00A0401D124F0020422
:10C5800044F0010421430583018430BD002C0140A7
:10C5900030B5048C24F010052C04250C0584048B84
:10C5A000058C24F440742405240D44EA022242EA56
:10C5B0000333144AADB290429BB212D002F500622E
:10C5C00090420ED0B0F1804F0BD0A2F5983290423D
:10C5D00007D002F58062904203D002F5806290425B
:10C5E00007D125F0200242F0100545EA011189B279
:10C5F00004E025F0A00545F01005294303830184DC
:10C6000030BD00BF002C0140224A038890429BB2FB
:10C6100012D002F5006290420ED0B0F1804F0BD0E4
:10C62000A2F59832904207D002F58062904203D082
:10C6300002F58062904203D14A8823F070031343CD
:10C64000154A904208D002F58062904204D023F44B
:10C650004073CA889BB2134303808B880A88838502
:10C660000C4B028598420FD003F5006290420BD02C
:10C6700002F54063984207D003F58062904203D0F0
:10C6800002F58063984201D1097A018601228282F3
:10C69000704700BF002C014000100040038C70B5B3
:10C6A00023F001021404250C0584068C8388028B78
:10C6B0009CB222F073052B040D881A0C26F002069A
:10C6C00033042A434E880D891B0C3543ADB22B43EE
:10C6D000134DA8420FD005F50065A8420BD005F513
:10C6E0004065A84207D005F58065A84203D005F54E
:10C6F0008065A8420ED123F008064B898D881E4321
:10C7000026F004032B43CE898D8924F440743543ED
:10C71000ADB22C43C988848002838186038470BDB6
:10C72000002C0140038C30B523F010021404250CBA
:10C730000584038C8288048B23F0200324F4E645CF
:10C740002C040D88240C44EA05241D042B0C0D89AF
:10C7500092B243EA05134D88A4B243EA0513124D81
:10C760009BB2A84203D005F50065A84215D14D89BA
:10C7700023F080039BB243EA05134FF6BF751D40BB
:10C780008B8822F4406245EA0315ABB28D8942EAF8
:10C790008502CD8942EA850292B2C98882800483EB
:10C7A0000187038430BD00BF002C0140038C30B5ED
:10C7B00023F480721404250C0584038C8288848BF6
:10C7C00023F4007324F073052C040D88240C2C43EF
:10C7D0001D042B0C0D8992B243EA05234D8843EAD0
:10C7E0000523124D9BB2A84203D005F50065A8426F
:10C7F00015D14D8923F400639BB243EA05234FF61C
:10C80000FF351D408B8822F4405245EA0325ABB228
:10C810008D8942EA0512CD8942EA051292B2C98891
:10C82000828084838187038430BD00BF002C014057
:10C83000038C30B523F480521404250C0584038C3A
:10C840008288858B94B225F4E64215042A0C0D8863
:10C8500023F4005342EA05221D042B0C0D8992B2E9
:10C8600043EA05334D8843EA05330A4D9BB2A8429B
:10C8700003D005F50065A84205D18D8924F48044D4
:10C8800044EA8514A4B2C98884808283A0F8401049
:10C89000038430BD002C014000214FF6FF738380DC
:10C8A0000180C18041800172704700230380438072
:10C8B0008380C380038143818381C38170470023C8
:10C8C0000122038043808280C380038170470388F4
:10C8D00019B199B241F0010303E023F001010A0408
:10C8E000130C03807047B0F8443029B16FEA43431A
:10C8F0006FEA53418AB201E059044A0CA0F844207F
:10C90000704783899BB20AB1194301E023EA010110
:10C9100081817047038B23F0080213041A0C114322
:10C9200001837047038B23F4006213041A0C42EA5C
:10C9300001218BB203837047838B23F00802130419
:10C940001A0C114381837047838B23F40062130414
:10C950001A0C42EA01218BB28383704781847047AD
:10C96000038B23F00C0213041A0C0283038B9AB27C
:10C97000114301837047038B23F4406213041A0CA4
:10C980000283038B9AB242EA01218BB20383704780
:10C99000838B23F00C0213041A0C8283838B9AB2CC
:10C9A000114381837047838B23F4406213041A0C74
:10C9B0008283838B9AB242EA01218BB283837047D0
:10C9C000F8B50B880D4604464988AA8843B92B89D7
:10C9D000FFF7AAFDE9882046BDE8F840FFF7C0BF91
:10C9E000042B08D12B89FFF7D3FDE9882046BDE849
:10C9F000F840FFF7C0BF082B0E462F89008C3BD1B3
:10CA000020F480731804030C2384A08B83B223F0DA
:10CA1000F30343EA0717374B208CBFB29C4280B226
:10CA200047EA020212D003F500639C420ED0B4F133
:10CA3000804F0BD0A3F598339C4207D003F5806359
:10CA40009C4203D003F580639C4207D120F4007020
:10CA500040EA06218BB243F4807305E020F42060A5
:10CA600041F4807140EA0103E9882046A2832384CF
:10CA7000BDE8F840FFF78CBF20F480531804030C86
:10CA80002384A38B208C23F440731B051B0D43EAE6
:10CA9000022242EA0733174A80B294429BB212D074
:10CAA00002F5006294420ED0B4F1804F0BD0A2F593
:10CAB0009832944207D002F58062944203D002F586
:10CAC0008062944207D120F4005040EA063291B2CD
:10CAD00041F4805205E047F6FF52024041F4805194
:10CAE0000A43E9882046A3832284BDE8F840FFF783
:10CAF0005ABF00BF002C0140808E80B27047008F6B
:10CB000080B27047808F80B27047B0F8400080B22A
:10CB10007047038A828911EA030092B203D011425E
:10CB20000CBF002001207047C9438AB202827047BF
:10CB3000038A30B50D460446EA8898B220F4405185
:10CB400011432182A3892889A98823F4B05340EA9C
:10CB50000102688923F00C0102430804030C1A4304
:10CB600091B2A181A08AAA8983B223F4407187B0CF
:10CB70001143A18201A800F0EBF81848A389844270
:10CB80000CBF0498039819B200294FF019032A68C2
:10CB900003FB00F001DA510000E09100B0FBF1F17D
:10CBA0006423B1FBF3F21201100903FB1011A089F9
:10CBB00000B2002806DAC9003231B1FBF3F303F00A
:10CBC000070005E009013231B1FBF3F303F00F0078
:10CBD000024390B2208107B030BD00BF0038014051
:10CBE000838919B199B241F4005303E023F4005151
:10CBF0000A04130C83817047C1F3421310B501245A
:10CC000001F01F01A34204FA01F101D10C3004E04C
:10CC1000022B01D1103000E01430036812B143EA56
:10CC2000010201E023EA0102026010BD838A9BB287
:10CC30000AB1194301E023EA010181827047000033
:10CC4000034A044B02F188305A605860704700BFB5
:10CC50002301674500200240024B1A6942F0800020
:10CC60001861704700200240014BD860704700BF38
:10CC700000200240084BDA68D20709D4D868400780
:10CC800008D4D96811F0100F0CBF0420032070479E
:10CC900001207047022070470020024010B5044672
:10CCA000FFF7E8FF012806D11CB1FFF7E3FF013CC5
:10CCB000F8E7052010BD002C08BF052010BD0000BE
:10CCC00073B5002306464FF400500D460193FFF75D
:10CCD000E5FF04281AD10E4CAAB2206940F00101E8
:10CCE00021614FF400503280FFF7D8FF042808D1AB
:10CCF00002360196019B2D0C1D804FF40050FFF76A
:10CD0000CDFF216941F6FE720A4022617CBD00BF61
:10CD10000020024038B505464FF43020FFF7BEFF33
:10CD2000042812D1094C236943F002002061656197
:10CD300021694FF4302041F040022261FFF7AEFF3D
:10CD4000216941F6FD730B40236138BD002002408C
:10CD5000204B10B55A6802F00C01042903D00829B1
:10CD600005D01D4B01E01D4C2368036011E05C6899
:10CD70005968C4F38342941CC90301D4184A06E0DD
:10CD800016495B680A6813F4003F18BF5208544301
:10CD90000460104B5968C1F3031212498C5C02689D
:10CDA00022FA04F242605C68C4F302240C5D22FAA9
:10CDB00004F484605C68C4F3C224095D22FA01F2C1
:10CDC000C2605B680849C3F38133CB5CB2FBF3F20A
:10CDD000026110BD0010024000127A0060010020C4
:10CDE00000093D006C01002068010020044B5A69D5
:10CDF00009B1104301E022EA00005861704700BF0A
:10CE000000100240044B9A6909B1104301E022EA84
:10CE100000009861704700BF00100240044BDA69BF
:10CE200009B1104301E022EA0000D861704700BF59
:10CE300000100240044BDA6809B1104301E022EA15
:10CE40000000D860704700BF00100240044B1A6910
:10CE500009B1104301E022EA00001861704700BFE9
:10CE600000100240024B5A6A42F0807058627047CC
:10CE70000010024008B50B4B984207D14FF4001048
:10CE80000121FFF7E3FF4FF4001006E04FF48000AC
:10CE90000121FFF7DBFF4FF480000021BDE80840CF
:10CEA000FFF7D4BF00540040F0B58688044687B031
:10CEB00026F03F000D46010401A80E0CFFF748FFC5
:10CEC0002C4A0399B1FBF2F087B23E43A680238837
:10CED00023F0010213041A0C22802B68264A934285
:10CEE0000AD85B00B1FBF3F0013783B2BFB22784ED
:10CEF000032B98BF042320E0EE884BF6FF72964286
:10CF000004D103225343B1FBF3F305E01922534349
:10CF1000B1FBF3F141F4804399B20A054FF49672E4
:10CF200008BF41F00101504341F400434FF47A71CE
:10CF300090FBF1F0421C91B22184A383228891B22C
:10CF400041F001032380208820F4816222F0020155
:10CF50000B04AA886989180C41EA02032989AA8965
:10CF6000184380B241EA0203208098B2208107B0C2
:10CF7000F0BD00BF40420F00A086010041F288339F
:10CF8000002103604BF6FF724FF480438180C28022
:10CF90000181418183817047038819B199B241F0C1
:10CFA000010303E023F001010A04130C038070471E
:10CFB000038819B199B241F4807303E023F48071BE
:10CFC0000A04130C03807047038819B199B241F425
:10CFD000007303E023F400710A04130C038070470C
:10CFE000038819B199B241F4806303E023F48061AE
:10CFF0000A04130C0380704783889BB20AB119435B
:10D0000001E023EA01018180704701827047008AB4
:10D01000C0B2704712B141F0010101E001F0FE0120
:10D020000182704702684FF6FE73134003602D4B78
:10D0300000219842016041608160C16022D02A498C
:10D04000884229D0294B984230D02949884237D08C
:10D05000284B98423ED0284B984206D153F8681C82
:10D0600041F4700043F8680C70472449884206D1A7
:10D0700051F87C0C40F0706241F87C2C7047204BDA
:10D08000984206D153F8042C42F00F0143F8041CD7
:10D0900070471C49884206D151F8183C43F0F00013
:10D0A00041F8180C7047184B984206D153F82C2CB5
:10D0B00042F4706143F82C1C70471449884206D131
:10D0C00051F8403C43F4704041F8400C7047104B1D
:10D0D000984205D153F8542C42F4702143F8541C63
:10D0E000704700BF080002401C00024030000240B0
:10D0F00044000240580002406C00024080000240A0
:10D10000080402401C04024030040240440402406F
:10D110005804024070B506688C680D6A26F4FF4218
:10D1200022F070060A6945EA04034C6913438A69D0
:10D130002343CC6913431C434B6A44EA03028B6AC2
:10D140001A4332430260CB680A68496843608260D0
:10D15000C16070BD0023036043608360C3600361EE
:10D1600043618361C361036243628362704719B1A3
:10D17000016841F0010303E002684FF6FE731340BB
:10D180000360704703680AB1194301E023EA010113
:10D190000160704741607047406880B2704700008E
:10D1A000C3004CBF014B024B586070470004024063
:10D1B0000000024000B540F6D87320F00042C3F6EC
:10D1C00049739A4283B0014615DDB2F1FF4F03DB8C
:10D1D000F3F76EFC03B000BD694601F0C9F800F03A
:10D1E0000302012A009801990ED0022A07D082B9C1
:10D1F00001F0D4FAEEE7002101F0D0FAEAE701F0FD
:10D20000CDFA00F10040E5E702F074F900F10040CA
:10D21000E0E7012202F06EF9DCE700BF30B5C0F3B1
:10D22000C754A4F17F031E2B83B0014621DC581C98
:10D230001DDBCD0F162B0CDD21F07F4323F4000006
:10D2400040F40000963C00FA04F005B1404203B0FF
:10D2500030BD114850F825402046F3F72BFC0190D3
:10D2600021460198F3F724FC20F0004121B9002069
:10D27000EDE7F3F7EDFEEAE720F07F4222F400034A
:10D28000C0F3C75043F40001C0F1960221FA02F046
:10D29000002DDCD0DAE700BF7430010800B540F69D
:10D2A000D87320F00042C3F649739A4283B0014616
:10D2B00016DDB2F1FF4F03DBF3F7FAFB03B000BD5D
:10D2C000694601F055F800F00300012815D0022846
:10D2D0000BD0B8B900980199012202F00BF9EDE7E3
:10D2E0000021002202F006F9E8E7009801990122E6
:10D2F00002F000F900F10040E0E70098019901F028
:10D300004DFADBE70098019901F048FA00F100407E
:10D31000D4E700BF70B58AB0064600F02FFA224C61
:10D32000054694F90030013303D0304602F080FB0B
:10D3300010B928460AB070BD304602F023FB4FF00A
:10D340007E51F3F77BFE0028F3D0184A0121002517
:10D350003046019200910895F3F768F802460B46B3
:10D360001348CDE90423CDE9022302F045F994F9ED
:10D370000030CDE90601022B0BD0684602F03AF9E5
:10D3800038B1089850B9DDE90601F3F73DFB0546D1
:10D39000CFE702F05DFC21210160F2E702F058FCCA
:10D3A000089A0260EFE700BF7C0100207C30010892
:10D3B0008830010800F096BB2DE9F0418AB007469D
:10D3C0000D4600F035FC854E044696F900300133D9
:10D3D00003D0284602F02CFB18B920460AB0BDE85D
:10D3E000F081384602F024FB8046002833D12846DD
:10D3F0000021F3F7FBFD0028EFD0794A01213846E0
:10D4000001920091CDF82080F3F710F8CDE90201E8
:10D410002846F3F70BF8002396F900400022C3F6E4
:10D42000F073CDE90623631CCDE904010DD0022C75
:10D430000BD0684602F0DEF8002800F09A800898C9
:10D4400018B102F005FC08990160DDE90601F3F767
:10D45000DBFA0446C1E738460021F3F7C7FD20B3E5
:10D4600028460021F3F7C2FD002855D05C4B01226D
:10D4700000243846009201930894F2F7D7FFCDE9D3
:10D4800002012846F2F7D2FF96F90040002200235D
:10D49000CDE90401CDE90623002CCAD000230022E7
:10D4A000C3F6F073CDE90623CFE7204602F06EFA0B
:10D4B0008046002862D020460021F3F797FD00281F
:10D4C0008BD0384602F062FA002886D0284602F057
:10D4D0005DFA002881D0424A042100243846019296
:10D4E00008940091F2F7A2FFCDE902012846F2F775
:10D4F0009DFF96F9004000220023022CCDE9040193
:10D50000CDE9062365D0684602F074F8002860D0A3
:10D510000898002899D094E7284602F037FA0028A6
:10D520003FF45BAF28460021F3F76AFD00283FF483
:10D5300054AF2B4A002301213846019208930091F1
:10D54000F2F774FFCDE902012846F2F76FFF347855
:10D55000CDE9040100220023002C32D0CFF6F07375
:10D56000022CCDE906232ED102F072FB21210160AD
:10D57000CEE702F06DFB2123036060E7384602F03E
:10D5800005FA002897D0284602F000FA002892D029
:10D59000204602F04DFA0146384619BB104B0122D5
:10D5A000009201930891F2F741FFCDE9020128466C
:10D5B000F2F73CFF3478CDE90401002C65D100225C
:10D5C0000023CDE90623684602F014F800289FD115
:10D5D000CAE702F03DFB2223036099E77C010020AB
:10D5E000843001083D4C032200920194CDF8208044
:10D5F000F2F71CFFCDE902012846F2F717FF96F972
:10D600000030CDE9040138460021D3B94FF6FF734D
:10D610004FF06042C4F2EF73CDE90623F3F7F0FC5C
:10D6200000283ED196F90000022805D0684601F096
:10D63000E1FF00287FF403AF02F00AFB2221016022
:10D64000FDE600230022C7F6F073CDE90623F3F7C9
:10D65000D7FC0028E6D04FF07C512846F3F732FB88
:10D66000F2F7E4FE04460D4601F0CCFF02460B46FD
:10D6700020462946F3F796F90028D3D1002300224B
:10D68000CFF6F073CDE90623CCE700200021024657
:10D690000B46F3F749F8022CCDE906013FF464AFDD
:10D6A00091E74FF07C512846F3F70CFBF2F7BEFEF2
:10D6B00004460D4601F0A6FF02460B4620462946C9
:10D6C000F3F770F90028ADD14FF6FF734FF06042C9
:10D6D000CCF2EF73CDE90623A4E700BF8430010844
:10D6E00070B58AB0054600F0EFFF224C064694F96B
:10D6F0000030013308D0284602F09AF920B12846BC
:10D700000021F3F77DFC10B930460AB070BD1A4A0B
:10D71000012128460026009101920896F2F786FE24
:10D720002478CDE90401CDE902017CB9002200236F
:10D73000CDE90623684601F05DFF88B10898A0B9DD
:10D74000DDE90601F3F760F90646DDE70020002178
:10D7500002460B46F2F7E8FF022CCDE90601E9D1BB
:10D7600002F076FA21230360E8E702F071FA0899E3
:10D770000160E5E77C0100208C300108F8B520F05D
:10D780000043B3F17E5F044613D00BDCB3F17C5F42
:10D7900014DAB3F10C5F00F3A48040F6DB70C3F63B
:10D7A000C970F8BD0146F3F783F90146F3F73EFB74
:10D7B000F8BD002840F30E810020F8BD0028C0F21B
:10D7C0000E8101464FF07E50F3F772F94FF07C5115
:10D7D000F3F778FA044600F077FF4EF60871064634
:10D7E00020F47F65C3F611012046F3F76BFA47F684
:10D7F0000471C3F64F21F3F75DF92146F3F762FA9E
:10D8000041F24611C3F62451F3F752F92146F3F7DA
:10D8100059FA40F6A821C3F64E61F3F74BF92146B9
:10D82000F3F750FA4BF29001C3F6A661F3F740F913
:10D830002146F3F747FA4AF6AB21C3F62A61F3F71C
:10D8400039F92146F3F73EFA4CF22E610746C3F64A
:10D850009D512046F3F736FA43F26131C3F6307139
:10D86000F3F726F92146F3F72DFA45F22D71C4F2AC
:10D870000101F3F71FF92146F3F724FA4DF23911AC
:10D88000C4F21901F3F714F92146F3F71BFA4FF02C
:10D890007E51F3F70FF901463846F3F7C7FA3146E0
:10D8A000F3F710FA25F00F05074629462846F3F747
:10D8B00009FA01462046F3F7FBF8294604463046AC
:10D8C000F3F7F8F801462046F3F7B0FA0146384678
:10D8D000F3F7F0F82946F3F7EDF80146F3F7EAF825
:10D8E000F8BD0146F3F7EEF94EF60871C3F61101E3
:10D8F0000546F3F7E7F947F60471C3F64F21F3F74E
:10D90000D9F82946F3F7DEF941F24611C3F624515E
:10D91000F3F7CEF82946F3F7D5F940F6A821C3F678
:10D920004E61F3F7C7F82946F3F7CCF94BF29001B3
:10D93000C3F6A661F3F7BCF82946F3F7C3F94AF634
:10D94000AB21C3F62A61F3F7B5F82946F3F7BAF924
:10D950004CF22E610646C3F69D512846F3F7B2F904
:10D9600043F26131C3F63071F3F7A2F82946F3F7B9
:10D97000A9F945F22D71C4F20101F3F79BF829468C
:10D98000F3F7A0F94DF23911C4F21901F3F790F849
:10D990002946F3F797F94FF07E51F3F78BF80146DC
:10D9A0003046F3F743FA01462046F3F78BF9014678
:10D9B00042F26810C3F2A230F3F77AF8014620462B
:10D9C000F3F776F8014640F6DA70C3F6C970F3F75C
:10D9D0006FF8F8BD40F6DB70C4F24900F8BD4FF0B7
:10D9E0007E51F3F767F84FF07C51F3F76BF94EF681
:10D9F0000871C3F611010446F3F764F947F60471A0
:10DA0000C3F64F21F3F756F82146F3F75BF941F2DD
:10DA10004611C3F62451F3F74BF82146F3F752F9B8
:10DA200040F6A821C3F64E61F3F744F82146F3F718
:10DA300049F94BF29001C3F6A661F3F739F8214694
:10DA4000F3F740F94AF6AB21C3F62A61F3F732F84F
:10DA50002146F3F737F90646204600F035FE4CF232
:10DA60002E610546C3F69D512046F3F72BF943F28C
:10DA70006131C3F63071F3F71BF82146F3F722F951
:10DA800045F22D71C4F20101F3F714F82146F3F7C2
:10DA900019F94DF23911C4F21901F3F709F82146C9
:10DAA000F3F710F94FF07E51F3F704F801463046D2
:10DAB000F3F7BCF92946F3F705F942F26811C3F20E
:10DAC000A231F2F7F5FF01462846F2F7F3FF0146CF
:10DAD000F2F7F0FF014640F6DA70C4F24900F2F7BF
:10DAE000E7FFF8BDF8B521F00044B4F1FF4F03465D
:10DAF00017DC20F00045B5F1FF4F064611DCB1F10F
:10DB00007E5F42D08F1707F0020040EAD37775B9E5
:10DB1000022F35D0032F08D140F6DB73CCF2490336
:10DB200003E01846F2F7C6FF03461846F8BDD4B125
:10DB3000B4F1FF4F2DD0B5F1FF4F14D02C1BE415DD
:10DB40003C2C18DC002952DB1846F3F76FF901F082
:10DB500019FF01F0EBFD012F46D0022F35D0002F29
:10DB600025D10346E1E7002E40F6DB731CDBC3F64C
:10DB7000C9731846F8BD40F6DB70C3F6C970EAE712
:10DB800040F6DB73C4F24903CFE7BDE8F84001F08B
:10DB9000CDBDB5F1FF4F2FD0022FF1D0032FBBD059
:10DBA000012F34D00023C0E7CBF6C973BDE74BF695
:10DBB0002E51C3F2BB31F2F77DFF40F6DB71C4F2A8
:10DBC0004901F2F775FF0346AFE74BF62E51C3F25A
:10DBD000BB31F2F76FFF014640F6DB70C4F249003B
:10DBE000F2F766FF0346A0E700F100439DE714F15A
:10DBF0003C0FA9DA0020AEE7022F13D0032F0CD080
:10DC0000012F40F6DB7305D0C3F649738DE74FF063
:10DC100000438AE7CBF6497387E74CF6E433CCF24E
:10DC2000160382E74CF6E433C4F216037DE700BF27
:10DC30002DE9F04F31F0004987B00C460D460746FC
:10DC400011D020F0004ABAF1FF4F804605DD54485C
:10DC500007B0BDE8F04F01F017BFB9F1FF4F08DD85
:10DC6000BAF17E5FF3D14FF07E54204607B0BDE895
:10DC7000F08F002854DB0026B9F1FF4F49D0B9F1ED
:10DC80007E5F64D0B5F1804F38463ED0B5F17C5F01
:10DC90001FD001F077FEBAF1FF4F014621D0BAF153
:10DCA000000F1ED0BAF17E5F1BD04FEAD87808F182
:10DCB000FF3856EA08015FD0B9F19A4F72DD4FF68E
:10DCC000F771C3F67F718A4513DC002D19DB002440
:10DCD000CBE7B8F1000FDCDB07B0BDE8F04F00F098
:10DCE000F3BC002D50DB0846B8F1000F3ADB0446C8
:10DCF000BBE70723C3F680739A4540F3E982002D02
:10DD0000E5DD4FF2CA20C7F249100146F2F7DAFF0B
:10DD1000EDE7BAF17E5FA6D01FDD002DA5DAD6E7CC
:10DD2000B9F1974F17DAB9F17E5F09DB4FEAE95392
:10DD3000C3F1960049FA00F202FA00F1494501D018
:10DD400000269CE702F00106C6F1020697E7002DC7
:10DD50001FDB3C4689E702268EE7002DB7DA04F187
:10DD6000004482E7AAF17E5156EA010A05D0012E4D
:10DD7000BDD100F1004478E738460146F2F798FE3D
:10DD80000146F3F753F8B2E74FF07E50F3F74EF841
:10DD9000AAE74FF07E503946F3F748F8044664E7A7
:10DDA00088300108BAF5000F80F222824FF09741C7
:10DDB000F2F788FF6FF0170782462AF07F434CF294
:10DDC000714223F400014FEAEA50C0F21C027F388E
:10DDD000914200EB070C41F07E5740F306824BF274
:10DDE000D630C0F25D00814240F3B88200220CF1CF
:10DDF000010CA7F5000705920599A948CDF804C0C4
:10DE000050F821303846194604930392F2F750FE39
:10DE1000394681460498F2F74DFE01464FF07E5098
:10DE2000F3F704F80246114648460292F2F74AFF19
:10DE3000BB467F10039A47F00051824601F58023CC
:10DE400020F47F60D31820F00F071946384603935B
:10DE5000F2F738FF01464846F2F72AFE0399814659
:10DE600008460499F2F724FE01465846F2F720FED0
:10DE70003946F2F727FF01464846F2F719FE029AA3
:10DE80001146F2F71FFF514683465046F2F71AFF3C
:10DE900001468146F2F716FF4FF242110346C3F6E0
:10DEA000536148460293F2F70DFF43F25521C3F642
:10DEB0006C61F2F7FFFD4946F2F704FF4AF20531C3
:10DEC000C3F68B61F2F7F6FD4946F2F7FBFE4AF620
:10DED000AB21C3F6AA61F2F7EDFD4946F2F7F2FE77
:10DEE00046F6B751C3F6DB61F2F7E4FD4946F2F7B7
:10DEF000E9FE49F69A11C3F61971F2F7DBFD014606
:10DF00000298F2F7DFFE394681465046F2F7D2FD1D
:10DF10005946F2F7D7FE4946F2F7CCFD3946049050
:10DF20003846F2F7CFFE0021C4F240010390F2F729
:10DF3000C1FD0499F2F7BEFD20F47F6121F00F09C5
:10DF400049463846F2F7BEFE494607465846F2F7BC
:10DF5000B9FE00218346C4F240014846F2F7A8FD0D
:10DF6000039B1946F2F7A4FD01460498F2F7A0FDC1
:10DF70005146F2F7A7FE01465846F2F79BFD83464D
:10DF800059463846F2F796FD20F47F6C2CF00F0AC4
:10DF90004FF46051C3F676715046F2F793FE4CF29F
:10DFA000A0318146C3F29D615046F2F78BFE39469F
:10DFB000024650460292F2F77BFD01465846F2F7C0
:10DFC00077FD43F64F01C3F67671F2F77BFE01460B
:10DFD0000298F2F76FFD059F324951F82710F2F7CA
:10DFE00069FDDDF804B007465846F2F717FE2E4BE0
:10DFF000059A049053F822B039464846F2F75AFD84
:10E000005946F2F757FD0499F2F754FD20F47F6C5E
:10E010002CF00F0A04995046F2F74AFD5946F2F7E0
:10E0200047FD4946F2F744FD01463846F2F740FD08
:10E03000013E56EA0806814640F0D4800027CBF620
:10E04000807725F47F6525F00F0529462046F2F7F5
:10E050002FFD5146F2F736FE494606462046F2F7B6
:10E0600031FE01463046F2F725FD294680465046EE
:10E07000F2F728FE014604464046F2F71BFD002851
:10E0800006460546A246014620F0004940F30181BC
:10E09000B9F1864F00F3BF8000F0AC8006E000BF0E
:10E0A000A43001089C30010894300108B9F17C5F6C
:10E0B00000F3C0804FF0000BD94621F47F6525F0B6
:10E0C0000F044FF4E4412046C3F63171F2F7FAFD34
:10E0D000514605462046F2F7EBFC01464046F2F772
:10E0E000E7FC47F21821C3F63171F2F7EBFD4BF66E
:10E0F0008C610646C3F2BF512046F2F7E3FD0146AC
:10E100003046F2F7D7FC064631462846F2F7D2FCF5
:10E1100029460446F2F7CCFC01463046F2F7C8FC2B
:10E12000214606462046F2F7CDFD4BF64C31C3F2B0
:10E1300031310546F2F7C6FD4EF60E21C3F2DD5130
:10E14000F2F7B6FC2946F2F7BDFD4BF25531C3F6A6
:10E150008A01F2F7AFFC2946F2F7B4FD40F66131CF
:10E16000C3F63631F2F7A4FC2946F2F7ABFD4AF6C6
:10E17000AB21C3F62A61F2F79DFC2946F2F7A2FD16
:10E1800001462046F2F794FC054629462046F2F760
:10E1900099FD4FF0804180462846F2F789FC014600
:10E1A0004046F2F743FE314605462046F2F78AFD27
:10E1B0003146F2F77FFC01462846F2F779FC21460A
:10E1C000F2F776FC01464FF07E50F2F771FC834483
:10E1D000BBF5000FC0F2C78059463846F2F772FD12
:10E1E000044642E54FF07E572BE70022059203E6F6
:10E1F0000027E2E54AF63C21C3F238314046F2F707
:10E2000059FC214682463046F2F752FC0146504600
:10E21000F2F714FF70B14FF2CA21C7F24911384624
:10E22000F2F750FD4FF2CA21C7F24911F2F74AFD49
:10E2300004461AE54FEAE953A3F17E004FF40006C5
:10E2400046FA00F14B19C3F3C75223F07F4E4FF645
:10E25000FF76A2F17F002EF4000CC0F27F064CF492
:10E26000000AC2F1960246FA00F64AFA02F923EAD7
:10E270000601002D2046B8BFC9F10009F2F718FCCD
:10E28000824651464046F2F715FC4FEAC95B01460B
:10E2900013E70022C4F2163291450ADC7FF406AF80
:10E2A0002146F2F705FC01464046F2F7B3FE00288E
:10E2B000C0D044F26021C0F6A2513846F2F702FD08
:10E2C00044F26021C0F6A251F2F7FCFC0446CCE413
:10E2D0004FF07E51F2F7ECFB4FF42A41C3F6B871D0
:10E2E0000746F2F7EFFC4AF270518146C3F2EC6147
:10E2F0003846F2F7E7FC394682463846F2F7E2FC48
:10E300004FF07A5183463846F2F7DCFC01464AF674
:10E31000AB20C3F6AA60F2F7CBFB3946F2F7D2FC8A
:10E3200001464FF07C50F2F7C3FB01465846F2F726
:10E33000C9FC4AF63B21C3F6B871F2F7C3FC0146AB
:10E340005046F2F7B5FB074639464846F2F7B2FBAE
:10E3500020F47F6020F00F0A504662E601234FF45C
:10E360000012059348E5494601F092FB014634E767
:10E370002DE9F04F40F6D87320F00044C3F64973FE
:10E380009C4289B006460D4640F38B804CF6E33143
:10E39000C4F216018C4226DC4FF478610028C3F6E3
:10E3A000C97140F32B81F2F783FB4FF47D6224F0B7
:10E3B0000F04C3F6C9729442064600F0818044F20D
:10E3C0004341C3F23571F2F773FB014628603046D2
:10E3D000F2F76EFB44F24341C3F23571F2F768FB8A
:10E3E0000127686061E04FF47867C4F24937BC42A6
:10E3F00040F38180B4F1FF4F5BDA4FEAE459A9F1B1
:10E400008609A4EBC9542046F2F722FEF2F706FC77
:10E410000246014620460592F2F74AFB4FF087413B
:10E42000F2F750FC0746F2F713FEF2F7F7FB01464E
:10E43000044638460694F2F73BFB4FF08741F2F76B
:10E4400041FC00210790F2F7D1FD002800F0F68092
:10E450000327204600210DF11808013FF2F7C6FD01
:10E4600040B158F8044D00212046013FF2F7BEFDAF
:10E470000028F6D1924B02200090019305A83B465C
:10E4800029464A4600F066FA002E07460DDA95E85E
:10E490000C0002F1004103F1004229606A6047422A
:10E4A00003E00023286000274B60384609B0BDE830
:10E4B000F08F0146F2F7FCFA002768602860F4E765
:10E4C0004FF48841C3F23571F2F7F2FA4AF208319B
:10E4D000C2F685610446F2F7EBFA01462860204651
:10E4E000F2F7E6FA4AF20831C2F68561F2F7E0FA8D
:10E4F00001276860D9E701F045FA4FF68411C3F6A9
:10E5000022718046F2F7DEFB4FF07C51F2F7D2FA2F
:10E51000F2F79EFD0746F2F781FB4FF47861C3F6F0
:10E52000C9718346F2F7CEFB01464046F2F7C0FAC6
:10E5300044F243418146C3F235715846F2F7C2FBBB
:10E540001F2F8246514648461FDC5E4B7A1E53F809
:10E55000223024F0FF029A4217D0F2F7A9FA80463F
:10E56000C5F8008041464846F2F7A2FA5146F2F754
:10E570009FFA002E686098DA08F1004800F1004127
:10E58000C5F8008069607F428FE7F2F791FAE315E2
:10E590008046C0F3C750191A0829E1DD4FF48841BD
:10E5A000C3F2357158460393F2F78CFB824651460D
:10E5B0004846F2F77DFA044621464846F2F778FAD3
:10E5C0005146F2F775FA4AF208318146C2F6856182
:10E5D0005846F2F777FB4946F2F76AFA8246514607
:10E5E0002046F2F765FA039BC0F3C7528046981A9B
:10E5F000192841DCC5F80080A146B3E7F2F75AFAC2
:10E600004FF47D6724F00F04C3F6C977BC42064679
:10E6100016D044F24341C3F23571F2F74BFA01468A
:10E6200028603046F2F744FA44F24341C3F23571B0
:10E63000F2F740FA4FF0FF37686036E7032719E733
:10E640004FF48841C3F23571F2F734FA4AF20831D7
:10E65000C2F685610446F2F72DFA0146286020468D
:10E66000F2F726FA4AF20831C2F68561F2F722FA89
:10E670004FF0FF37686018E74FF42341C2F6856119
:10E680005846F2F71FFB804641462046F2F710FA43
:10E69000814649462046F2F70BFA4146F2F708FA5E
:10E6A00043F232110446C2F28D415846F2F70AFB9A
:10E6B0002146F2F7FDF98246514648464DE700BF34
:10E6C0002C310108AC30010820F00042B2F1FF4FBC
:10E6D000F8B50446034646D2002A42D0002852DB51
:10E6E000C415B2F5000F09D210F4000553D15B0038
:10E6F00001351902FBD5C5F10100241823F07F4133
:10E700007F3C21F40006E20746F4000048BF4000C9
:10E7100043004FF08072002760109A423C462CDD87
:10E720005B004FF400021825A61851089E4205F11F
:10E73000FF3502DCB4189B1BBF185B0062189A42BD
:10E7400002DC9B1A54187F185B004A08013DEBD18C
:10E7500013B107F001017F187C1004F17C5303EB27
:10E76000C0542046F8BD0146F2F7ACFA01462046F7
:10E77000F2F7A0F904462046F8BD4FF0007403F10B
:10E780007F431746CCE70146F2F792F90146F2F7CC
:10E790004DFB0446E5E70120AFE700BF2DE9F84354
:10E7A00020F00046B6F1485F05460F465BDAF2F707
:10E7B0004FFC002800F0CA8029462846F2F782FA6A
:10E7C0004DF24E71CAF647510446F2F77BFA47F212
:10E7D000F641C3F20F11F2F76DF92146F2F772FA22
:10E7E0004FF27C21C3F29341F2F762F92146F2F72E
:10E7F00069FA40F60151C3F2D071F2F75BF9214694
:10E80000F2F760FA40F66131C3F6B621F2F750F93B
:10E810002146F2F757FA4AF6AB21C3F62A51F2F72E
:10E8200049F92146F2F74EFA804620464FF07C51D6
:10E83000F2F748FA414606462046F2F743FA3946CF
:10E8400004462846F2F73EFA01462046F2F730F930
:10E8500001463046F2F72CF901464FF07E50F2F7B0
:10E8600027F9BDE8F8830146F2F72CFA4DF24E7114
:10E87000CAF647510446F2F725FA47F2F641C3F2C9
:10E880000F11F2F717F92146F2F71CFA4FF27C212B
:10E89000C3F29341F2F70CF92146F2F713FA40F66E
:10E8A0000151C3F2D071F2F705F92146F2F70AFAE5
:10E8B00040F66131C3F6B621F2F7FAF82146F2F7D5
:10E8C00001FA4AF6AB21C3F62A51F2F7F3F82146D2
:10E8D000F2F7F8F949F69913C3F699639E42804618
:10E8E000A3DD0020C3F64870864227DC06F17F4690
:10E8F0004FF07E503146F2F7DBF8814620464FF06C
:10E900007C51F2F7DFF93146F2F7D2F8414606467C
:10E910002046F2F7D7F9394604462846F2F7D2F9ED
:10E9200001462046F2F7C4F801463046F2F7C0F837
:10E9300001464846F2F7BCF8BDE8F8834FF00009FD
:10E940000026C3F63879C3F69066D7E74FF07E50BD
:10E95000BDE8F8832DE9F04FDFB00C930C9D224BFE
:10E96000689C0A91691ED61E48BF161D834653F83F
:10E970002400F71027EAE7730890049104980D9398
:10E98000089DDC43DDF834C002EBC4024119079254
:10E99000C0EB0C0750D47E18699BC7EB0609013603
:10E9A000002F03EB870522AC09F0010AC0F2FE82BA
:10E9B0002868F2F733F90137B74220604FF00408B6
:10E9C0003AD0BAF1000F26D0002FC0F2F18255F8EC
:10E9D0000800F2F723F90137B74244F8080008F1BC
:10E9E000040818D128E000BF4434010855F8080095
:10E9F000F2F714F9013708F1040944F8080013D4B8
:10EA000055F80900F2F70AF90137B74244F809004E
:10EA100009F1040810D0002FE8DA0020013708F1CE
:10EA2000040944F80800EBD501370020B74244F848
:10EA3000090009F10408EED1089A002AC0F24585C0
:10EA400008990C9E8D004AAB5C19039549AF02945E
:10EA50004FEA860A049A002AC0F296820DF18808CD
:10EA600008EB860555F8041CAAF10403DBF8000046
:10EA7000C3F38009F2F726F901460020F2F71AF8ED
:10EA80000424043D544580462BD0B9F1000F0DD02D
:10EA900055F8041DDBF80400F2F714F9014640466E
:10EAA000F2F708F80824544580461AD055F8041C9B
:10EAB0005BF80400F2F706F901464046F1F7FAFF69
:10EAC0000434804655F8081C5BF80400F2F7FAF8A5
:10EAD00001464046F1F7EEFF0434083D54458046B8
:10EAE000E4D1029847F8048F01368742B2D1039FE0
:10EAF0000EA9CE190996089EB2005EAB9D18002E95
:10EB0000029255F8509C7DDD0DF5947C4FF06E51CE
:10EB100048460DACA7180CEB0205F2F7D3F8F2F754
:10EB200097FAF2F77BF84FF087410190F2F7CAF8B5
:10EB300001464846F1F7BCFFF2F78AFA0EAC2060B6
:10EB40000198014655F8040DF1F7B4FFBC42814627
:10EB5000C7F3800156D0E9B14FF06E51F2F7B2F829
:10EB6000F2F776FAF2F75AF84FF087410190F2F790
:10EB7000A9F801464846F1F79BFFF2F769FA019AB6
:10EB80000FAC2060114655F8040DF1F793FFBC421D
:10EB9000814637D04FF06E514846F2F793F8F2F7BE
:10EBA00057FAF2F73BF84FF087418046F2F78AF8C0
:10EBB00001464846F1F77CFFF2F74AFA41466060A9
:10EBC00055F8040DF1F776FF4FF06E518146F2F7DC
:10EBD00079F8F2F73DFAF2F721F84FF087418046D5
:10EBE000F2F770F801464846F1F762FFF2F730FAA3
:10EBF0004146A06055F8040DF1F75CFF0834BC42B3
:10EC00008146C7D10799484600F042FF4FF078513E
:10EC10000546F2F757F800F0C1FE4FF08241F2F7D7
:10EC200051F801462846F1F743FF0746F2F710FA7C
:10EC30008146F1F7F3FF01463846F1F739FF0799AE
:10EC40000746002940F33981721E0EAC079D54F827
:10EC50002230C5F1080043FA00F101FA00F0C5F1D5
:10EC600007041B1A43FA04F40DF1380C89444CF8DC
:10EC70002230002C55DD002E09F1010940F394816A
:10EC8000029D0EABDDF808C053F8042B281F0DF1D0
:10EC9000380E00250EEB0C01C0F3800022B1C2F546
:10ECA000807243F8042C01258B4226D060B10F9A64
:10ECB0000433002D40F0F38022B1C2F5807543F893
:10ECC000045C01258B4218D053F8042B002D40F032
:10ECD000EC80C2F5807012B143F8040C012553F8A2
:10ECE000042B002D40F0DB80C2F58070002AE9D0B3
:10ECF00001258B4243F8040CE6D1079900290DDD6C
:10ED0000012900F0E280022908D1701E0DF1380EB1
:10ED10005EF8202002F03F034EF82030022C00F075
:10ED2000E08038460021F2F761F9002800F0F38016
:10ED30000898751EA84225DC029B0DF1380E0EEBDB
:10ED400003010B46DDF824C053F8042DCCEB010081
:10ED5000011F6345C1F3800011D030B153F8041D89
:10ED6000DDF824E00A43734509D0099F53F8040DE8
:10ED700053F8041D0243BB4242EA0102F6D1002AC5
:10ED800040F01A81089F0EAD781E55F82020002A09
:10ED900040F0108105EB8004012354F8041D013379
:10EDA0000029FAD0F018771C87420B9075DCDDF84B
:10EDB00010E00D9D0B9B0C9C0EEB0702DDF808C0CC
:10EDC000699F991B06EB05094AA8A61922AB07EB18
:10EDD000890900EB0C05571C8A0003EB860102959C
:10EDE00006920591002659F8040FF1F717FF059CCC
:10EDF000A051049800285EDB22AD05EB8702AAF142
:10EE00000403C3F3800452F8041CDBF800000394ED
:10EE1000141FF1F757FF01460020F1F74BFE4FF0AA
:10EE20000408D04505462DD0039971B154F8041D4E
:10EE3000DBF80400F1F746FF01462846F1F73AFEF9
:10EE40004FF00808D04505461CD054F8041C5BF868
:10EE50000800F1F737FF01462846F1F72BFE08F1CD
:10EE60000408054654F8081C5BF80800F1F72AFF6F
:10EE700001462846F1F71EFE08F10408083CD0457B
:10EE80000546E2D1DDF808E0069804364EF8045F46
:10EE900001378642CDF808E0A5D10B9E2CE6C2F1E1
:10EEA000FF0243F8042C01250CE7C2F1FF0543F8EB
:10EEB000045C012513E70025E4E75ED1701E0DF127
:10EEC000380E5EF820301C12D3E6711E0DF1380C9E
:10EED0005CF82100022C00F07F024CF821207FF426
:10EEE00020AF39464FF07E50F1F7E2FD0746002D86
:10EEF0003FF417AF07994FF07E5000F0C9FD01466F
:10EF00003846F1F7D5FD074638460021F2F76EF88E
:10EF100000287FF40DAF0294079C38466142CDF87B
:10EF2000109000F0B5FD4FF087410546F2F77CF8F0
:10EF3000002800F0D2824FF06E512846F1F7C2FE51
:10EF4000F2F786F8F1F76AFE4FF087410746F1F7CE
:10EF5000B9FE01462846F1F7ABFDF2F779F80EA9A4
:10EF600041F826003846F2F773F8079A013608325E
:10EF70000EAC079244F8260034E04FF07C51F2F7D3
:10EF800053F858B90024CCE64FF00008029847F82F
:10EF9000048F013687427FF45DADA8E50224002E80
:10EFA00009F101093FF76CAE0025A6E6002002E555
:10EFB000002010E50123F5E6079A0EAE56F825303D
:10EFC000083ACDF8109002940792002B40F08E8200
:10EFD00006EB85042E4654F8045D013E083A002DE8
:10EFE000F9D007924FF07E50079900F051FD002EA6
:10EFF0000446C0F2AC804FEA860AC6EB867B0EAFB1
:10F000004FEA8B095744C9F100034AA9386801EB5C
:10F010000A08C3F3800BF1F701FE2146F1F752FE17
:10F020004FF06E51C8F800002046F1F74BFEA9F1F1
:10F0300004096FF0030ACA45054631D0BBF1000F41
:10F040000BD057F8040CF1F7E9FD2946F1F73AFE29
:10F050006FF0070A48F8040C1AE057F80A00F1F7B5
:10F06000DDFD2946F1F72EFE4FF06E5148F80A00FB
:10F070002846F1F727FEAAF1040405463859F1F7AE
:10F08000CDFD2946F1F71EFEAAF1080A48F8040052
:10F0900028464FF06E51F1F715FECA450546DCD102
:10F0A000701CDFF84C94DDF820A003900027059633
:10F0B000BAF1000FC0F20582002FC0F202820026D2
:10F0C00000241AF0010F354620D0D8F80010D9F8E6
:10F0D0000000F1F7F7FD01462046F1F7EBFC0125B2
:10F0E000AA45044626DB0426BD420FDD22E0BB45CF
:10F0F00020DC58F8021059F80200F1F7E3FD014650
:10F100002046F1F7D7FCBD42044613DC58F8061040
:10F1100059F80600F1F7D6FD01462046F1F7CAFC82
:10F1200005F1010B06F104020235DA45044602F14D
:10F130000406DCDA5EABDDF80CC003EB87010137B7
:10F14000674541F8A04CA8F10408B1D1059E689C20
:10F15000032C16D8DFE814F085011F011F011B00E6
:10F1600000230299002900F00B81379C369804F1A6
:10F1700000420A9C00F1004503F1004325606260F3
:10F18000A360049D05F007005FB0BDE8F08F002E7E
:10F19000E6DD06F1FF3836AF07EB88094D4655F836
:10F1A00004290DF1D40AD5F808B010465946019249
:10F1B000F1F780FC804641460198F1F779FC014661
:10F1C0005846F1F777FC5545C9F38003A860C5F8A8
:10F1D000048044D0BBB155F80429D5F808B01046D6
:10F1E00059460192F1F766FC01998046084641466E
:10F1F000F1F75EFC01465846F1F75CFC5545C5F851
:10F200000480A8602BD02C4654F80439D4F808B0F8
:10F21000184659460193F1F74DFC80464146019846
:10F22000F1F746FC01465846F1F744FCC4F8048067
:10F23000A06055F804BC251FD5F808805846414603
:10F24000F1F738FC044621465846F1F731FC0146F7
:10F250004046F1F72FFC55456C60A860D3D1012ED4
:10F260007FF77EAF4D4655F804B9C7EB090ED5F8C8
:10F2700008A058465146AEF10409F1F71BFC804640
:10F2800041465846F1F714FC01465046F1F712FC8E
:10F29000BD42C9F38009C5F80480A86043D0B9F124
:10F2A000000F15D055F804A9D5F8089050464946E6
:10F2B000F1F700FC804641465046F1F7F9FB014664
:10F2C0004846F1F7F7FBBD42C5F80480A8602AD094
:10F2D0002C4654F804A9D4F8089050464946F1F752
:10F2E000E9FB804641465046F1F7E2FB01464846BD
:10F2F000F1F7E0FBC4F80480A06055F8049C251FDA
:10F30000D5F8088048464146F1F7D4FB044621462B
:10F310004846F1F7CDFB01464046F1F7CBFBBD4235
:10F320006C60A860D4D1013607EB860708353E46ED
:10F330007A1B131F56F8041D0020C3F38007F1F752
:10F34000B9FBAE4203463FF40CAF3FB156F8041D83
:10F35000F1F7B0FBAE4203463FF403AF184656F850
:10F36000041C341FF1F7A6FB083E54F8041CF1F707
:10F37000A1FBAE42F3D10299034600297FF4F5AE1A
:10F38000DDF828C036993798CCF80010CCF8040086
:10F39000CCF80830F5E60023002E29DB36AF751CCB
:10F3A00007EB85042546E21B55F8041DA2F1040E67
:10F3B0000020CEF38008F1F77DFBBD42034617D055
:10F3C000B8F1000F06D055F8041DF1F773FBBD42EC
:10F3D00003460DD0184655F8041C2C1FF1F76AFBA4
:10F3E000083D54F8041CF1F765FBBD42F3D1034618
:10F3F0000299002967D003F10040DDF828C01946C2
:10F40000CCF800003698F1F753FB002E034621DDBF
:10F4100036AF07EB8606F51B2A1F3799C2F3800724
:10F42000F1F748FB37ACB442034613D037B16168FB
:10F43000F1F740FB38ACB44203460BD0184654F801
:10F44000041FF1F737FB54F8041FF1F733FBB44204
:10F45000F5D10346029909B103F100430A9C6360A8
:10F460008FE6002E40DB36AF013607EB86000546FF
:10F47000C21B55F8041D0020141FF1F71BFBBD42F1
:10F48000C4F38006034615D036B155F8041DF1F7D4
:10F4900011FBBD4203460DD0184655F8041C2C1F25
:10F4A000F1F708FB083D54F8041CF1F703FBBD42DB
:10F4B000F3D10346029909B103F100430A9C23608A
:10F4C0005FE6002436E6184697E7DDF830E0900066
:10F4D00003904FEA8E0AFFF70ABB2846F1F7B8FD02
:10F4E0000EAB43F826007DE50023E3E72E4679E5E1
:10F4F000503401082DE9F84320F00043B3F1485F90
:10F5000004460F46904603DAF1F7A2FD002859D0D1
:10F5100021462046F1F7D6FB21460546F1F7D2FBFE
:10F520004CF6D311C2F62E7106462846F1F7CAFBF7
:10F5300042F63471C3F2D721F1F7BAFA2946F1F74E
:10F54000C1FB4EF61B71C3F23861F1F7B3FA2946DD
:10F55000F1F7B8FB40F60151C3F65011F1F7A8FAE4
:10F560002946F1F7AFFB48F68901C3F60841F1F7E8
:10F57000A1FA8146B8F1000F27D04FF07C513846F0
:10F58000F1F7A0FB494680463046F1F79BFB014668
:10F590004046F1F78DFA2946F1F794FB3946F1F729
:10F5A00087FA4AF6AB210546C3F62A613046F1F7E1
:10F5B00089FB01462846F1F77DFA01462046F1F71E
:10F5C00077FA04462046BDE8F88301462846F1F75D
:10F5D00079FB4AF6AB21C3F62A61F1F769FA3146A5
:10F5E000F1F770FB01462046F1F764FA0446204625
:10F5F000BDE8F8830020704700210020C7F6F871AD
:10F60000704700BF2DE9F041C1F30A58A8F2FF3757
:10F61000132F82B002460B4604460D468C464FEA35
:10F62000D17635DC002F51DB4FF6FF71C0F20F01B0
:10F6300041FA07F101EA0300104324D04A081340BD
:10F640001C430BD04FF4802141FA07F125EA020553
:10F65000132F0CBF4FF0004400240D432246324CC0
:10F660002B4604EBC606D6E9004520462946F0F7AE
:10F670007FFDCDE90001DDE9000122462B46F0F7D0
:10F6800075FD02460B461046194602B0BDE8F081F2
:10F69000332F07DDB7F5806FF5D1F0F769FD02462E
:10F6A0000B46F0E7A8F213484FF0FF3121FA08F0BB
:10F6B0001042E8D042082242D0D04FF0804343FAB3
:10F6C00008F824EA020444EA0804C7E721F00040ED
:10F6D00050EA0201D7D023F07F4525F4700343EAB6
:10F6E0000204614241EA04000F4C050B4FEA5C4EF4
:10F6F00005F4002304EBC601D1E9004543EA4E437B
:10F7000020462946F0F734FDCDE90001DDE900018E
:10F7100022462B46F0F72AFD0446024621F000401F
:10F720000D4640EAC673AEE7803401082DE9F0418A
:10F7300020F00045B5F1A14F044606460DDBB5F1BA
:10F74000FF4F00F39C80002840F6DB7440F3D48028
:10F75000C3F6C9742046BDE8F0814FF6FF73C3F6C7
:10F76000DF639D4200F3A280B5F1445FC0F28E805A
:10F770004FF0FF3721462046F1F7A4FA01468046B4
:10F78000F1F7A0FA46F6D711C3F685410546F1F721
:10F7900099FA4DF65921C3F64B51F1F78BF92946E9
:10F7A000F1F790FA46F63531C3F68851F1F782F950
:10F7B0002946F1F787FA42F66E61C3F6BA51F1F7BE
:10F7C00079F92946F1F77EFA44F62511C3F612615C
:10F7D000F1F770F92946F1F775FA4AF6AB21C3F64D
:10F7E000AA61F1F767F94146F1F76CFA4AF2212173
:10F7F0008046CBF615512846F1F764FA4FF26B11AB
:10F80000C3F66E51F1F754F92946F1F75BFA48F265
:10F810009571C3F69D51F1F74BF92946F1F752FA6C
:10F8200048F63861C3F6E351F1F742F92946F1F79A
:10F8300049FA4CF6CD41C3F64C61F1F739F9294646
:10F84000F1F740FA7B1C0146404658D0F1F732F9F7
:10F850002146F1F737FA494B53F82710F1F728F909
:10F860002146F1F725F90146454850F82700F1F700
:10F870001FF9002E3DDB04462046BDE8F08101461D
:10F88000F1F718F904462046BDE8F0814FF2CA218D
:10F89000C7F24911F1F70EF94FF07E51F1F7CEFBA7
:10F8A00000283FF465AF2046BDE8F08100F06AF81B
:10F8B0004FF6FF71C3F697718D4204464FF6FF7203
:10F8C00028DCC3F62F72954246DC0146F1F7F2F8C8
:10F8D0004FF07E51F1F7ECF84FF08041054620469D
:10F8E000F1F7E8F801462846F1F7A0FA00270446A8
:10F8F00040E700F100442DE7CBF6C9742AE7F1F7A1
:10F90000D9F82146F1F7DEF901462046F1F7D0F8A3
:10F9100004461FE7C4F21B02954214DC4FF07F51EE
:10F92000F1F7C6F84FF07F5105462046F1F7CAF9C6
:10F930004FF07E51F1F7BEF801462846F1F776FA0E
:10F940000227044616E700202146CBF68070F1F727
:10F950006DFA032704460DE74FF07E51F1F7A8F842
:10F960004FF07E5107462046F1F7A4F8014638468D
:10F97000F1F75CFA01270446FCE600BF9034010869
:10F98000A034010820F00040704700BF20F0004084
:10F99000B0F1FF4FACBF002001207047F8B520F058
:10F9A0000046F50D7F3D162D014604461BDC002D5B
:10F9B000074620DB4FF6FF73C0F27F0343FA05F6DC
:10F9C00006420ED04FF2CA21C7F24911F1F772F880
:10F9D0000021F1F733FB18B1002C1BDB27EA0604EA
:10F9E00021460846F8BDB6F1FF4FFAD3F1F762F8A9
:10F9F00001460846F8BD4FF2CA21C7F24911F1F796
:10FA000059F80021F1F71AFB0028E9D0002C07DB98
:10FA10000024E5E74FF4000040FA05F56719DDE73B
:10FA20000021CBF68071002E18BF0C46D8E700BF2E
:10FA300008B902207047B0F1004FFAD0A0F50002DB
:10FA40006FF001439A4201D80420704700F1FF4152
:10FA50009942F9D94FF6FE73421EC0F27F039A42D3
:10FA600001D80320704700F100414A1E9A42F8D99C
:10FA7000B0F1FF4F05D010F5000F14BF002001209A
:10FA800070470120704700BF0020C7F6C070704764
:10FA900038B530F00044034602460D460FD0B4F1AD
:10FAA000FF4F0ED2B4F5000F11D3E40D6419FE2CF4
:10FAB00033DC002C1BDD22F0FF4141EAC453184621
:10FAC00038BD0146F0F7F6FF0346184638BD4FF043
:10FAD0009841F1F7F7F843F6B041CFF6FF718D4248
:10FAE000034612DBC0F3C7540246193CDEE714F1AB
:10FAF000160F21DA4CF25032954219460EDC44F2D0
:10FB00006020C0F6A25000F023F844F26021C0F655
:10FB1000A251F1F7D7F80346D1E719464FF2CA20B0
:10FB2000C7F2491000F014F84FF2CA21C7F2491188
:10FB3000F1F7C8F80346C2E722F0FF4304F11900C9
:10FB400043EAC0504FF04C51F1F7BCF80346B6E71A
:10FB500001F0004120F00040084370472DE9F041DA
:10FB6000274C84B025680746D5F84841002C41D081
:10FB700066681F2E1CDD234810B94FF0FF301FE0D0
:10FB80004FF4C870039102920193AFF30080039980
:10FB90000446029A019B0028EFD0D5F84861002066
:10FBA00060602660C5F84841C4F88801C4F88C013B
:10FBB000656847B9A81C013544F82010656000202D
:10FBC00004B0BDE8F081012000FA05F0D4F88861A6
:10FBD00004EB85080643022FC8F88820C4F8886122
:10FBE000C8F80831E6D1D4F88C3143EA0002C4F8F1
:10FBF0008C21DFE705F5A674C5F84841B8E700BFDA
:10FC0000B83501080000000000210A2201F028B8E0
:10FC10002DE9F84FDDF828B081468A4698469AB11A
:10FC200093B11646002503E00FD0651CAE420BD9F8
:10FC30007419640808FB04A748463946D8470028C9
:10FC4000F2DA2646AE42F3D800273846BDE8F88FF0
:10FC500040F2B053C2F2000318687047114B124AC9
:10FC600070B5981A831018D0591E02EB83040D4604
:10FC700054F8042D01F00106904775B126B154F8EF
:10FC8000040D8047013D08D054F8043D9847013DDC
:10FC900054F8041D8847013DF6D1BDE8704003F0DB
:10FCA00093BC00BFE0350108DC350108F8B5204FF2
:10FCB000204C381B871017D07A1E2368012502F0CC
:10FCC00001069847AF420FD02EB154F8041F022509
:10FCD0008847AF4208D0606880470235A268261D79
:10FCE00090470834AF42F6D1134F144C03F066FC32
:10FCF0003B1B9F1018D07D1E216805F001060125D1
:10FD00008847AF4211D02EB154F8040F0225804726
:10FD1000AF420BD0626890470235A368261D984712
:10FD20000834AF42F6D1F8BDF8BDF8BDF8BD00BF4C
:10FD3000D4350108D4350108DC350108D435010873
:10FD40000F2A2DE9F00340F2A18041EA00039B074E
:10FD500040F09E800C68A2F1100504604B68AC4630
:10FD600043608C68BCF10F0F8460CC68C5F300154C
:10FD7000C46000F1100301F110042BD975B125689E
:10FD8000ACF1100C1D6065685D60A5689D60E5685C
:10FD90001034DD601033BCF10F0F1BD9276804F15C
:10FDA00010061F60676803F110055F60A768ACF17B
:10FDB000200C9F60E768DF6024691C61776806F1AA
:10FDC00010046F60B7682033AF60F668BCF10F0FA6
:10FDD000EE60E3D8A2F1100828F00F0302F00F0440
:10FDE00003F1100C032C00EB0C0301EB0C0851D9B0
:10FDF000211F4FEA9109444608EB890C54F8046B23
:10FE0000C8EB0C010CF1040C1D46644545F8046B6D
:10FE1000C1F3800112D029B154F8041B644545F8A0
:10FE2000041B0BD0274657F8041B2E4646F8041B2C
:10FE300064686C603C1D351D6445F3D109F1010C0B
:10FE40004FEA8C0902F0030208EB09014B44D2B1DE
:10FE50000D789A18DC4303F8015B1419934204F0FF
:10FE6000010410D02CB111F8014F03F8014B93425B
:10FE700009D04D781C4604F8015B8D7802315D7025
:10FE8000631C9342F5D1BDE8F00370470346DEE7FB
:10FE90000346DDE741462246D9E700BFF0B48407B8
:10FEA000034600F08D80541E002A00F08780E5078D
:10FEB000CEB211D41A4602F8016B134615469207CA
:10FEC00010D0621E002C79D003F8016B14469A07FB
:10FED0001D4607D0013CEDE7034603F8016B9A0786
:10FEE0001D46F7D1032C52D9CEB246EA06270F2C75
:10FEF00047EA07432DD9A4F1100217460F2FC2F38A
:10FF000000162B606B60AB60EB6005F1100216D938
:10FF10003EB1103F136053609360D36010320F2FD7
:10FF20000DD9203F02F11006136053609360D36037
:10FF3000136153619361D36120320F2FF1D8A4F183
:10FF4000100222F00F0204F00F041032032C1544AB
:10FF50001DD9271F3E462A46032E42F8043BC7F30D
:10FF600080070DD927B1043E032E42F8043B07D980
:10FF7000174647F8043B083E53603A1D032EF7D856
:10FF8000231F23F00302131D04F00304ED18ACB18A
:10FF9000C9B2EA432C1905F8011BA318A54203F0C6
:10FFA00001020BD01AB105F8011BA54206D02B4661
:10FFB00003F8011B69705D1CA542F8D1F0BC7047C5
:10FFC000054614468EE700BF830770B5064614D178
:10FFD0000368A3F1013222EA030010F0803F0CD144
:10FFE000331D1A4653F8044BA4F1013525EA0404E5
:10FFF00014F0803FF5D0104600E0304603782BB176
:020000040801F1
:10000000421C147810460132002CFAD100F080F81E
:10001000304670BDC9B2F0B400294BD082070FD072
:100020000278002A71D0914242D0431C05E013F8B7
:10003000012B002A3BD091423AD09A071846F6D1BC
:10004000036841EA0127A3F1013222EA030212F018
:10005000803F47EA07471CD17B40A3F1013222EAE7
:10006000030313F0803F14D1021D02E014F0803F1F
:100070000FD1104652F8043BA3F1013687EA03047E
:1000800026EA0303A4F1013513F0803F25EA0404B6
:10009000ECD00278002A38D0914209D0431C01E00C
:1000A000914205D0184613F8012B002AF8D11046CA
:1000B000F0BC704783070BD00278002AF8D0431CAD
:1000C00003E0017801330029F2D099071846F8D1EE
:1000D0000168A1F1013323EA010212F0803F0AD145
:1000E000031D184653F8041BA1F1013424EA010250
:1000F00012F0803FF5D00378002BD9D0421C117844
:10010000104601320029FAD1D2E71046D0E700BFED
:1001100080EA0102844612F0030F4FD111F0030F61
:1001200032D14DF8044D11F0040F51F8043B0BD0BF
:10013000A3F101329A4312F0803F04BF4CF8043B14
:1001400051F8043B16D100BF51F8044BA3F1013222
:100150009A4312F0803FA4F101320BD14CF8043BDA
:10016000A24312F0803F04BF51F8043B4CF8044B0B
:10017000EAD023460CF8013B13F0FF0F4FEA33237C
:10018000F8D15DF8044B704711F0010F06D011F85B
:10019000012B0CF8012B002A08BF704711F0020F49
:1001A000BFD031F8022B12F0FF0F16BF2CF8022B34
:1001B0008CF8002012F47F4FB3D1704711F8012B57
:1001C0000CF8012B002AF9D1704700BF20F0030181
:1001D00010F00300C0F1000051F8043B00F1040CE2
:1001E0004FEACC0C6FF000021CBF22FA0CF2134352
:1001F0004FF0010C4CEA0C2C4CEA0C4CA3EB0C021B
:1002000022EA030212EACC1204BF51F8043B043084
:10021000F4D013F0FF0F1FBF013013F47F4F0130F4
:1002200013F47F0F18BF0130704700BFF0B4002AED
:1002300063D0344B04461B6814F8010B571E1D187D
:100240006E7807F0010706F00305012D58D011F86C
:10025000015B5E19767806F00306012E08BF203593
:10026000401B4BD1002D49D0013A47D02FB314F891
:10027000010B1D186E7806F00305012D11F8015BC6
:1002800008BF20305E19767806F00306012E08BFFD
:100290002035401B32D18DB3013A0ED12EE011F83A
:1002A000012B9E18767806F00306012E08BF203237
:1002B000801A23D112B36A1E20D014F8010B1D1826
:1002C0006E7806F00305012D11F8015B08BF2030A0
:1002D0005E19767806F00306012E08BF2035401B14
:1002E0000CD15DB114F8010B551E1A18567806F0A2
:1002F0000302012AD3D12030D1E71046F0BC704769
:100300002030A4E78001002041EA00039B07F0B4FD
:1003100074D1032A72D90C4654F8045B161FA5F158
:10032000013727EA050717F0803F0346C6F3800C24
:1003300031D10346032E324643F8045B2AD9BCF17F
:10034000000F0AD0214654F8045BA5F1013626EAD5
:10035000050616F0803F18D01DE0264656F8045BCF
:100360002146A5F1013727EA050717F0803F12D192
:1003700043F8045B65683146A5F1013626EA0506B7
:10038000043A0C1D16F0803F05D1043A032A43F8C5
:10039000045BE2D821467AB30D78013A03F8015B99
:1003A0009DB112F0010F1C462AD1234622B311F849
:1003B000015F013A03F8015B3DB111F8015F013AB9
:1003C00065705C1C2346002DEFD1AAB100219C185A
:1003D000DA4303F8011BA218A34202F001020BD07A
:1003E0001AB103F8011BA34206D01A4602F8011BFA
:1003F0005970531CA342F8D1F0BC70470346CAE7BA
:1004000011F8015F1C4604F8015B013A2346002DF8
:10041000CBD1DAE72DE9F00701273C4600254FF064
:10042000FF3663198B4200EB060C0DD21CF804A0BA
:1004300010F80380D0452ED201241D469F1B63195E
:100440008B4200EB060CF1D34FF0010A17605446C3
:1004500000254FF0FF3C6319994200EB0C080ED9C0
:1004600018F8048010F80390C1451AD901241D46DC
:10047000CCEB030A6319994200EB0C08F0D80CF19D
:1004800001000136B0423CBFBA463046C2F800A077
:10049000BDE8F00770470BD001272E463C46ED190A
:1004A000BFE709D04FF0010AAC4654465544D2E7A5
:1004B000BC4205D00134B4E7544505D00134CAE745
:1004C00027461D460124ACE7A2461D460124C2E78B
:1004D0002DE9F04FADF2244D1546064689461046EB
:1004E000194607AA1C46FFF795FF07AB82460DF297
:1004F0001C411A1D5C6008338B425460F9D114B35F
:1005000001232F78611E08A8A34240F8271001EAB2
:10051000030218D032B16A7802234F1EA34240F87A
:10052000227010D0B046A4465C1C15F803E0CE1A29
:100530002A5D02330F1B634540F82E6040F822709D
:10054000F2D146466446079928466918524600F09B
:1005500045FC002840F0B6800AF1FF3E05EB0E0C8A
:10056000CDF808E0CAF1010E834604F1FF38CDF85A
:100570000CC0CDF814E00746CDF810A04A4600950F
:10058000019408E027B1079FBB4201D20199CB1B20
:100590009B4400272246019CB0185C440021A21A0B
:1005A00000F07CFB002840F08780002C00F0848065
:1005B000301910F8013C08A951F82330002BE1D183
:1005C000049B9F4228BF3B46434527D2DDF800905D
:1005D00006EB0B0119F80350CA5C09EB03009542C6
:1005E00066D1DD43454415F0010F024613D00133B7
:1005F000434513D24078CD5C013285420BD057E0A1
:1006000012F8010FCD5C854252D1013312F8010F6F
:10061000CD5C85424CD101334345F1D3DDF81090D8
:10062000029B4F4528BF4B4639D2DDF808C0DDF8A4
:10063000009006EB0B0519F80C1015F80C00814220
:1006400040F0C080DDF80CE009EB070ACAEB0E01B0
:10065000C80772461ED5DDF8089009F1FF31DDF8B4
:100660000C90685C19F801CC09F1FF32844516D171
:100670000B460FE012F8019C15F800E04A1EF14508
:100680000DD10346013815F800C011F8011C614571
:1006900005D10346581E524502F1FF31EAD1013718
:1006A0009F4200F29180079F019ABB44D71B71E7DC
:1006B000DDF814E0F3446BE7002009B00DF5806D20
:1006C000BDE8F08FCAEB0400504538BF5046CAF170
:1006D0000102431C0AF1FF3C05EB0A0704F1FF3B52
:1006E000019200944A460793B1464FF000086446D1
:1006F0003E46009909EB020008EB0107BA1A0021F7
:1007000000F0CCFA0028D7D1002FD5D009EB070094
:1007100010F8013C08AA52F8230000284AD1DA4513
:1007200009EB08002AD210F80A303178994218BF34
:10073000534642D16FEA0A0303EB0B01C907324665
:10074000534618D50AF101035B4517D2324612F819
:10075000011F10F803E08E450DD02EE012F8011FA6
:1007600010F803C08C4528D1013312F8011F10F88E
:1007700003E08E4521D101335B45EFD3621C234654
:100780009BD0295D025D914213D1E10709D5631E1B
:10079000E95CC25C914204D00BE0E95CC25C91422E
:1007A00007D15A1E002B88D0A95C825C023B914283
:1007B000F3D0079880443A469BE7DDF804C0E04454
:1007C0009844F8E7049B6AE706EB0B0075E700BF67
:1007D0002DE9F04F037889B080460D46002B00F0DC
:1007E00065810A789AB184460131012602E011F848
:1007F000012B5AB1934214BF002606F001061CF8E3
:10080000013F0C46002BF2D1207820B936B140468A
:1008100009B0BDE8F08F4FF00008F8E708F10100DB
:100820002978FFF7F7FB641B06460028F3D0012C5C
:1008300000F0B580A044404594BFC0EB08070127F5
:100840001F2C06D939462A462346FFF741FE80462B
:10085000DDE7214607AA2846FFF7DCFD079903904C
:1008600069182846039A00F0B9FA002840F09980E8
:10087000DDF80CC0DDF80C900CF1FF3E05EB0E012D
:10088000C9F1010C8346CDF808E080460491CDF80B
:1008900014C03A46B146019508EB040609EB020084
:1008A0000021B21A00F0FAF90028B4D1002EB2D01B
:1008B000039B9B4528BF5B469C4227D9019D09EBC2
:1008C000030010F80820E95CE81891425FD1DD438D
:1008D0002D1915F0010F024609EB080113D0013361
:1008E0009C4213D94078CD5C013285420BD04EE05A
:1008F00012F8010FCD5C854249D1013312F8010F86
:10090000CD5C854243D101339C42F1D8DDF80CE047
:10091000029ADE4540F2CD80019B09EB0805995C07
:10092000A85C814240F0C580DDF804A0049BDA4455
:10093000CAEB0301C8071AD5029FDDF810C0791E63
:10094000685C1CF8017C0CF1FF33874214D10A4625
:100950000DE013F801EC2F5C4B1EBE450CD1024696
:1009600001382F5C11F8011CB94205D10246501E16
:10097000534503F1FF31ECD10BF1010B934500F22C
:100980009A80079A9044C2EB040B324684E7059D97
:1009900005EB080B0BEB03084FF0000BF5E7804667
:1009A00035E7DDF80CA00399CAEB0403534538BFC3
:1009B0005346CAF1010B581C06EB0A0205EB0A0864
:1009C000CDF808B03B4607904FF00009019201F1C5
:1009D000FF3B37468A4609EB0406F8180021F21A55
:1009E00000F05CF900287FF416AF002E3FF413AF3F
:1009F000544598BF07EB09002CD9DDF804E098F8BE
:100A000000001EF8093098424AD16FEA0A02111913
:100A1000C9074246534607EB090018D50AF10103FE
:100A20009C4217D9424612F8011F10F803C08C45AA
:100A30000DD036E012F8011F10F803E08E4530D1DA
:100A4000013312F8011F10F803C08C4529D101337E
:100A50009C42EFD8BBF1FF3F5B463FF4F8AE15F880
:100A60000B1010F80B20914216D11BF0010F0AD089
:100A70000BF1FF33E95CC25C914204D00CE0E95C0D
:100A8000C25C914208D15A1E002B3FF4E0AEA95C33
:100A9000825C023B9142F2D00798814433469AE748
:100AA0005346DDF808E0F1449944F7E70C46012687
:100AB000AAE6039A60E74E46C844A8E640F2B0535F
:100AC000C2F200031A6801235C3200F001B800BFD3
:100AD000F0B4002825D0074638463E780D46013749
:100AE00015F8014B3CB1A642FAD1002BF4D11760A6
:100AF00007F8013C11E0C6B13D4600E01BB915F80E
:100B0000016B0C46284614F8013B9E42F6D136B1E3
:100B1000002105F8011C1060781EF0BC70473046BB
:100B2000F9E710680028D6D1F7E716603046F4E7F9
:100B30002DE9F00F494C82B0D4F800C001900F4667
:100B40003C4614F8015B0CEB05004678274606F09E
:100B50000800C6B2002EF3D12D2D61D02B2D04BF7D
:100B6000244614F8015BB346002B41D1302D43D00D
:100B70000A239A46BBF1000F0CBF6FF000474FF0FD
:100B80000047B7FBFAF90AFB197000900020804675
:100B90000CE0303DAB421BDD461C05D0C84539D8C2
:100BA00035D00AFB0858012014F8015B0CEB050650
:100BB000767806F00407FFB2002FEAD116F003069C
:100BC00006D0012E14BF57263726AD1BAB42E3DCFF
:100BD000431C2AD0BBF1000F01D0C8F10008002A45
:100BE00031D0D0B94046116002B0BDE8F00F704777
:100BF000102BBED1302DBCD12578782D25D0582D85
:100C000023D043BB4FF0080A30255346B2E7009883
:100C10008542C6DD4FF0FF30C6E74046611EE2E781
:100C200014F8015B4FF0010B9EE7BBF1000F019937
:100C30000CBF6FF000404FF0004022230B60002AF1
:100C4000D2D0611ECFE74046CEE74FF0100A65785C
:100C5000534602348EE79A4630258BE78001002008
:100C600070B440F2B054C2F2000406460D4620684B
:100C7000134631462A4670BCFFF75ABF024B13B1E8
:100C8000024800F005B87047000000005DFC000855
:100C90000146002002460346FEF760BF8307F0B41A
:100CA000C9B200F09680531E002A00F094800278AA
:100CB0008A420BD0421CD8071AD512F0030F1046F7
:100CC0001CD01478013B01328C4211D1F0BC70472A
:100CD000002B7CD01278013B8A42F7D014F0030F2E
:100CE000204604F1010209D02478013B8C42EDD06A
:100CF00012F0030F104602F10104E9D1032B3FD992
:100D0000046841EA012545EA054585EA0407A7F19B
:100D1000013222EA07021E1F041D12F0803FC6F3B3
:100D200080072DD1032E334629D967B12668204686
:100D300085EA0602A2F1013626EA0202043412F024
:100D4000803F19D01CE020462468061D85EA040275
:100D5000A2F1013424EA020212F0803F10D134687B
:100D6000043B85EA0402A2F1013424EA0202341DA4
:100D700012F0803F304603D1043B032BE3D82046DA
:100D80005D1E23B303788B42A0D0431C0022E807EA
:100D900014D51C781846012201338C4296D0954216
:100DA000184603F1010402F102020ED01B788B42B7
:100DB0008CD020462478431C8C4287D0954218461C
:100DC00003F1010402F10202F0D100207EE718468F
:100DD0007CE7134692E7104678E700BF032AF0B499
:100DE00031D941EA00039C072ED106680F68151F10
:100DF000031D0C1DBE42C5F3800C24D1032D2A46D1
:100E00001FD9BCF1000F08D01E682568214618467E
:100E100004340433AE4211D015E0214618461C6854
:100E20000B68051D0E1D9C420DD1314628462E68CB
:100E30000D68043A031D0C1DAE4204D1043A032A86
:100E4000EBD8214618461AB303780C78A3420AD18E
:100E5000551E0022EB0714D510F8013F11F8014F81
:100E60000122A3420DD0181B10E010F8013F11F829
:100E7000014FA342F7D110F8013F11F8014FA342EF
:100E8000F1D1AA4202F10202EFD10020F0BC70477A
:100E90001046FBE71E1E646464646464000C014039
:100EA00008001002000C0140100010020008014070
:100EB000001014021048498A8B8C8D84858687FF28
:100EC0001048494A4B4C4D44454647FF20212223B8
:100ED0002425262748498A8B8C8DFF00EC0E0108BB
:100EE000C00E0108CC0E0108B40E010820212223F7
:100EF0002425262748494A4B4C4DFF000F2C00085B
:100F0000BD2B0008E12B0008A92B0008AF2B00081F
:100F1000AB2B000800000040000801400100000069
:100F2000001C00000000004000080140020000001A
:100F3000041C000000000040000801400400000004
:100F4000081C0000000000400008014008000000EC
:100F50000C1C00000004004000080140400000009C
:100F6000001D000000040040000801408000000057
:100F7000041D000000040040000C014001000000BE
:100F8000081D000000040040000C014002000000A9
:100F90000C1D0000002C0140000801400001000071
:100FA000001B0100002C0140000801400008000067
:100FB0000C1B010000080040000C01404000000034
:100FC000001E000000080040000C014080000000EE
:100FD000041E000000080040000C01400001000059
:100FE000081E000000080040000C01400002000044
:100FF0000C1E0000002C01400000004000040040D6
:10100000000800400004080CD00732003200320013
:101010003200320032003200C80064000000414556
:1010200054523132333400002965000851640008FD
:10103000F9640008AF640008676400084F640008A2
:101040000000803F00000000A8AAAA3F0000803FE7
:101050000000803F000080BFB0AA2ABF000080BF10
:101060000000803F0000803FB0AA2ABF000080BF80
:101070000000803F00000000A8AAAA3F000080BF37
:101080000000803F000080BFB0AA2ABF0000803F60
:101090000000803F0000803FB0AA2ABF0000803FD0
:1010A0000000803F00000000A8AAAA3F0000000046
:1010B0000000803F000080BFB0AA2ABF00000000EF
:1010C0000000803F0000803FB0AA2ABF000000005F
:1010D0000000803F000080BF0000803F000080BF14
:1010E0000000803F000080BF000080BF0000803F04
:1010F0000000803F0000803F0000803F0000803FF4
:101100000000803F0000803F000080BF000080BFE3
:101110000000803F00000000000000000000000010
:101120000000803F00000000000000000000000000
:101130000000803F000000000000803F0000803F72
:101140000000803F000080BF000080BF0000000062
:101150000000803F000000000000803F000080BFD2
:101160000000803F0000803F000080BF0000008042
:101170000000803F000000000000803F000080BFB2
:101180000000803F000080BF000000000000803FA2
:101190000000803F0000803F000000000000803F12
:1011A0000000803F00000000000080BF000080BF02
:1011B000000000000000000003010000A010010872
:1011C0000400000070110108040000002813010849
:1011D00002010000C8120108000100000000000028
:1011E0000600000040100108060000006812010817
:1011F000010100000000000004000000E8120108E6
:1012000006000000E8130108080000004814010867
:1012100008000000E8140108080000006813010835
:1012200001010000000000000001000000000000BB
:10123000000100000000000004000000301101085F
:1012400006000000D01001080001000000000000AE
:1012500002010000C81401080101000000000000A4
:1012600000000000000000000000803FD0B35DBF20
:101270000000003F0000803F0000803FD0B35DBF12
:10128000000000BF000080BF0000803FD0B35D3F82
:101290000000003F0000803F0000803FD0B35D3F72
:1012A000000000BF000080BF0000803F0000000081
:1012B000000080BF0000803F0000803F0000000071
:1012C0000000803F000080BF0000803F0000803FA2
:1012D00000000000000000000000803F000080BF10
:1012E00000000000000000000000803F000000003F
:1012F0000000803F000080BF0000803F000080BFF2
:10130000000080BF000000000000803F00000000DF
:101310000000803F0000803F0000803F0000803FD1
:10132000000080BF000000000000803F000080BF80
:101330000000803F000080BF0000803F000080BFB1
:10134000000080BF0000803F0000803F0000803F21
:101350000000803F0000803F0000803F0000803F91
:10136000000080BF000080BF0000803F0000803F81
:10137000000000BF0000803F0000803F000000BF71
:10138000000080BF0000803F0000803F000080BF61
:101390000000003F0000803F0000803F0000003F51
:1013A0000000803F0000803F0000803F0000003FC1
:1013B000000080BF000080BF0000803F000080BFB1
:1013C000000000BF000080BF0000803F000000BFA1
:1013D0000000803F000080BF0000803F0000803F91
:1013E0000000003F000080BF0000803F000000BF01
:1013F000D0B35D3F0000803F0000803F000000BF91
:10140000D0B35DBF0000803F0000803F0000003F80
:10141000D0B35D3F000080BF0000803F0000003F70
:10142000D0B35DBF000080BF0000803F000080BFE0
:1014300000000000000080BF0000803F0000803FEF
:10144000000000000000803F0000803F000080BFDF
:101450000000803F000080BF0000803F000080BF90
:10146000000080BF0000803F0000803F0000803F00
:101470000000803F0000803F0000803F0000803F70
:10148000000080BF000080BF0000803F000080BFE0
:101490000000803F0000803F0000803F000080BFD0
:1014A000000080BF000080BF0000803F0000803F40
:1014B0000000803F000080BF0000803F0000803FB0
:1014C000000080BF0000803F0000803F000000005F
:1014D00000000000000080BF0000803F000000000E
:1014E000000000000000803F0000803FF704353F0F
:1014F000F70435BF0000803F0000803FF70435BF90
:10150000F70435BF0000803F0000803FF70435BF7F
:10151000F704353F0000803F0000803FF704353F6F
:10152000F704353F0000803F0000803F00000000CE
:10153000000080BF000080BF0000803F000080BF2F
:1015400000000000000080BF0000803F000000009D
:101550000000803F000080BF0000803F0000803F0F
:1015600000000000000080BF24505542582C343148
:101570002C312C303030332C303030312C3131356F
:101580003230302C302A31450D0A0024504D544B56
:101590003235312C3131353230302A31460D0A00A6
:1015A00024505542582C34312C312C303030332CCF
:1015B000303030312C35373630302C302A32440D33
:1015C0000A0024504D544B3235312C3537363030EB
:1015D0002A32430D0A0024505542582C34312C3104
:1015E0002C303030332C303030312C3338343030F4
:1015F0002C302A32360D0A0024504D544B323531EE
:101600002C33383430302A32370D0A0024505542FA
:10161000582C34312C312C303030332C30303031A8
:101620002C31393230302C302A32330D0A0024501C
:101630004D544B3235312C31393230302A32320D63
:101640000A00B56206010300F00500FF19B5620645
:10165000010300F00300FD15B56206010300F0016F
:1016600000FB11B56206010300F00000FA0FB5623D
:1016700006010300F00200FC13B56206010300F04E
:101680000400FE17B562060103000102010E47B512
:1016900062060103000103010F49B5620601030060
:1016A000010601124FB562060103000112011E6717
:1016B000B5620616080003070300510800008A41BE
:1016C000B56206080600C80001000100DE6A0000DD
:1016D0000000000000C20100681501088B15010818
:1016E0000100000000E10000A0150108C21501087A
:1016F0000200000000960000D6150108F815010848
:1017000003000000004B00000C1601082E16010813
:101710000400000080250000441E0108441E01084A
:10172000414552543132333400000000672601082D
:101730006B26010870260108812601088A26010807
:1017400095260108A0260108AB2601088925010875
:10175000B426010883250108BD260108C726010813
:10176000D2260108D826010800000000B92501088A
:10177000BD250108C3250108C9250108CC2501089C
:10178000D3250108D6250108DB250108E725010836
:10179000EA250108F0250108F725010801260108BE
:1017A0000B26010814260108222601082E2601080E
:1017B000352601083B260108482601085326010862
:1017C0006026010800000000CB230108CF23010898
:1017D000C9A80008F6230108FB230108C5AD0008CD
:1017E0000F2401081824010809A70008352401085E
:1017F0003A24010811AC000869240108441E0108BC
:10180000D1A600086E24010876240108E5A5000889
:101810008A24010899240108C5A50008B3240108F9
:10182000441E0108CDA30008B8240108BC24010807
:101830001DA5000809240108D824010835A70008BF
:10184000EB240108F124010821A800080C25010857
:1018500014250108D5A7000823250108282501081B
:10186000EDA40008551D010838250108BDAA00088F
:10187000662501085A250108F9A300086D2501080D
:10188000441E0108C1A30008441E01089525010853
:101890009D250108A5250108AD250108B4250108ED
:1018A00000000000303132333435363738394142A8
:1018B000434445464748494A4B4C4D4E4F50515280
:1018C000535455565758595A004166726F33322057
:1018D000434C492076657273696F6E20322E322038
:1018E0004170722031392032303134202F20303194
:1018F0003A31323A333500417661696C61626C6528
:1019000020636F6D6D616E64733A0D0A0025730973
:1019100025730D0A0053797374656D2055707469D1
:101920006D653A202564207365636F6E64732C20A7
:10193000566F6C746167653A202564202A20302E2A
:1019400031562028256453206261747465727929A8
:101950000D0A004350552025644D487A2C206465BB
:101960007465637465642073656E736F72733A2077
:10197000002573200041434348573A202573002E29
:101980002563004379636C652054696D653A2025B1
:10199000642C20493243204572726F72733A2025BD
:1019A000642C20636F6E6669672073697A653A20DC
:1019B00025640D0A00536176696E672E2E2E000D88
:1019C0000A5265626F6F74696E672E2E2E004D7518
:1019D000737420626520616E79206F726465722075
:1019E0006F662041455452313233340D0A0043753D
:1019F0007272656E742061737369676E6D656E7463
:101A00003A20004572726F723A20456E61626C65D1
:101A100020616E6420706C756720696E204750539A
:101A20002066697273740D0A00456E61626C696E9E
:101A3000672047505320706173737468726F7567C5
:101A4000682E2E2E0D0A00456E61626C656420665C
:101A5000656174757265733A2000417661696C61E5
:101A6000626C652066656174757265733A20004921
:101A70006E76616C69642066656174757265206E4E
:101A8000616D652E2E2E0D0A0044697361626C65CE
:101A9000642000456E61626C656420000D0A4C652F
:101AA0006176696E6720434C49206D6F64652E2E08
:101AB0002E0D0A00526573657474696E6720746F29
:101AC0002064656661756C74732E2E2E0D0A0043BA
:101AD000757272656E74206D697865723A2025732F
:101AE0000D0A00417661696C61626C65206D6978F0
:101AF0006572733A2000496E76616C6964206D6985
:101B000078657220747970652E2E2E0D0A004D694D
:101B10007865722073657420746F2025730D0A0038
:101B200043757272656E742070726F66696C653A87
:101B30002025640D0A0055736167653A0D0A6D6FC3
:101B4000746F7220696E646578205B76616C756570
:101B50005D202D2073686F77205B6F722073657432
:101B60005D206D6F746F722076616C75650D0A0073
:101B70004E6F2073756368206D6F746F722C2075C3
:101B800073652061206E756D626572205B302C205C
:101B900025645D0D0A004D6F746F72202564206905
:101BA00073207365742061742025640D0A00496EEA
:101BB00076616C6964206D6F746F722076616C75EC
:101BC000652C20313030302E2E323030300D0A006E
:101BD00053657474696E67206D6F746F722025642D
:101BE00020746F2025640D0A00617578202575200A
:101BF00025750D0A00496E76616C69642046656141
